:0200000490006A
:1000000000000000000000000000000000000000F0
:1000100000000000000000000000000000000000E0
:1000200000000000000000000000000000000000D0
:1000300000000000000000000000000000000000C0
:1004000060A30024BD3F00907D360390A93F00907B
:10041000A93F0090A93F0090A93F00900000000074
:10042000000000000000000000000000F941009002
:10043000A93F009000000000954100906590009059
:10044000AD430090AD430090AD430090AD430090AC
:10045000AD430090AD430090AD430090AD4300909C
:10046000AD430090AD430090AD430090AD4300908C
:10047000AD430090AD430090AD430090AD4300907C
:1006980081F0004102E000BF83F0004330B54FEA2B
:1006A80041044FEA430594EA050F08BF90EA020F98
:1006B8001FBF54EA000C55EA020C7FEA645C7FEA2B
:1006C800655C00F0E2804FEA5454D4EB5555B8BF4E
:1006D8006D420CDD2C4480EA020281EA030382EABF
:1006E800000083EA010180EA020281EA0303362D51
:1006F80088BF30BD11F0004F4FEA01314FF4801C24
:100708004CEA113102D0404261EB410113F0004F35
:100718004FEA03334CEA133302D0524263EB4303EC
:1007280094EA050F00F0A780A4F10104D5F1200E8A
:100738000DDB02FA0EFC22FA05F2801841F10001E5
:1007480003FA0EF2801843FA05F359410EE0A5F1B9
:1007580020050EF1200E012A03FA0EFC28BF4CF0EA
:10076800020C43FA05F3C01851EBE37101F00045A0
:1007780007D54FF0000EDCF1000C7EEB00006EEBAD
:100788000101B1F5801F1BD3B1F5001F0CD3490837
:100798005FEA30004FEA3C0C04F101044FEA44528E
:1007A80012F5800F80F09A80BCF1004F08BF5FEA15
:1007B800500C50F1000041EB045141EA050130BDF5
:1007C8005FEA4C0C404141EB0101013C28BFB1F507
:1007D800801FE9D291F0000F04BF01460020B1FA52
:1007E80081F308BF2033A3F10B03B3F120020CDA25
:1007F8000C3208DD02F1140CC2F10C0201FA0CF003
:1008080021FA02F10CE002F11402D8BFC2F1200C67
:1008180001FA02F120FA0CFCDCBF41EA0C0190401D
:10082800E41AA2BF01EB0451294330BD6FEA040466
:100838001F3C1CDA0C340EDC04F11404C4F1200251
:1008480020FA04F001FA02F340EA030021FA04F363
:1008580045EA030130BDC4F10C04C4F1200220FABA
:1008680002F001FA04F340EA0300294630BD21FAF8
:1008780004F0294630BD94F0000F83F4801306BFBE
:1008880081F480110134013D4EE77FEA645C18BFB2
:100898007FEA655C29D094EA050F08BF90EA020F49
:1008A80005D054EA000C04BF1946104630BD91EA41
:1008B800030F1EBF0021002030BD5FEA545C05D144
:1008C8004000494128BF41F0004130BD14F5800483
:1008D8003CBF01F5801130BD01F0004545F0FE41F7
:1008E80041F470014FF0000030BD7FEA645C1ABF2C
:1008F800194610467FEA655C1CBF0B46024650EA63
:10090800013406BF52EA033591EA030F41F400218E
:1009180030BD00BF90F0000F04BF0021704730B514
:100928004FF4806404F132044FF000054FF00001E9
:1009380050E700BF90F0000F04BF0021704730B5AA
:100948004FF4806404F1320410F0004548BF40427F
:100958004FF000013EE700BF42004FEAE2014FEAD4
:1009680031014FEA02701FBF12F07F4393F07F4FAF
:1009780081F06051704732F07F4208BF704793F0B2
:100988007F4F04BF41F40021704730B54FF46074C5
:1009980001F0004521F000411CE700BF50EA0102C8
:1009A80008BF704730B54FF000050AE050EA010271
:1009B80008BF704730B511F0004502D5404261EBE1
:1009C80041014FF4806404F132045FEA915C3FF422
:1009D800D8AE4FF003025FEADC0C18BF03325FEABF
:1009E800DC0C18BF033202EBDC02C2F1200300FA70
:1009F80003FC20FA02F001FA03FE40EA0E0021FA95
:100A080002F11444BDE600BF70B54FF0FF0C4CF482
:100A1800E06C1CEA11541DBF1CEA135594EA0C0F34
:100A280095EA0C0F00F0DEF82C4481EA030621EA6F
:100A38004C5123EA4C5350EA013518BF52EA0335AA
:100A480041F4801143F4801338D0A0FB02CE4FF05C
:100A58000005E1FB02E506F00042E0FB03E54FF08C
:100A68000006E1FB03569CF0000F18BF4EF0010E84
:100A7800A4F1FF04B6F5007F64F5407404D25FEA80
:100A88004E0E6D4146EB060642EAC62141EA555133
:100A98004FEAC52040EA5E504FEACE2EB4F1FD0C75
:100AA80088BFBCF5E06F1ED8BEF1004F08BF5FEAF3
:100AB800500E50F1000041EB045170BD06F00046A5
:100AC80046EA010140EA020081EA0301B4EB5C0452
:100AD800C2BFD4EB0C0541EA045170BD41F480114A
:100AE8004FF0000E013C00F3AB8014F1360FDEBF6F
:100AF800002001F0004170BDC4F10004203C35DA4B
:100B08000C341BDC04F11404C4F1200500FA05F3CD
:100B180020FA04F001FA05F240EA020001F000426E
:100B280021F0004110EBD37021FA04F642EB0601E4
:100B38005EEA430E08BF20EAD37070BDC4F10C040E
:100B4800C4F1200500FA04F320FA05F001FA04F2D2
:100B580040EA020001F0004110EBD37041F10001BE
:100B68005EEA430E08BF20EAD37070BDC4F12005C9
:100B780000FA05F24EEA020E20FA04F301FA05F231
:100B880043EA020321FA04F001F0004121FA04F2D9
:100B980020EA020000EBD3705EEA430E08BF20EAA9
:100BA800D37070BD94F0000F0FD101F000464000E3
:100BB80041EB010111F4801F08BF013CF7D041EA65
:100BC800060195F0000F18BF704703F00046520069
:100BD80043EB030313F4801F08BF013DF7D043EA3A
:100BE8000603704794EA0C0F0CEA135518BF95EAF0
:100BF8000C0F0CD050EA410618BF52EA4306D1D177
:100C080081EA030101F000414FF0000070BD50EA95
:100C1800410606BF1046194652EA430619D094EA1F
:100C28000C0F02D150EA013613D195EA0C0F05D109
:100C380052EA03361CBF104619460AD181EA03015D
:100C480001F0004141F0FE4141F470014FF0000015
:100C580070BD41F0FE4141F4780170BD70B54FF0B0
:100C6800FF0C4CF4E06C1CEA11541DBF1CEA135530
:100C780094EA0C0F95EA0C0F00F0A7F8A4EB050412
:100C880081EA030E52EA03354FEA013100F0888009
:100C98004FEA03334FF0805545EA131343EA1263D2
:100CA8004FEA022245EA111545EA10654FEA002687
:100CB8000EF000419D4208BF964244F1FD0404F540
:100CC800407402D25B084FEA3202B61A65EB03059C
:100CD8005B084FEA32024FF480104FF4002CB6EB59
:100CE800020E75EB030E22BFB61A754640EA0C00D9
:100CF8005B084FEA3202B6EB020E75EB030E22BF19
:100D0800B61A754640EA5C005B084FEA3202B6EB59
:100D1800020E75EB030E22BFB61A754640EA9C0018
:100D28005B084FEA3202B6EB020E75EB030E22BFE8
:100D3800B61A754640EADC0055EA060E18D04FEAA6
:100D4800051545EA16754FEA06164FEAC30343EA46
:100D580052734FEAC2025FEA1C1CC0D111F4801F13
:100D68000BD141EA00014FF000004FF0004CB6E70C
:100D780011F4801F04BF01430020B4F1FD0C88BFAB
:100D8800BCF5E06F3FF6AFAEB5EB030C04BFB6EBB6
:100D9800020C5FEA500C50F1000041EB045170BDA9
:100DA8000EF0004E4EEA113114EB5C04C2BFD4EBD6
:100DB8000C0541EA045170BD41F480114FF0000E5A
:100DC800013C90E645EA060E8DE60CEA135594EAD6
:100DD8000C0F08BF95EA0C0F3FF43BAF94EA0C0FD9
:100DE8000AD150EA01347FF434AF95EA0C0F7FF44E
:100DF80025AF104619462CE795EA0C0F06D152EAA2
:100E080003353FF4FDAE1046194622E750EA410685
:100E180018BF52EA43067FF4C5AE50EA41047FF496
:100E28000DAF52EA43057FF4EBAE12E74FF0FF3CFB
:100E380006E000BF4FF0010C02E000BF4FF0010CCC
:100E48004DF804CD4FEA410C7FEA6C5C4FEA430C45
:100E580018BF7FEA6C5C1BD001B050EA410C0CBF94
:100E680052EA430C91EA030F02BF90EA020F0020F6
:100E7800704710F1000F91EA030F58BF994208BF5D
:100E880090422CBFD8176FEAE37040F0010070471A
:100E98004FEA410C7FEA6C5C02D150EA013C07D171
:100EA8004FEA430C7FEA6C5CD6D152EA033CD3D0BC
:100EB8005DF8040B704700BF8446104662468C46B6
:100EC8001946634600E000BF01B5FFF7B7FF0028E9
:100ED80048BF10F1000F01BD4DF808EDFFF7F4FF12
:100EE8000CBF012000205DF808FB00BF4DF808ED9D
:100EF800FFF7EAFF34BF012000205DF808FB00BFC0
:100F08004DF808EDFFF7E0FF94BF012000205DF8E1
:100F180008FB00BF4DF808EDFFF7CEFF94BF012096
:100F280000205DF808FB00BF4DF808EDFFF7C4FF8F
:100F380034BF012000205DF808FB00BF4FEA4102E2
:100F4800B2F1E04324BFB3F5001CDCF1FE5C0DD91F
:100F580001F0004C4FEAC0024CEA5070B2F1004F69
:100F680040EB830008BF20F00100704711F0804F6C
:100F780021D113F13872BCBF01F00040704741F431
:100F880080114FEA5252C2F11802C2F1200C10FA35
:100F98000CF320FA02F018BF40F001004FEAC12319
:100FA8004FEAD32303FA0CFC40EA0C0023FA02F3BD
:100FB8004FEA4303CCE77FEA625307D150EA013393
:100FC8001EBF4FF0FE4040F44000704701F0004063
:100FD80040F0FE4040F40000704700BF80F0004041
:100FE80002E000BF81F0004142001FBF5FEA4103F9
:100FF80092EA030F7FEA226C7FEA236C6AD04FEAF9
:101008001262D2EB1363C1BFD2184140484041403D
:10101800B8BF5B42192B88BF704710F0004F40F4EF
:10102800000020F07F4018BF404211F0004F41F40B
:10103800000121F07F4118BF494292EA030F3FD0D7
:10104800A2F1010241FA03FC10EB0C00C3F12003EA
:1010580001FA03F100F0004302D5494260EB400079
:10106800B0F5000F13D3B0F1807F06D340084FEAE4
:10107800310102F10102FE2A51D2B1F1004F40EBD9
:10108800C25008BF20F0010040EA03007047490041
:1010980040EB0000013A28BFB0F5000FEDD2B0FADE
:1010A80080FCACF1080CB2EB0C0200FA0CF0AABF01
:1010B80000EBC25052421843BCBFD040184370479F
:1010C80092F0000F81F4000106BF80F400000132A5
:1010D800013BB5E74FEA41037FEA226C18BF7FEA7C
:1010E800236C21D092EA030F04D092F0000F08BFBE
:1010F8000846704790EA010F1CBF0020704712F0A5
:101108007F4F04D1400028BF40F00040704712F1E3
:1011180000723CBF00F50000704700F0004343F048
:10112800FE4040F4000070477FEA226216BF08467E
:101138007FEA23630146420206BF5FEA412390EA41
:10114800010F40F4800070474FF0000304E000BF37
:1011580010F0004348BF40425FEA000C08BF7047E8
:1011680043F0964301464FF000001CE050EA0102AC
:1011780008BF70474FF000030AE000BF50EA0102C1
:1011880008BF704711F0004302D5404261EB4101AE
:101198005FEA010C02BF84460146002043F0B643D3
:1011A80008BFA3F18053A3F50003BCFA8CF2083AF8
:1011B800A3EBC25310DB01FA02FC634400FA02FC01
:1011C800C2F12002BCF1004F20FA02F243EB020008
:1011D80008BF20F00100704702F1200201FA02FC6A
:1011E800C2F1200250EA4C0021FA02F243EB02005D
:1011F80008BF20EADC7070474FF0FF0C1CEAD052A1
:101208001EBF1CEAD15392EA0C0F93EA0C0F6FD061
:101218001A4480EA010C400218BF5FEA41211ED03F
:101228004FF0006343EA501043EA5111A0FB01312B
:101238000CF00040B1F5000F3EBF490041EAD37100
:101248005B0040EA010062F17F02FD2A1DD8B3F17C
:10125800004F40EBC25008BF20F00100704790F0EB
:10126800000F0CF0004C08BF49024CEA502040EA3D
:1012780051207F3AC2BFD2F1FF0340EAC250704703
:1012880040F400004FF00003013A5DDC12F1190F41
:10129800DCBF00F000407047C2F10002410021FAB3
:1012A80002F1C2F1200200FA02FC5FEA310040F1CB
:1012B800000053EA4C0308BF20EADC70704792F044
:1012C800000F00F0004C02BF400010F4000F013A7C
:1012D800F9D040EA0C0093F0000F01F0004C02BF77
:1012E800490011F4000F013BF9D041EA0C018FE7E6
:1012F8000CEAD15392EA0C0F18BF93EA0C0F0AD0EC
:1013080030F0004C18BF31F0004CD8D180EA010011
:1013180000F00040704790F0000F17BF90F0004FAA
:10132800084691F0000F91F0004F14D092EA0C0F8C
:1013380001D142020FD193EA0C0F03D14B0218BF1F
:10134800084608D180EA010000F0004040F0FE4065
:1013580040F40000704740F0FE4040F44000704701
:101368004FF0FF0C1CEAD0521EBF1CEAD15392EA80
:101378000C0F93EA0C0F69D0A2EB030280EA010C70
:1013880049024FEA402037D04FF0805343EA111109
:1013980043EA10130CF000408B4238BF5B0042F167
:1013A8007D024FF4000C8B4224BF5B1A40EA0C000C
:1013B800B3EB510F24BFA3EB510340EA5C00B3EB3E
:1013C800910F24BFA3EB910340EA9C00B3EBD10F2C
:1013D80024BFA3EBD10340EADC001B0118BF5FEA7E
:1013E8001C1CE0D1FD2A3FF650AF8B4240EBC250A7
:1013F80008BF20F0010070470CF0004C4CEA502068
:101408007F32C2BFD2F1FF0340EAC250704740F4B6
:1014180000004FF00003013A37E792F0000F00F0A8
:10142800004C02BF400010F4000F013AF9D040EA26
:101438000C0093F0000F01F0004C02BF490011F4BA
:10144800000F013BF9D041EA0C0195E70CEAD153B2
:1014580092EA0C0F08D142027FF47DAF93EA0C0F99
:101468007FF470AF084676E793EA0C0F04D14B027D
:101478003FF44CAF08466EE730F0004C18BF31F02F
:10148800004CCAD130F000427FF45CAF31F0004329
:101498007FF43CAF5FE700BF4FF0FF3C06E000BFC2
:1014A8004FF0010C02E000BF4FF0010C4DF804CDE5
:1014B8004FEA40024FEA41037FEA226C18BF7FEAF5
:1014C800236C11D001B052EA530C18BF90EA010FF7
:1014D80058BFB2EB030088BFC81738BF6FEAE17086
:1014E80018BF40F0010070477FEA226C02D15FEA22
:1014F800402C05D17FEA236CE4D15FEA412CE1D08E
:101508005DF8040B704700BF844608466146FFE754
:101518000FB5FFF7C9FF002848BF10F1000F0FBD36
:101528004DF808EDFFF7F4FF0CBF012000205DF82F
:1015380008FB00BF4DF808EDFFF7EAFF34BF0120B4
:1015480000205DF808FB00BF4DF808EDFFF7E0FF4D
:1015580094BF012000205DF808FB00BF4DF808ED9E
:10156800FFF7D2FF94BF012000205DF808FB00BF01
:101578004DF808EDFFF7C8FF34BF012000205DF8E3
:1015880008FB00BF4FEA40024FEA41037FEA226CA2
:1015980002D15FEA402C08D17FEA236C02D15FEACE
:1015A800412C02D14FF0000070474FF00100704706
:1015B8004FEA4002B2F1FE4F0FD34FF09E03B3EB58
:1015C80012620DD94FEA002343F0004310F0004F98
:1015D80023FA02F018BF404270474FF000007047EE
:1015E80012F1610F01D1420205D110F0004008BF8D
:1015F8006FF0004070474FF00000704742000ED275
:10160800B2F1FE4F0BD34FF09E03B3EB126209D435
:101618004FEA002343F0004323FA02F070474FF0EB
:101628000000704712F1610F01D1420202D14FF060
:10163800FF3070474FF00000704700BF7BB972B9A8
:101648000029BEBF00204FF0004106E008BF002877
:101658001CBF6FF000414FF0FF3000F057B8ADF1FC
:10166800080C6DE904CE002909DB002B1ADB00F019
:1016780069F8DDF804E0DDE9022304B07047404270
:1016880061EB4101002B1BDB00F05CF8DDF804E0A6
:10169800DDE9022304B0404261EB4101524263EBB1
:1016A80043037047524263EB430300F04BF8DDF805
:1016B80004E0DDE9022304B0404261EB41017047D8
:1016C800524263EB430300F03DF8DDF804E0DDE946
:1016D800022304B0524263EB4303704753B94AB93B
:1016E800002908BF00281CBF4FF0FF314FF0FF3022
:1016F80000F00CB8ADF1080C6DE904CE00F022F84A
:10170800DDF804E0DDE9022304B07047704700BF4C
:1017180010F8012B11F8013B012A28BF9A42F7D093
:10172800D01A7047034611F8012B03F8012B002A41
:10173800F9D17047034613F8012B002AFBD1181A78
:10174800013870472DE9F04786468C460846089EC2
:10175800154674461946002B40F0C2808542B2FAFD
:1017680082F245D94AB1C2F1200300FA02FC2EFAEE
:1017780003F3954043EA0C0C94404FEA154EA8B287
:10178800BCFBFEF8230C0EFB18CC08FB00F943EA5F
:101798000C43994528D9EB1808F1FF3704D299452D
:1017A80002D9A8F102072B44A3EB0903A4B2B3FBA7
:1017B800FEFC0EFB1C330CFB00F044EA0344A04281
:1017C80014D92C190CF1FF3304D2A04202D9ACF180
:1017D80002032C44241A43EA07401EB1D4400023D4
:1017E80034607360BDE8F0874746DDE76346F1E79C
:1017F80092BB431B01214FEA154EAFB2B3FBFEFC6F
:10180800200C0EFB1C330CFB07F840EA03439845F9
:1018180062D9EB180CF1FF3004D2984502D9ACF12B
:1018280002002B44A3EB0803A4B2B3FBFEFC0EFB9F
:101838001C330CFB07F744EA0344A7424ED92C1982
:101848000CF1FF3304D2A74202D9ACF102032C44B5
:10185800E41B43EA0040C0E7C2F1200320FA03F189
:10186800954090402EFA03F303434FEA154EAFB26A
:10187800B1FBFEFC0EFB1C10190C0CFB07F841EA2F
:101888000041884504FA02F422D969180CF1FF30A6
:1018980004D2884502D9ACF102002944A1EB080121
:1018A8009BB2B1FBFEFC0EFB1C110CFB07F743EAD5
:1018B80001439F420ED9EB180CF1FF3104D29F422D
:1018C80002D9ACF102012B44DB1B41EA004192E74B
:1018D8006046E3E76146F7E76046A3E76346B7E794
:1018E800834206D916B9002108467BE7C6E900E01D
:1018F800F9E7B3FA83F78FB9834201D3724508D861
:10190800BEEB020460EB030301209C461EB90021D4
:1019180068E73846FAE7C6E9004CF8E7C7F1200C53
:10192800BB4022FA0CF41C432EFA0CF120FA0CF3FB
:10193800B84001434FEA14490EFA07F5B3FBF9F82A
:101948001FFA84FE09FB18300B0C08FB0EFA43EA59
:1019580000439A4502FA07F240D9E31808F1FF302C
:1019680004D29A4502D9A8F102002344A3EB0A0342
:1019780089B2B3FBF9F809FB183308FB0EFE41EAFC
:1019880003418E452CD9611808F1FF3304D28E45E6
:1019980002D9A8F10203214443EA0040A0FB0298BF
:1019A800A1EB0E014145CE46434602D306D14D4533
:1019B80004D2B9EB020E68EB04030138002EA6D05E
:1019C800B5EB0E0261EB030101FA0CFC22FA07F3F6
:1019D8004CEA0303F940C6E9003198E74046C5E7F9
:1019E8004346D9E7000000002DE9F04390F8A53000
:1019F80085B004460D4623B94FF07E50FFF7F2FA42
:101A08000546D4F884202E4B9A4212D12846FEF778
:101A1800A3FF29A3D3E90023FFF786FA011E04F1E7
:101A2800840018BF01210CF01BFE0120C4F8985057
:101A380005E0B4F89C30B3F5807F03D1002005B0F1
:101A4800BDE8F08304F15009484624F059F900280C
:101A5800F4D01C492846FFF7CFFB94F89C60FFF7A9
:101A6800CDFD94F88080C3B2276E206DB8F1000FC9
:101A78000DD08DF80D30022301220021009303AB15
:101A88008DF80C60B84748463FF031FCCDE78DF83B
:101A98000B60012641468DF80C3032460DF10B03E0
:101AA8000096B847009603AB276E42463146206D34
:101AB800E8E700BFAFF30080AE47E17A14AEEF3F2E
:101AC80038F5049000007F4330F000422DE9F84FCC
:101AD8000146034604D1BDE8F84F012030F08EB826
:101AE800002803DABDE8F84F30F090B8B0F1FF4FA6
:101AF80003DBFFF779FABDE8F88FB0F5000F35DAA8
:101B08004FF09841FFF778FB6FF018020346C3F3D4
:101B18001604DE15764B234403F400007F3E80F064
:101B28007E5016444FF07E51204306EBD356FFF704
:101B380059FA704B04F10F0213400546002B3ED1B1
:101B48000021FFF7EDFC98B1002E00F0C880304668
:101B5800FFF7FEFA68490546FFF74EFB674904465A
:101B68002846FFF749FB01462046C2E70022CEE798
:101B78005DA1D1E90001FFF7E1F92946FFF73CFB38
:101B880001464FF07C50FFF72DFA294604462846B7
:101B9800FFF732FB01462046FFF72EFB04460EB93D
:101BA80021466FE03046FFF7D3FA53490746FFF75F
:101BB80023FB524906463846FFF71EFB72E04FF0FA
:101BC8008041FFF711FA01462846FFF7C9FB814615
:101BD8003046FFF7BDFA494680464846FFF70CFBFA
:101BE80001468246FFF708FB4549DFF818B107466A
:101BF800FFF702FB4449FFF7F7F93946FFF7FCFA0C
:101C08004249FFF7F1F93946FFF7F6FA4049FFF77D
:101C1800EBF95146FFF7F0FA3E4982463846FFF79E
:101C2800EBFA3D49FFF7E0F93946FFF7E5FA3B499A
:101C3800FFF7DAF93946FFF7DFFA01465046FFF7B2
:101C4800D3F9C4F55713A34403F5227343EA0B03EE
:101C5800002B074630DD4FF07C512846FFF7CCFAC1
:101C68002946FFF7C9FA014604463846FFF7BCF98A
:101C78004946FFF7C1FA074646B901462046FFF72D
:101C8800B1F901462846FFF7ADF934E71A4940464D
:101C9800FFF7B2FA194906464046FFF7ADFA39464A
:101CA800FFF7A2F901462046FFF79CF92946FFF7FE
:101CB80099F901463046E6E701462846FFF792F9CA
:101CC8004946FFF799FA0446002E3FF469AF0A49DE
:101CD8004046FFF791FA0949064640466CE700205E
:101CE80009E700BFAFF30080555555555555D53F09
:101CF80020FB4A00F0FF7F008071313FD1F7173792
:101D08009788173E305CCFFF25333A3E2549923EEF
:101D1800ABAA2A3F4FD01C3E298E633ECDCCCC3E89
:101D28002DE9F04F31F0004387B080460F468146D9
:101D38000C460ED180F480094FEA490919F5000FC5
:101D480040F2618239464046FFF74EF907B0BDE8D8
:101D5800F08F20F00046B6F1FF4F02D8B3F1FF4FE5
:101D680008D9B9F17E5FEDD184F48004640014F5DC
:101D7800000FE5E7002832463DDAB3F1974F1BD351
:101D8800B3F1FF4F3AD00225B4F17C5F4DD1B9F1E0
:101D9800000F80F29780B6F1FF4F28F0004040F026
:101DA8004982A6F17E562E4340F0A080404607B0F7
:101DB800BDE8F04F2FF02ABFB3F17E5F2ED3D915BF
:101DC800C1F1960143FA01F505FA01F18B423BD1C5
:101DD800B3F17E5F4AD1002C80F293800021404607
:101DE800FFF79EFB00284FD04FEAD97007B0BDE837
:101DF800F04F2FF003BFB3F1FF4F3CD1B6F17E5F38
:101E080000F0018204D9002CC0F2008238469DE718
:101E1800002C80F2FB8107F1004097E7B1F1804F79
:101E280038D0B1F17C5F53D0002529F04041B1F1A1
:101E38007E5F28F000403BD1002C32DA01464FF09B
:101E48007E50FFF78DFA2CE0B3F17E5FC3D00025FA
:101E5800B4F1804FE9D1B6F1BF4F1DD2B6F1D05FD2
:101E680024D941464046FFF7C7F96FE705F0010559
:101E7800C5F10205ECE7B3F17E5FACD0B1F1804F5C
:101E88004FF00005E7D07FE741464FF07E50FFF75F
:101E980067FA5BE70025DEE7B6F1FF4F28F0004060
:101EA80031D1B9F1000FBFF651AF7AE728F0004001
:101EB8004EBB002C22DAB9F1000F1DDA6B1E584216
:101EC800584193E7404607B0BDE8F04F45F09ABC4B
:101ED800B6F1FF4F20F000403FF438AFB6F17E5F17
:101EE8003FF464AF002E3FF431AF5FE7012D7FF47C
:101EF8002DAF00F1004029E7304677E7012D7FF448
:101F080025AF404622E74FEAD971013902912943AA
:101F18003FF44CAFB3F19A4F40F29981604B9E4227
:101F280007D8002C0ADA002007B0BDE8F04F2FF0E0
:101F38005DBE5C4B9E4207D9002CF4DC002007B044
:101F4800BDE8F04F45F0BDBC4FF07E51FFF74AF8B1
:101F580055490646FFF750F9544980463046FFF781
:101F68004BF981464CA1D1E90001FEF7E7FF4FF09C
:101F78007A5182463046FFF73FF901465046FFF74F
:101F880031F83146FFF738F901464FF07C50FFF73A
:101F980029F8314682463046FFF72EF90146504669
:101FA800FFF72AF94249FFF727F901464846FFF7A4
:101FB80019F8014606464046FFF716F820F47F6BED
:101FC8002BF00F0B41465846FFF70CF801463046F8
:101FD800FFF708F824F47F64029B013D24F00F0406
:101FE8001D430646214638460CBF324D4FF07E55FC
:101FF800FEF7F8FF5946FFF7FFF8394680463046A6
:10200800FFF7FAF801464046FEF7EEFF214606467E
:102018005846FFF7F1F8014607463046FEF7E4FF59
:1020280000280446804620F0004320DDB3F1864FA7
:102038000BD900212846FFF77DFA003818BF012088
:1020480072E700210EE1012221E139D11A49304617
:10205800FEF7CAFF394681462046FEF7C3FF014610
:102068004846FFF785FA0028E3D186232DE0134A76
:10207800934207D900212846FFF75CFA003818BFB9
:1020880001205CE71CD13946FEF7ACFF3146FFF76B
:1020980065FA0028E9D0EDE7E13D55555555D53F9E
:1020A800F3FF7F3F0700803F00AAB83F70A5EC36DA
:1020B8003BAAB83F000080BF3CAA38330000164353
:1020C800B3F17C5F40F29B80DB157E3B4FF400044C
:1020D8001C414444C4F3C7534D497F3B1941214037
:1020E800C4F31604C3F1170344F400041C41B8F107
:1020F800000F3846B8BF6442FEF774FF0746314602
:102108003846FEF771FF20F47F6828F00F08414930
:102118004046FFF771F8394681464046FEF762FFB0
:1021280001463046FEF75EFF3B49FFF765F83B493D
:1021380006464046FFF760F801463046FEF754FF72
:10214800074601464846FEF74FFF49460646FEF752
:1021580049FF01463846FEF745FF3146804630467E
:10216800FFF74AF82E490746FFF746F82D49FEF7CC
:1021780039FF3946FFF740F82B49FEF735FF394656
:10218800FFF73AF82949FEF72DFF3946FFF734F8EB
:102198002749FEF729FF3946FFF72EF80146304652
:1021A800FEF720FF074601463046FFF725F84FF0B7
:1021B800804181463846FEF715FF01464846FFF73D
:1021C800CFF8414607463046FFF716F84146FEF776
:1021D8000BFF01463846FEF705FF3146FEF702FFC2
:1021E80001464FF07E50FEF7FDFE00EBC453B3F5F9
:1021F800000F06DA21462FF09BFC294633E600241F
:102208007DE71846F9E74FF07E509FE500209DE5F1
:10221800000080FF0072313F1872313F8CBEBF351D
:102228004CBB31330EEADD3555B38A38610B363B8A
:10223800ABAA2A3EB6F17E5F3FF4B3AD002E3FF461
:102248005DAE002D3FF4B2AD00230225029319F0D4
:10225800FF4F7FF4F6AE4FF09741FEF7CDFF6FF0DA
:1022680017010246D3157F3B0B440393804BC2F3FF
:1022780016029A4242F07E5608DD7E4B9A427FF75C
:10228800E2AE039B01330393A6F5000600227A4BC6
:10229800049253F822B030465946FEF7A3FE314661
:1022A80081465846FEF7A0FE01464FF07E50FFF7E4
:1022B80057F8014605904846FEF79EFF6F49019082
:1022C800019B049AB24601EA660646F0005623F4DA
:1022D8007F6806F5800606EB425628F00F0841464F
:1022E8003046FEF789FF01464846FEF77BFE594611
:1022F80081463046FEF776FE01465046FEF772FEEE
:102308004146FEF779FF01464846FEF76BFE059BFE
:102318001946FEF771FF019983460846FEF76CFFE0
:1023280057490646FEF768FF5649FEF75DFE3146F7
:10233800FEF762FF5449FEF757FE3146FEF75CFF91
:102348005249FEF751FE3146FEF756FF5049FEF757
:102358004BFE3146FEF750FF4E49FEF745FE31462B
:1023680081463046FEF748FF01464846FEF744FFDF
:10237800414606460198FEF737FE5946FEF73CFFF0
:102388003146FEF731FE414681464046FEF734FFAE
:1023980041498246FEF728FE4946FEF725FE20F40D
:1023A8007F6626F00F0641463046FEF725FF3A497C
:1023B80080463046FEF716FE5146FEF713FE0146EC
:1023C8004846FEF70FFE0199FEF716FF3146814693
:1023D8005846FEF711FF01464846FEF705FE8246BD
:1023E80001464046FEF700FE20F47F6626F00F0601
:1023F8002A493046FEF700FF414681463046FEF73F
:10240800F1FD01465046FEF7EDFD2549FEF7F4FEC5
:10241800244980463046FEF7EFFE01464046FEF767
:10242800E3FD049A204B019253F82210FEF7DCFDDD
:1024380006460398FEF78CFE1C4B019A53F822A01F
:10244800804631464846FEF7CFFD5146FEF7CCFDA3
:102458004146FEF7C9FD20F47F6B2BF00F0B414678
:102468005846FEF7BFFD5146FEF7BCFD4946ABE5B1
:1024780071C41C00D6B35D00A024059000F0FFDFF6
:1024880042F1533E55326C3E05A38B3EABAAAA3EA1
:10249800B76DDB3E9A99193F000040400040763FF7
:1024A8004F38763FC623F6B89024059098240590B7
:1024B8002DE9F04F91B0840705460E46009302F0CF
:1024C8000403DDF868800293C2F3C203039203F1A8
:1024D8000103059340F0BA81041D30B1072909D8DA
:1024E8006FF01B0011B0BDE8F08F01F0070634440F
:1024F800C6F10806009B4FF000094FF0040A591E68
:102508004FF0FF334F46CB4601935346CDF810901A
:102518000DB1009A22600598002800F3E8809848D9
:10252800009A824203D397488242C0F0E080039A1F
:10253800A4EB050E92074FEA9E0000F103810F2FCE
:1025480000F2B180002D00F0058107F140020DEB8B
:10255800020C019A0CF8200C0CF8102C049801308D
:102568000490E7E07A285DD84B280ED8472859D838
:1025780029282DD8252852D054D820287AD0233875
:10258800D0F1000B4BEB000B74E04C382E2849D8E7
:10259800DFE800F0704848484848484848484848F4
:1025A8004B484848484848484859484B4B59595956
:1025B800704B6D487048184B184848827F4B484804
:1025C8004B487F0000204FF0000B4FF0040A38E022
:1025D8002A380122C0B202FA00F010EA0E0F49D1DF
:1025E80010F0625C2FD110EA020B43D06046013C28
:1025F8005444B4FBFAF40AFB04F4002D61D0A3EBB5
:10260800050CA444B4453FF66BAF002868D1042BF1
:1026180047D158F8043B2360043404232AE0019A84
:10262800013A01924FF0000B24E011F8010C6C28DC
:1026380034D111F8023C00206C2B8346C5D14FF0F1
:10264800080A5346D3E708F10708073428F00708B3
:1026580024F00704F8E802AB35B106982044B042EC
:102668003FF63EAFC4E900AB08344FF0000B4FF023
:10267800080A534611F8010F002878D0BBF1000F63
:102688007FF470AF2528F5D1019B4FF0010B013382
:1026980001934FF0040AECE7584694E7002083467C
:1026A800A5E7082B02D06FF015001BE708F1070813
:1026B80028F00708F8E80223C4E9002308340823AF
:1026C800D8E768B9042B02D108F10408A4E7082B5D
:1026D800E9D108F1070828F0070808F10808EDE72C
:1026E800059A013A059258F8042B009210E7039ACC
:1026F800900720D5A4EB050E4FF0010C4FEA9E0081
:10270800BEF5007FCFD20F2FCDD8F5B107F140022B
:10271800C0B20DEB020E019A0EF8200C0EF8102C28
:10272800BCF1000F3FF41AAF60F07F0009F1010916
:102738000EF8200C0137C5F1080204344FF6DA7E92
:10274800069297E74FF0000CDAE7BCF1000F01D0D2
:102758000136EFE7029802360028EBD10098CDE960
:102768000631FEF7E7FF0644DDE90631E2E7631BC1
:10277800B3F5806F97D23DB9A6F10804E018B1E629
:10278800F078049084A305909B08029A28602B7027
:102798009DF81030C2B1EB7085F80290B9F1000FC6
:1027A80005D008A80022C5F1010C97420ED1C5F149
:1027B80001030DF120084FF0000A0DF1300B0193D1
:1027C800574512D1601B8DE66B70E5E710F8013BA9
:1027D800190608D50CEB040E03F07F03B6453FF647
:1027E8007FAE04F8013B0132DFE7B9F1000F03D0F7
:1027F80098F90020002A17DB029BD3B11AF80B20A6
:1028080004F8012B0022019B18191044B0423FF62E
:1028180067AE98F80000009904F8010B204603926F
:1028280044F00FFF039A14440AF1010A08F1010861
:10283800C6E798F8002055F822300093029B0098CC
:1028480045F82230FEF776FF421CDCE76FF00D00FA
:1028580048E600BF2DE9F04F97B00446894600AF1F
:1028680090F802A0D7F880B03B62CBF3C003FA62BD
:10287800BB6141B9457800780AEB800020444D459A
:1028880017D8A0EB0409E378FB61BAF1000F02D076
:102898001BF0010F16D1FB6953BBFB6A1BB13A6AE7
:1028A8004946204698474D4628465C37BD46BDE810
:1028B800F08F461C09F101093046FEF73BFF013055
:1028C8003044DCE72378626899007A62FA6A7961B1
:1028D80004EB8301002A40F000814D460E4601EBCF
:1028E8000A094FF000084E454CD101EB0A0610E0EA
:1028F8001BF0020FD1D023789A0004EB83017A6190
:1029080062687A62FA6A002A77D14D4601EB0A06B4
:1029180090461BF0050F0CBF02230123FB62FB69E5
:1029280006EB430A0BF00203BB625645BCD016F80F
:10293800021B16F8013C54F82390994B994502D391
:10294800984B994536D3BB69002B40D0786A30F054
:10295800D4F900283BD0E9468AB06A46924B5361C5
:102968007B6AC2E906314FF4007313848F4B42F837
:10297800103F00234FF412518D48023D00F0B4FC83
:10298800CD46D2E716F8013BF96254F82300FEF76A
:10299800D1FED7F884300130F96A4BB1D7F88830C6
:1029A80098453EBFD7F8843023F8180008F101088D
:1029B800054498E7BB6923B1786A30F09EF900288E
:1029C800C9D11BF0010F05D1FB6AED1AADE7BB6A4F
:1029D800002BAAD04846FEF7ADFED7F8843053B195
:1029E800D7F8883098453FBF431CD7F8842022F891
:1029F800183008F10108054497E7BAF1000F72D0C2
:102A08001BF0040672D0D046002607F14800524653
:102A18003B61B96244F015FEB96A3B6901EB0A02F1
:102A2800F969BA62FA695200FA60BA6A02EB4102BD
:102A38003A610BF00202BA603A69B96A8A4257D120
:102A48001BF0020F62780CBF4FEA580100217A622E
:102A58001BF0010F3244D2B240F09F801BF0040FEC
:102A680014BF40460020BB616270A0702046E17030
:102A78003A6A7969FB6A9847051EFFF615AFBB6984
:102A880041463A6A07F1480023707B6A84F802A03D
:102A98006370FB69E370FB6A9847B0F10008C0F205
:102AA800BB807B69A9EB0A013A6AC91AFB68C91A93
:102AB800D7E90A0398470028C0F2B080A8444FF02D
:102AC800000B07F1380A08EB0005B34572D3002163
:102AD8003A6AFB6A08469847E6E656464FF0000809
:102AE80007F1380093E75646D04697E7B04695E792
:102AF800BA6A12F8021B12F8015CBA6254F825008F
:102B0800274A904202D3274A90421ED3BA6932B16B
:102B1800786A7B6030F0F1F87B6800288CD1BA685D
:102B280002BB08F1280207F1300C08F1010008F196
:102B38000208944407F158025FFA88F852FA80F0C4
:102B48000CF8101C00F8105C76E7BA693AB1786A9C
:102B58007B6030F0D2F87B6800287FF46DAF1BF003
:102B6800010F09D006F1280207F13000711C161870
:102B780006F8205CCEB25FE71BF0040F3FF45CAFB1
:102B880008F1280207F1300008F1010102EB000802
:102B980008F8105C5FFA81F84EE7002063E700BF91
:102BA800F078049084A30590802E0590040000011D
:102BB800A07D04901BF80A3054F8239087F837302A
:102BC800D7F884302BB3D7F888309B4521D2D7F873
:102BD800843033F81B803A6A012107F13700FB6A19
:102BE800984700281ADB0544B8F1000F06D148467B
:102BF800FEF7A0FD00F101081FFA88F83A6A41467D
:102C08004846FB6A9847002808DB05440BF1010B8E
:102C18005BE74FF00008DEE7454645E6054643E634
:102C2800014B1860704700BF3000002480B505468E
:102C38000E461746984608F0A9FEDFF8209003468E
:102C480001F0C2FB0446424649F800303946304696
:102C5800A84754F8090001F083FA00BF08000000F3
:102C6800044608B5EFF31183102383F31288BFF3EA
:102C78006F8F01F0DDFB01F037FC32F00DFA2046D2
:102C880001F0C2F9024830F05FF830F010FDFCE7BF
:102C9800342F0590054B00205A6822F002025A6032
:102CA8005A6822F001025A60704700BF0010005CA9
:102CB800EFF31180102383F31288BFF36F8F094B52
:102CC8001A683AB9084A116841F4807111601168AC
:102CD800C905FCD51A6801321A6080F31188BFF360
:102CE8006F8F7047AC1F00240048025810B5EFF3EF
:102CF8001184102383F31288BFF36F8F134B1A6864
:102D0800C2B9134B0122BFF35B8F53E8001F0029A0
:102D180003D143E800200028F7D1BFF35B8F04D12B
:102D28000C4A02210C4830F041FB84F31188BFF3B0
:102D38006F8F10BD012A04D108490A6822F48072F5
:102D48000A601A68013A1A60EFE700BFAC1F002456
:102D5800A81F0024682F0590307E04900048025870
:102D680008B501F0A7FB01F035FB0C4B0C4A1A60C3
:102D78000C4AD36823F0070343F00203D3600A4BDD
:102D88001A6841F20303B3EB124F06D1074AD2F88F
:102D9800083143F00103C2F8083108BDB00300242C
:102DA8000090D003004802580010005C00800051D9
:102DB8002DE9F047044607464FF00109DFF8508037
:102DC80014B93846BDE8F08794FAA4F5B5FA85F544
:102DD80009FA05F32E0108EB05156FEA030A24EA40
:102DE80003042B7B002BEBD058F806301B694BB93A
:102DF80046440222284607EA0A077368196830F031
:102E080065FADDE7284698470028D9D1F0E700BFE2
:102E1800A87E049030B5002289B00F490F4833F0DE
:102E280008FB0022002300240D4D0E49284600947B
:102E3800CDE906230E234FF44072CDE90334CDE9E2
:102E48000144094B08F0D8FA0849284633F02DF90F
:102E5800204609B030BD00BF792E009068190024C3
:102E6800C0140024002D002495310090B72F059040
:102E7800014808F00FB800BF980C00242DE9F0476E
:102E8800804620480F4630F0F9F90646002832D02F
:102E980000252846BDE8F087237B83B12368DB68DB
:102EA8000BB120469847636883F8069023681B692E
:102EB800CBB9636802222046196830F007FA013658
:102EC80010345445E8D3B8F1000FE2D0002DDFD01C
:102ED8002846FFF76DFF0546002FF7D00021642034
:102EE80033F097F9F2E7204698470028E1D009FA2D
:102EF80006F31D43E3E7044C0546DFF810A04FF046
:102F08000109DEE7C01F0024A87E0490B87E049063
:102F1800014B53F820007047047F049008B503461E
:102F280008462BB1044A136000F074FC002008BD69
:102F38006FF01500FBE700BF3400002410B5044C07
:102F4800237813B9034807F0A5FF0123237010BDA8
:102F58009E280024980C002410B504460B4830F035
:102F68008DF95CB10A4BBFF35B8F53E8001F013941
:102F780043E80012002AF8D1BFF35B8F054833F00D
:102F880064FA0548BDE8104007F084BFB81F002464
:102F9800BC1F002468190024980C00240020064B4C
:102FA800BFF35B8F014653E8000F43E80012002A85
:102FB800F9D1BFF35B8F7047B81F002470B5FFF7D6
:102FC800EDFF084C0546084EB44200D370BD636857
:102FD8005B792BB123685B6813B129462046984773
:102FE8001034F1E7A87E0490B87E049010B5044C24
:102FF800044920462FF0B8FF034B1C6010BD00BFEA
:10300800B00B0024F07E0490B01F002400230D4A6A
:103018004FF47A710C4810B513700C4A13600C4ABF
:103028001360FFF77BFFFFF7E1FF0A4B0A491846D9
:103038008B4200D310BD1A1A5C681033121101328A
:103048002271F5E79F2800249F320390B81F0024BF
:10305800BC1F0024A87E0490B87E0490014600227C
:10306800002301482FF0A1BFB00B0024014830F025
:103078003AB800BFB00B0024024B0146186830F084
:103088008DB800BFB01F0024014830F0C2B800BF9F
:10309800B00B0024264B70B51878002846D0FFF7EF
:1030A800E5FF054600283ED1224B234C1B68002B28
:1030B80012DD33F076F90A220023FEF70FFBD4E97C
:1030C8000032C01A40F2E93361EB0201984271F113
:1030D800000101D3FFF772FFD4E9003213F57A73C8
:1030E80042F10002C4E90032BDE87040FFF7CCBFEE
:1030F80063685B7923B12368294620461B68984793
:103108001034B442F4D32846FFF7B6FF0B4BBFF395
:103118005B8F53E8001F013943E80012002AF8D1F9
:10312800BFF35B8FC0E7064C064EEAE770BD00BFF1
:103138009E280024B81F002460190024BC1F002406
:10314800A87E0490B87E049070B50D4D297861B9B9
:103158000C4C01200C4EFFF791FEB44206D3FFF74A
:1031680099FF0028FBD101232B7070BD63685B7940
:103178001BB1236820469B6898471034EDE700BFD1
:103188009F280024A87E0490B87E049000212DE991
:10319800F0470846FFF772FE044658B34FF4FA7832
:1031A8004FF000091C4B01F00FF91C4A1B58136023
:1031B80033B11B4B1B68092B02DD1A4807F06AFE66
:1031C8000025194FDFF85CA044B12046FFF7F0FD59
:1031D800044618B94FF0FF384FF0FF39FFF75AFF90
:1031E800064628B9B5B942464B46504607F08EFE0A
:1031F8003546E9E74FF0FF384FF0FF39D2E72B6843
:103208009B691BB100222846114698471035BD42DC
:10321800F5D3E8E7054DFAE708000000B41F0024DD
:10322800BC1F0024980C0024B87E0490A87E04904B
:1032380013B5184830F022F8174B1B7873B1EFF329
:103248001184102383F31288BFF36F8FFFF722FFD7
:1032580084F31188BFF36F8F02B010BD0F4B1B684A
:10326800002BF9D050B9002200230D48CDE90023E6
:1032780042F21072002308F09BFEEDE70928EBD11B
:10328800074833F0E2F8074802B0BDE8104007F0FD
:1032980001BE00BFBC1F00249F280024B41F0024C7
:1032A80068190024980C0024064B10B504461B68C6
:1032B80098472146A06004482FF0F6FEBDE810406C
:1032C800FFF7B6BF34000024B00B0024044A054BB6
:1032D8009B1AB1EBD30F34BF52F83100002070476E
:1032E800987D0490A87E04902DE9F04F8FB0C1F32B
:1032F8004A280D46914604AF0C0DB8607B60B8F1C2
:10330800000F63D0002607F114034FF0040B4FF0B1
:103318000A0AC7F80C8032467E624846C7E9076643
:10332800019307F11C03CDF808B0CDF800A0F968A7
:10333800FFF790FAB0F5006F03461CD36C468AB0CD
:10334800D9F8041004AB26481A46C3E9050140F22F
:10335800FF71D9614FF400711984224B42F8103F74
:103368004FF4125133462048FFF7BEFFA5462C37CD
:10337800BD46BDE8F08FC0F30A0804F117003B60B2
:10338800184468F3532520F007008008FFF766FE0D
:10339800044690B13B6800F11001144A4846F961AF
:1033A800C7E9083607F11403CDF808B0CDE900A342
:1033B80007F11C03F968FFF74DFA68F353257B689A
:1033C800B96820462A462FF0A1FFD0E704F117007C
:1033D80020F007008008FFF741FE0446EDE700BF34
:1033E800CC2F059004000001E07D0490E7320390A3
:1033F8002DE9F04F87B00446934698460391DDE9DE
:103408001279DDE9105ABFB13B465246102100201F
:10341800CDF80090CDF81490FFF74AF8B0F5006F9A
:1034280006460AD340F2FF73174A0221174807B02D
:10343800BDE8F04F2FF0C3BF3E4604F0070405F186
:1034480017000BF0070BE400304444EA8B1420F01B
:10345800070044EA4624800844EA0554FFF7FEFDC5
:10346800054640B13FB13B46524631461030CDF893
:103478000090FFF71DF8434622460399284607B0F7
:10348800BDE8F04F2FF042BF0B300590E07D04906F
:10349800406820B1034BC01A40F3CF0070474FF08B
:1034A800FF307047987D04900EB403B503AB014616
:1034B800054853F8042B019301F0AEF902B05DF80A
:1034C80004EB03B0704700BF29340390CA0605D443
:1034D8008B064CBF02490349FFF7E6BF704700BFA0
:1034E800108205907F4505902DE9F04F89B09B46E5
:1034F80004460D46149B90469DF84CA00693159BD8
:10350800179E0593169B0493BAF1000F00F09D8057
:1035180006F4807306F0020907932FF0D5FE0246E1
:1035280000283ED091492046FFF7BEFF0746B9F173
:10353800000F08D016F0440F35D12A468C49204692
:10354800FFF7B2FF074406F0010353B1894B204649
:10355800894953F82A20894B002A08BF1A46FFF7E1
:10356800A3FF06F48073002B49D006F00803002B54
:1035780063D1B8F1000F66D0424681492046FFF773
:1035880093FF0546069B3D44002B6DD1049B002B01
:1035980073D1F30700F1E48031462046FFF796FF28
:1035A800D8E00746C3E7774B18680028CAD0764B9F
:1035B8004FF47A794FF03C0C1B68B5FBF3F5B5FB7B
:1035C800F0F100FB11554FF4616309FB05F5B1FB00
:1035D800F3F2B5FBF0FE03FB121100FB1E55B1FB25
:1035E800FCF309FB05F50CFB1311B5FBF0F5009195
:1035F80020466649CDE901E5FFF756FFA2E706F048
:103608000803EBB1624B2046624953F82A20FFF7C2
:103618004BFF0546B8F1000F05D0424658492046F1
:10362800FFF742FF0544BBF1000FABD05A465A4999
:103638002046FFF739FF0544A4E74FF0000BE1E708
:1036480006F00805E6E745469CE7BBF1010F069B37
:1036580006D1002B64D1049B002B7BD000250CE005
:10366800002BF8D04D485CE04D48069B22464D495A
:103678002FF012FB049B002B68D0DFF82C81DFF8B9
:103688002C91049F4FF0000B31462046102F28BF85
:103698001027FFF71BFF5D4545DC059B4FF0010B2D
:1036A800494620461A78FFF7FFFE1BF0070F03D1A3
:1036B80041462046FFF7F8FE5F453BD9059B494642
:1036C800204613F80B20FFF7EFFE0BF1010BBBF1BF
:1036D800100FEAD14FF0000B35492046FFF7E4FE02
:1036E8005A46059B20469A5CA2F120015F29314980
:1036F80028BF2E22FFF7D8FE0BF1010BBBF1100FEC
:103708001DD01BF0070F03D141462046FFF7CCFE22
:103718005F455A46E5D841462046FFF7C5FEEBE728
:103728001F485546A1E7414620460BF1010BFFF71C
:10373800BBFEB0E720492046FFF7B6FEC5E7059B6C
:103748003B440593049BDB1B04939AD1BAF1000F09
:103758007FF41FAF204609B0BDE8F04F2FF053BEED
:10376800064A20460449FFF79FFE15E748300590B2
:103778004C300590147F049059840590433005908F
:1037880071300590C81F0024C41F002455300590CF
:10379800287F0490753005907B3005905F34039046
:1037A8002934039021480090289A0590803005908C
:1037B80086300590A5800590269A059042F20F73F1
:1037C800114A8B4273B5044628BF0B46056805218C
:1037D80068462CF02BFD636806460B2228465B687A
:1037E8000A492FF002FE63683246694628465B683C
:1037F8002FF0FBFD63681B2205495B6828462FF004
:10380800F4FD02B070BD00BFD39E0590A4300590B2
:103818008830059000210123064A904206D8064ABE
:1038280001B901231360054B186070474008012156
:103838005B00F2E740420F00C41F0024C81F0024A9
:10384800F8B50D4604464618054FB44201D128463E
:10385800F8BD14F8011BBB6801485B689847F4E79A
:10386800D47B0490014B036002207047707F049062
:10387800104B70B51C680D46B4B10F4B1968002386
:103888008B4202DB6FF0010070BD224612F8146B08
:10389800864202D001331446F2E7E06832F0A5F917
:1038A80028B100202C60EFE76FF00C00ECE76FF018
:1038B8001200E9E740000024907F04902DE9F843C6
:1038C8000646FDF737FF0546EFF31188102383F30B
:1038D8001288BFF36F8F114B1C68D3F804909C4279
:1038E80008BF002434B988F31188BFF36F8F2046CE
:1038F800BDE8F883A7683846FDF71CFFA84206D143
:103908002A463946304643F0E9FE0028EBD04C45BC
:1039180001D02468E6E70024E5E700BF440000245E
:103928002DE9F0410E461546FFF7C8FF044628B3B7
:10393800C3681BB35F690FB3062E07D0072E20D0CC
:103948002A4631463B46BDE8F0411847838A3BB9D1
:103958002A463146B84750B9A38A0133A38206E004
:103968004FF6FF72934204D00133A3820020BDE8D2
:10397800F081124A012112482FF018FD6FF015004E
:10398800F5E745B12A7832B10022314682822A46CB
:103998005B699847EAE7A38A012B08D12A460721E1
:1039A8002046B8470028E2D1A38A013BD6E70BB1ED
:1039B800013BDAE7034A0221DDE700BF2331059026
:1039C800A87D04904531059003480021034A08B5B5
:1039D800121A2FF047FE08BD800D0024D42C0024B5
:1039E8000748084A0849121A08B52FF03DFE07484B
:1039F800074A0849121ABDE808402FF035BE00BF33
:103A080000000024440D002484A305900000002435
:103A18000000002484A305902DE9F047064600AF76
:103A28000C46002936D0E9468AB0A3686D46D1E92C
:103A3800001221484FF0050AA846C5E90501C5E965
:103A4800072348F810AF002342464FF421511B4882
:103A5800FFF74AFCCD466369AD46D4E9031218481E
:103A6800C5F810A0C5E90501C5E9072300234246AA
:103A78004FF421511148FFF737FCCD46E369114A4D
:103A880001210E482FF09BFCA3690F4A01210B4826
:103A98002FF095FC012E07D1EFF305830B4A103B5D
:103AA800314606482FF08BFC2146304606F040FE92
:103AB800BD46BDE8F08700BF6E310590207E0490BA
:103AC8009D310590CC310590DB3105900932059088
:103AD80030BFFFF7FDBF00BF2DE9F0410B4E054693
:103AE800DFF82C80324606EB0807CC1B0949204634
:103AF80043F0A7FDA019083C4246002143F0C9FD48
:103B080007F10800C5F89040BDE8F081000000000A
:103B180008000000B87E0490054B5A699B689A42D9
:103B280004D0044A536843F080535360704700BF81
:103B38006021002400ED00E070B5294C06460D46D2
:103B4800284829492FF09DFDA36AD9043CD525486A
:103B580026492FF096FD1720A36A1A0504D5214897
:103B680023492FF08EFD18201D4CA36A9B0512D502
:103B78001C4820492FF085FDA36BA26A100409D5C3
:103B88001D4A012117482FF01AFC1EB1A36A23F41D
:103B98000043A3621920124CA36A590504D51148A1
:103BA80016492FF06EFD1A20A36ADA050ED50D48C6
:103BB80013492FF066FD1B20094A936A43F47F439B
:103BC800936200232B7070BD1620C5E7A36A9B047F
:103BD800F2D504480B492FF054FD1C20ECE700BF38
:103BE80000ED00E0207E04901C32059032320590F2
:103BF80043320590563205906F3205908432059015
:103C08009F320590B732059010B5204C20492148C5
:103C18002FF037FDA36A990136D51E481E492FF0AB
:103C280030FD1E20A36ADA0104D51A481B492FF07B
:103C380028FD1F20154CA36A1B0304D515481849F5
:103C48002FF01FFD2120A36A590304D511481549F7
:103C58002FF017FD22200D4CA36A9A0304D50D48B6
:103C680011492FF00EFD2320A36ADB0304D5094870
:103C78000E492FF006FD2420044A936A6FEA034395
:103C88006FEA1343936210BD1D20CBE700ED00E0FF
:103C9800E6320590207E0490FE320590113305909F
:103CA8002B330590493305906E3305908833059082
:103CB8002DE9F843364D8046894636483649174639
:103CC8002FF0DFFCAB6ADE0627D5112433493148D3
:103CD8002FF0D7FCAB6A1D0704D5122430492D48B4
:103CE8002FF0CFFC2A4DAB6A980718D52D492948E3
:103CF8002FF0C7FC6E6BAB6A190646D52A4A3346C5
:103D0800012124482FF05BFBB9F1000F03D0AB6A07
:103D180023F08003AB62132403E01024DAE76FF08A
:103D280015061B4DAB6ADA0704D514241F49194838
:103D38002FF0A7FCAB6A9B0604D515241C4915482F
:103D48002FF09FFC124B9A6AD50602D49A6A900704
:103D58000AD55B68190507D54146304600F0D8FA00
:103D680010B180F309880224094B9A6A920603D598
:103D78005A6A22F400525A629A6A204642F0FF02B6
:103D88009A6200233B70BDE8F8836FF01506C2E71E
:103D980000ED00E0207E0490B3330590C933059010
:103DA80043320590FC330590143405902A3405906D
:103DB800B73205902DE9F041664B8AB004460026DB
:103DC800D3F8048000AFC8F3080586F31188BFF361
:103DD8006F8F02F07F43B3F17F4F07D102F00C03DE
:103DE800082B12D15C495D482FF04BFC0026344665
:103DF8000023FB71EB1E092B00F28B80DFE803F038
:103E08000A81847D89898989898710074CBF0C4676
:103E18000126EDE7524951482FF033FC4D4D002360
:103E2800FB71EB6A9A0705D54E494C482FF029FCDF
:103E3800002332E0EB6A002B01DA4B49F5E7EB6A25
:103E48005B00F5D5494945482FF01BFC6B69A26911
:103E580043F480736B61BFF34F8FBFF36F8F6B6950
:103E680032F8022C23F480736B61BFF34F8FBFF3DA
:103E78006F8F4DF602739A4208D0AB6ADBB27BB300
:103E8800FA1D01212046FFF713FF38E02368384A5E
:103E9800012132482FF093FA2368FA79E2B907F141
:103EA800080504F1200C2068083454F8041C2A463C
:103EB800644503C21546F6D17A6A002E45D0C2F38E
:103EC800080121B96FEA52226FEA42227A6207F1A9
:103ED80008011846FFF7A0FD2837BD46BDE8F08168
:103EE800AB6A13F47F4F04D0F91D0120FFF724FEBD
:103EF80005E0AB6AB3F5803F9AD3FFF785FE03462A
:103F0800CBE7FA1D0021BDE7F91D0020EEE71949AE
:103F18008BE718F4F87F184AE8468AB0174B18BFA1
:103F280013466A461649103DC2E905134FF400735B
:103F3800D5611384134B42F8103F00234FF41151FD
:103F48000648FFF7D1F9C54672E722F4FF7222F05E
:103F58000102BBE700ED00E077340590207E049075
:103F6800A2340590B9340590DA340590E834059008
:103F780007350590233505905E3405904934059042
:103F88004735059004000001044B5A6942F01002BD
:103F98005A615A6922F008025A61704700ED00E040
:103FA800EFF30880EFF3098101B57246FFF702FFCE
:103FB80001BD00BF002080F31488BFF36F8F0F4846
:103FC80080F308882FF047F900200D490860BFF3F7
:103FD8004F8F00F03DF8102080F3118809484FF406
:103FE8000461401880F30988EFF314800221084324
:103FF80080F31488BFF36F8F00F05CF960A300248E
:1040080094ED00E0C03A0024BFF34F8F0549064BFA
:10401800CA6802F4E0621343CB60BFF34F8F00BF5E
:10402800FDE700BF00ED00E00400FA0507490023A2
:10403800D1F890201846C2F30722934200DB70475C
:10404800C1F898300133C1F8A000F6E700ED00E0B0
:1040580070B572B6002484F31388FFF7E7FF3E4B70
:104068004FF0FF32C3F88020C3F88420C3F88820BB
:10407800C3F88C20C3F89020C3F89420C3F8982084
:10408800C3F89C20C3F88021C3F88421C3F8882191
:10409800C3F88C21C3F89021C3F89421C3F8982160
:1040A800C3F89C212D4A536913F4803339D0C2F8E0
:1040B8008440BFF34F8F536923F480335361BFF3B8
:1040C8004F8FD2F8803043F6E074C3F3C900C3F3CE
:1040D8004E335B0103EA0406014646EA817501395D
:1040E800C2F87452F9D2203B13F1200FF2D1BFF37A
:1040F8004F8FBFF36F8FBFF34F8FBFF36F8F174B88
:104108005A6922F400325A610022C3F85022BFF3E0
:104118004F8FBFF36F8F62B6BFF34F8FBFF36F8FB1
:1041280070BDC2F88430BFF34F8FD2F8803043F6A9
:10413800E074C3F3C900C3F34E335B0103EA04061A
:10414800014646EA81750139C2F86052F9D2203B2E
:1041580013F1200FF2D1CAE700E100E000ED00E022
:10416800084B9B6883420BD1EFF3058343B1064BA1
:104178005A6842F080525A605A6A22F400425A62DF
:1041880007F00ABC6021002400ED00E015498A68A8
:104198004FF030001044EFF3098C80E8F01F102036
:1041A80080F31288BFF36F8F0F4F4FF000664A6994
:1041B8008A603E60D2F890000C4C2060D2F89400DF
:1041C8000023C2F8943080F3118804B5104600F03B
:1041D800ABF9BDE8044002F1300090E8F01F8CF321
:1041E800098870476021002404ED00E0F81F0024CE
:1041F8001EF0040F0CBFEFF30880EFF3098081690C
:1042080011F8021C0229FFD001B572462FF02EFAD0
:1042180001BD00BF09010028C9B206DB00F16040FA
:1042280000F5614080F80013704700F00F00014B63
:104238001954704714ED00E000B2002807DB012391
:10424800410900F01F00024A834042F821307047BC
:1042580000E100E000B200280CDB4309012200F075
:104268001F0005492033824041F82320BFF34F8FB8
:10427800BFF36F8F704700BF00E100E04209054BB4
:1042880000F01F0053F82220012303FA00F0104029
:10429800704700BF00E100E0044B054A23F07F03AC
:1042A8009360BFF34F8FBFF36F8F70470004009088
:1042B80000ED00E008B5FFF7EFFF084AD2F88830B4
:1042C80023F47003C2F88830FFF77EFBFFF788FB02
:1042D80000F05CF82FF0F8F906F04EFB00ED00E076
:1042E80042F8203C203A009B08495360019B21F08A
:1042F80001019360029B9161D3604FF08073D36199
:1043080000230265C0F89430704700BF352C009038
:104318000A4A0346906878B113F1160FD0F8800066
:1043280005D0A0F140029A4205D8834203D28142C7
:1043380028BF002070470020704700BF602100247C
:1043480015460D4A0E4608B50C4B9060D0F89020E3
:104358001A6000F0E9F82C4686F309880020044B1F
:1043680098472046002100220023024C20470000E5
:10437800A9360390352C009060210024F81F0024F2
:10438800014B10221A61704700ED00E00023044839
:104398001021C2180133962B82F80013F9D1704707
:1043A80000E100E008B5EFF30583064A103B02EB95
:1043B800C30152F8330049688847BDE80840FFF751
:1043C800ABBB00BFD406002401480068704700005A
:1043D800F81F0024154A70B5536913F4803323D1AC
:1043E800C2F88430BFF34F8FD2F8803043F6E074C0
:1043F800C3F3C900C3F34E335B0103EA0406014665
:1044080046EA81750139C2F86052F9D2203B13F1AE
:10441800200FF2D1BFF34F8F536943F480335361B8
:10442800BFF34F8FBFF36F8F70BD00BF00ED00E08B
:10443800134A002370B5C2F88430BFF34F8F536915
:1044480023F480335361BFF34F8FD2F8803043F6A3
:10445800E074C3F3C900C3F34E335B0103EA0406F7
:10446800014646EA81750139C2F87452F9D2203BF7
:1044780013F1200FF2D1BFF34F8FBFF36F8F70BDD1
:1044880000ED00E0002910DD00F01F030B44BFF32E
:104498004F8F07490344C1F8680220301A1A002ACE
:1044A800F9DCBFF34F8FBFF36F8F0020704700BF59
:1044B80000ED00E00B4B5A6912F4003211D1BFF342
:1044C8004F8FBFF36F8FC3F85022BFF34F8FBFF3E7
:1044D8006F8F5A6942F400325A61BFF34F8FBFF3AE
:1044E8006F8F704700ED00E0BFF34F8FBFF36F8F02
:1044F800064B5A6922F400325A610022C3F850224E
:10450800BFF34F8FBFF36F8F704700BF00ED00E020
:10451800024B0121024A034800F08CB8000008242D
:1045280000000024E47F0490D0F880204021054B4F
:10453800403A18461A60044AC3E90112012100F002
:1045480083B800BFFC1F002400000B1508B5034604
:104558001048D0F89020C2F30722013A934207D9B5
:104568000D4801210D4A2EF02AFF6FF0150008BDF5
:10457800C0F898300A6822F01F021A4342F010026D
:10458800C0F89C208A6842F00102C0F8A0201846B2
:10459800EDE700BF00ED00E0087E04905E35059071
:1045A800F0B50E4685B01F4604460025B5420DDA23
:1045B800606810B397B1431E18420AD0104A2B46C0
:1045C800012110482EF0FBFE6FF01502104605B0D1
:1045D800F0BD1F28F2D921680B42EFD1236801A949
:1045E80001932FF072F8A3680343D0B20393FFF747
:1045F800ADFF10F1160FE7D0421C01350C34D5E79A
:1046080084350590087E0490044B0522C3F8942055
:10461800BFF34F8FBFF36F8F704700BF00ED00E00F
:10462800BFF35F8F024B0022C3F89420704700BF8E
:1046380000ED00E010B5034C01232278FFF7B0FF2E
:10464800207010BDA12800240B4A08B50023127859
:10465800FFF7A6FF10F1160F07D0084A0021D2F87D
:104668009030C3F30723984200DB08BDC2F89800D6
:104678000130C2F8A010F2E7A128002400ED00E004
:104688005F4860492DE9F043D0F8903085B00D6857
:10469800C3F307239D4200F2B080FFF7C1FF4968CA
:1046A8000022954201F10C011BD1574C6846574F27
:1046B8002570FFF7D7F800250646DFF85481DFF8A4
:1046C8005491AE4220D1237800204D49D1F8902052
:1046D800C2F307229342C0F28A800020FFF794FFBA
:1046E8004FE0C0F8982051F80C3C23F01F03134307
:1046F800013243F01003C0F89C3051F8043C43F0F9
:104708000103C0F8A030CCE700984FEA051C00EB85
:104718000511CB683B40B3F5000F49D00AD8B3F573
:10472800001F31D0B3F5800F37D0B3F5801F13D0F9
:104738000135C6E7B3F1007F43D0B3F1805F49D0BC
:10474800B3F1807FF4D150F80C3088682EF0BDFFAB
:104758004A6840F0887009E050F80C3088682EF0FC
:10476800B4FF40F088504A6840F43020039001A913
:104778002078CDE90123FFF7E9FE002833DA6FF04E
:10478800150005B0BDE8F08350F80C3088682EF0AD
:104798009CFF4A6840EA0900E8E750F80C3088684E
:1047A8002EF093FF40F000704A6840F40030DDE7D7
:1047B80050F80C3088682EF088FF4A6840F0827004
:1047C800D4E750F80C3088682EF07FFF4A6840F430
:1047D8008020CBE750F80C3088682EF076FF4A68C6
:1047E80040EA0800C2E7237801332370A0E7C1F844
:1047F80098300133C1F8A00068E74FF0FF30C0E7F8
:1048080000ED00E0C47E0490A12800240000F0FF21
:104818000000021100000811F0B587B007460E46E7
:1048280014460021102268461D4642F032FF02233A
:104838002A4621468DF802306846044BCDE90476B5
:1048480001932BF0F9FD07B0F0BD00BFF9360390D6
:1048580008B5024B1B689847002008BD08200024B3
:10486800034B044A1860937843F00203937070472F
:10487800082000244C00002408B505482EF064FAEE
:10488800002383F31188BFF36F8F0423184602DFD8
:10489800AA3505900649074821F00701C1F11052D1
:1048A80008B502F500222EF09FF9002008BD00BFD0
:1048B800CFAF00240C2000244FF0FF324FF0FF331D
:1048C800014806F0F1B900BF5C000024014806F079
:1048D8005FBA00BF5C00002438B50546FFF7ECFF5F
:1048E800082108482A462EF0C8F8044628B925B1F8
:1048F800054B0C22FFF768FD1A50FFF7E7FF20462B
:1049080038BD00BF0C2000240C00000038B5044658
:104918000D46FFF7D1FF082221462B4607482EF007
:104928002BF9044628B925B1054B0C22FFF74CFD9D
:104938001A50FFF7CBFF204638BD00BF0C200024DB
:104948000C00000010B50446FFF7B6FF03482146E7
:104958002EF031F8BDE81040FFF7B8BF0C20002456
:1049680070B541690446867A0A4D59B1437ADB0726
:1049780006D42C2303FB06535B6A1B689B68984785
:10498800002363612C20214606FB0050BDE87040DF
:1049980031F000BBD40C00242C22024B02FB003067
:1049A800704700BFD40C0024827A2C21054B01FBF0
:1049B80002339A6A1B7F801A1B3323F00303B0FB70
:1049C800F3F07047D40C002438B52C24827A064BB7
:1049D80004FB02335B6AD3E901240C601568FFF716
:1049E800E3FF04FB005038BDD40C00242DE9F0434C
:1049F80085B0054690461C466846039131F0D3FCC5
:104A0800DDE90067EFF31189102383F31288BFF300
:104A18006F8F6B8B002B41D02A8B9A4225D90022AD
:104A28000023284606F004FA0446F0B189F31188F9
:104A3800BFF36F8F039B002B41D032463B4668463D
:104A480031F0D6FCA27A2C21254B204601FB0233FB
:104A580003A95B6A1B681D68DDE90023A84760613C
:104A680070BB2046FFF77CFF24E0698B4B1E6B83ED
:104A780089F31188BFF36F8F2B7F2A8B1B33AC6AA6
:104A8800521A23F0030302FB0344154B154AEB1A91
:104A98009B105343A3722B7FE372CBE789F31188F2
:104AA800BFF36F8F23464246284606F0C1F90446F5
:104AB8000028BFD10024204605B0BDE8F08363611B
:104AC80001230025E27A04F1180023812946039B7B
:104AD8006560638242F0DDFD63692582E360EAE791
:104AE800D40C0024A38B2EBA70B50D4C2C2500B91C
:104AF80070BD037A4668002BFAD0013BDBB2037223
:104B0800002BF5D1C3604360837A05FB03431B6A1E
:104B180013B198473046EAE7FFF722FFFAE700BFEC
:104B2800D40C0024F7B506460D461446124F3846F5
:104B380031F05BF8E0B1BB68AAB2314638461B6871
:104B48009847002802DB002003B0F0BD002CFBD101
:104B5800AC42F8D22F1B042F28BF042704F04AFBCD
:104B680001A901903A46301942F06BFD3C44EFE749
:104B78006FF01200E8E700BFB87B04902DE9F04120
:104B880090F8283004460F4600F1280603F01F036A
:104B9800012B1BD0022B05D043BB90F829102EF017
:104BA800F5FE03E0818DC9B200F056FF0546E8B175
:104BB80030462EF03EFE024668688368A2B99B68BC
:104BC8004BB13A463146BDE8F0411847818DC9B22C
:104BD8002EF0C3FEEAE76FF08503104AFFF7F4FBF7
:104BE80013500020BDE8F081DB68E9E794F829104C
:104BF80020462EF0EBFD02460028ECD030462EF081
:104C080018FE40B91369002BE5D03A4631462046D4
:104C180098470346E1E7D368F5E700BF0C000000BA
:104C28002DE9F04F95B00D4600F128030446097EA2
:104C380002AF914631F08008BB600BD06FF00408DA
:104C4800A64A0121A6482EF00AFE40464C37BD462A
:104C5800BDE8F08F6B7E03F00102B9F1000F17D0A9
:104C680019F10C0F14D0B2B919F1710F03D12846FC
:104C7800FFF73AFFE9E79B4A0B4699480121CDF82F
:104C88000090C8462EF0A5FB2846FFF72DFFDCE76D
:104C9800002A00F0C784002940F087842B8A072B5C
:104CA8000FD9EA681368A3625368E362D5F804A0D1
:104CB800E28DBAF1000F17D18B4A012188482EF0F6
:104CC800CEFD8A4A012186482EF0C9FD2846FFF705
:104CD8000BFFB8682EF0ADFD0346A069002B00F06D
:104CE800B884802100F0BEBC04F128002EF0A1FD9C
:104CF800E0B99AF8193032B198071DD46E4688B0D9
:104D080002AA7B4B05E05E0716D46E4688B002AA5D
:104D1800784BC2E9053A032342F8103F70480B4626
:104D28004FF4C251FEF7E0FAB546CAE70AB9724A2B
:104D3800C3E79AF81930DFE7294600202EF0F7FC80
:104D4800054628B9684A012165482EF088FDC0E764
:104D580094F828200023FFF737FB684E12F0600F05
:104D68008351C2F3411308D0032B40F0EB816FF05D
:104D78008503FFF729FB335057E004F128002EF094
:104D880058FD94F82930002840F07681013B0A2B21
:104D9800EDD801A151F823F0634F0090774D0090B2
:104DA800E74F0090774D0090CD4D0090774D0090E3
:104DB800774D0090774D00906F4E0090774D0090A2
:104DC800154F0090A069618D03697F29D3F8803061
:104DD800CDD8A28D002ACAD1E28D002AC7D194F875
:104DE8002820D206C3D194F83420022A04D14FF0E7
:104DF800FF33FFF7E9FABEE71A070BD5C9B22EF061
:104E080053FD804648B1638D3D4A012134482EF058
:104E1800D6FA2CE7012384F83D3094F83430012B7E
:104E28001FD1638DEBB984F83430FFF7CDFA3358CE
:104E3800002B7FF44BAF0123B86823632EF0F9FCF5
:104E4800002840F0AB83E38D002B00F0A7832946B0
:104E580000202EF06CFC0546002840F09B83294A70
:104E680071E70123DFE720462EF0A6FC628D01469C
:104E7800FF2A3FF67CAFE38D002B7FF478AF94F8E0
:104E88002830DB067FF473AF94F83430002BAED0B3
:104E98002AB1D2B220462EF049FD0028A7D0618D54
:104EA80094F83C308B42C0D0C9B2204600F07CFD5B
:104EB800638D804630B1144A0121009008482EF0D5
:104EC80088FAD4E61A1E4FF00501204614BF0223C3
:104ED800012384F834302EF065FEA6E7DD35059011
:104EE800587E0490FE3505902D3605909036059035
:104EF8004F3605905E3605906F3605900C00000021
:104F0800A736059097370590C936059094F828304C
:104F180003F01F03012B7FF42AAFE38D002B7FF4EE
:104F280026AF628DFF2A3FF622AFA18DFF293FF6FB
:104F38001EAF94F83430022B7FF459AFD2B220461A
:104F4800C9B22EF08CFD10F1020F804640F0FF80B0
:104F5800FFF73AFA46F8008067E7E38DA18D002B4A
:104F68007FF405AF94F83430002B3FF440AF012BA9
:104F780010D100297FF43BAF12F01F020DD1638DD1
:104F8800012B7FF452AF94F870306FF3C30384F8A9
:104F980070304AE712F01F0217D0022A7FF445AF9B
:104FA800B4F82A80B8F1000F7FF43FAF5FFA81FAB6
:104FB8002046514600F05AFE0346FFF705FA3350E3
:104FC800013306D14FF0FF3851E600297FF40FAFC7
:104FD800D5E74246514620462EF031FC25E7E38DC1
:104FE800A18D002B7FF4C3AE638D5FFA81F8022B8D
:104FF80013D194F8283003F01F0358EA03037FF411
:10500800B6AE0122090AA0692EF02BFC00287FF415
:10501800AEAE012384F83D3007E794F83400002849
:105028003FF4E5AE01280DD100297FF4E0AE12F07F
:105038001F020AD1012B7FF4F8AE94F8703043F0C8
:105048000803A4E712F01F0212D0022A7FF4EDAE83
:10505800002B7FF4EAAE4146204600F0E5FD03460A
:10506800FFF7B2F933500133ACD001224146B2E721
:1050780000297FF4BCAEDDE70A2B3FF678AE01A12C
:1050880051F823F0B9500090774D0090774D00907B
:10509800774D0090774D0090774D009039510090F2
:1050A800774D009035550090774D009063550090EE
:1050B800E38DA18D022B7FF45AAE94F83430002B87
:1050C8003FF495AE012B10D100297FF490AE12F079
:1050D8001F020DD194F870304FEA9308C3F3001300
:1050E80008F0020848EA030806E012F01F0210D090
:1050F800022A12D04FF0000805F10C0A50462EF093
:105108004AFBE38D98420ED26FF00B03FFF75CF970
:1051180031E600297FF46BAEDCE7C9B220462EF0F9
:1051280037FD8046E8E7414650462EF023FB7CE6F3
:1051380094F82820B4F82AA0D0064FEA1A235FFA78
:105148008AFA09D029462046FFF718FD8046B8F1AB
:10515800000F7FF48CAD68E6013B0E2B3FF607AEDF
:1051680001A252F823F000BFAD510090F751009012
:10517800BB520090774D0090774D0090B35200904D
:10518800B3520090774D0090774D0090774D009086
:10519800774D0090774D0090774D0090774D0090B7
:1051A8001354009005F10C08B4F82EA040462EF0D8
:1051B800F2FA82450AD2B4F82EA020462EF0FCFA64
:1051C80048B101287FF4D3ADA16F05E040462EF029
:1051D800E2FA8246F1E7616F002900F021810A783E
:1051E8004046524528BF52462EF0B3FA1DE60AF152
:1051F800010820462EF0E0FA0146F8605FFA88F2CE
:1052080020462EF06DFB824630B9C14A4346012143
:10521800C0482EF0D4F8AAE505F10C08D0F804B07F
:1052280040462EF0B8FA9BF80020904203D2404640
:105238002EF0B1FA0246594640462EF08AFADAF8BC
:105248000CA0BAF1000F09D1298AE38D99427FF6A3
:10525800ECADC91A40462EF097FAE6E5DAF80400F4
:1052680083681B6B13B9DAF800A0EAE7F968984776
:105278000028F8D0A0F1040B5BF8043F002BF2D013
:105288001B78002BEFD040462EF085FADBF8003073
:105298001A78904203D240462EF07DFA82B2DBF8AB
:1052A800001040462EF055FAE6E720462EF084FA24
:1052B8005DE55246032120462EF09CFA82460028DE
:1052C8003FF455AD2EF0B0FAE38DE0B9BAF81420EA
:1052D80098463A85DAF8102005F10C0A12885046EB
:1052E8007A852EF058FA804509D2E08D97F8282063
:1052F80007F12801824228BF0246504674E750460B
:105308002EF049FAF2E79B460023DAF808203B75AD
:105318009AF815307B75804B1340804A934263D1CD
:10532800102107F1180003F0B5FA002842DB07F155
:105338002803102807F11802DFF8E4C19E4628BFA9
:105348001020404503F102033DD88000C7F80CE067
:105358000230387505F10C0A50462EF01CFA97F801
:105368001480D84528BFD846404503D250462EF071
:1053780012FA8046B8F1020FC34607F114015046ED
:1053880028BF4FF0020B5A46A8EB0B082EF0E1F9A4
:10539800D7F80CB04FEA58030BEB58025A452AD1FC
:1053A80018F0010F3FF441ADFA685046D15C2EF079
:1053B800D9F93AE558307FF4DAAC5A4A0121554810
:1053C8002EF04DFAD3E412F8011B08F101084FEA58
:1053D800111A01F00F011CF80AA01CF8011003F8BB
:1053E80002AC03F8011CACE79AF814303B75DAF804
:1053F8001030FB60AEE71BF8011B5046C7E90032CE
:105408002EF0B8F9D7E90032C8E720462EF0D4F9D3
:1054180020B101287FF4ABACA36F00E0636F13B930
:105428006FF0150823E45B88B3F5007F7FF69FAC27
:105438003D4B226DBB62002387F82C3004F15003EA
:105448009342FB6060D105F10C0A50462EF0A3F997
:10545800B7F82A80E38D984528BF9846404503D27F
:1054680050462EF098F9804697F8282007F1280131
:105478005046424528BF42462EF06BF9B8F1050F59
:1054880094BFA8EB0808A8F10508B8F1000F3FF48D
:10549800CCACD4F850B0FB689B453FF4C6ACBBF12C
:1054A800000F3FF4C2AC9BF815300F2B15D19BF8B9
:1054B80014205046DBF81010424528BF42462EF013
:1054C80048F99BF81430434594BFA8EB0308A8EBB0
:1054D8000808B8F1000F3FF4A8AC636D5B453FF4D2
:1054E800A4ACDBF800B0DAE7537D0F2B08D1137DAD
:1054F800798D0B447B8597F82C30013387F82C3055
:10550800636D93429FD01268002AEDD19BE700BFDC
:10551800EC360590587E049000FF0200000302005C
:10552800B437059012370590050F050094F834300C
:1055380094F83CA0002B3FF45AACE38D012B7FF488
:1055480016AC05F10C0840462EF025F9E38D98427B
:10555800FFF4DAAD5146404629E794F8283003F0C5
:105568001F03012B7FF443AC20462EF0CDF9002811
:105578003FF43DACA38D4268FF2B3FF6F8AB1279A0
:105588009A42FFF4F4AB0F2B3FF6F1AB234493F8A8
:105598003EA0D2E76B7E59077FF559AC29462046D5
:1055A80000F0FAFA8046FFF750BB5A077FF591AB37
:1055B80080297FF48EAB2846FFF796FA256B012DDC
:1055C80040D194F83D30002B3FF43FAB94F829309C
:1055D800052B0CD1618DA069C9B22EF065F9804602
:1055E80028B1638D234A294623482DF0E8FE94F814
:1055F8002930032B11D1638D022B0ED1A18D0022EE
:10560800A0690D0A29462EF02CF9804628B11B4ABC
:105618002B46012118482DF0D2FE002384F83D3096
:10562800FFF713BB5B077FF554AB0029C0D1236B91
:10563800012B3FF41CAB124A02210F482EF00FF940
:10564800FFF715BB0F4A02210B482EF008F9FFF7A8
:10565800FCBAE38D002B3FF444AB19F10C0118BFE1
:105668000121C9012EF0A4FD002380462363FFF722
:10567800ECBA00BFA7360590587E049055370590C0
:10568800343705907337059030B589B00022002370
:1056980000241E491E480094CDE906236FF0070335
:1056A8004FF48062CDE90334CDE90144194B05F08C
:1056B800A3FE1949164830F0F8FC184B18498B42DC
:1056C80007D3184B002018498B4210D3002009B08B
:1056D80030BD03F11402BFF35B8F52E8000F42E8BC
:1056E8000045002DF9D11833BFF35B8FE7E703F1CD
:1056F8001402BFF35B8F52E8004F42E80005002D0B
:10570800F9D11833BFF35B8FDEE700BF40300024C8
:10571800A019002489570090CE3705902C0D00243D
:10572800440D0024440D0024440D002438B50D46D2
:105738002EF0EAF830B9104A01211048BDE8384087
:105748002DF034BEC46804B938BD2B78032B07D0BC
:10575800052B0CD0022B08D1606883689B6902E096
:10576800606883685B6903B198472468EBE7606801
:105778008368DB69F7E700BFD3370590687E04903C
:105788002DE9F04784B0DFF80482102600AF4FF00F
:10579800FF334FF0FF32391D404605F021FAFB6810
:1057A8001B69D3F89C40236A73B1EFF3118386F326
:1057B8001288BFF36F8FD4F820A0BAF1000F1BD165
:1057C80083F31188BFF36F8F3B79062BDFD0072B4C
:1057D800DDD801A252F823F0775800906B5800905A
:1057E8009F5800907D580090D5580090C15800905F
:1057F8009757009085590090616ADAF800208A4529
:10580800226208BF626283F31188BFF36F8F9AF830
:1058180018305146DAF81E2020465D061ED1FFF7E3
:10582800FFF905460028BED0E9468AB09AF8183034
:105838006A465749C2E9073A0523C2E9051042F802
:10584800103F00234FF421515248FDF74DFD2A46E1
:1058580007212046CD462EF0A5F9A4E72EF08DF8B5
:10586800DFE70022012120462EF09CF98FE7002275
:105878001146F8E794F8703043F0040384F8703068
:1058880094F83430022B03D1391D2046FFF74EFF20
:1058980000220321E7E794F870306FF3820384F85D
:1058A800703094F83430022B03D1391D2046FFF7AD
:1058B8003DFF00220221D6E794F83430022B7FF412
:1058C80066AF391D2046FFF731FF60E794F8703066
:1058D800D4F818906FF3820384F87030D9F8103038
:1058E800D9F808A0BFF35B8FD3F8A030BFF35B8F64
:1058F8009A071BD5DAF83C3048469847DAF824303E
:105908000021484698470546DAF840304846984707
:105918007DB1214A01211F482DF048FD00220421B4
:1059280020462EF03FF92A4607219CE74FF0FF3525
:10593800EFE72946204600F037F8054608B1174A30
:10594800E8E7802120462EF020F920B1144A0121F1
:1059580010482DF02BFDA0692EF0DDFC831E0022DF
:105968000421584284F83420584194F8703023F0C8
:10597800680343EA401384F8703074E7094A012148
:1059880004482DF013FDBA6806216CE7680C002462
:1059980002380590687E04902C3805905A38059096
:1059A80086380590A33805902DE9F04105460E4646
:1059B8002DF002FF804695F83C303BB328462DF089
:1059C800A3FF0746F8B1014628462DF0F6FF10223E
:1059D8000446002105F13E0041F05BFE002385F8F6
:1059E8003C30FF6847B98CB1194A012119482DF09C
:1059F800DDFC2046BDE8F081786883685B6A03B106
:105A080098473F68EEE76FF03C04EDE71EB985F86C
:105A18003C600024EDE73246414628462DF060FF01
:105A2800074690B1024628462DF0F1FF04460028AB
:105A3800DFD185F83C60FC68002CEAD06068836898
:105A48001B6A03B198472468F6E76FF03C04D0E777
:105A5800C7380590507E049001F07F0311F0800F45
:105A680070B518BF1033012504469D4090F83430B6
:105A7800022B06D00C4A01210C482DF097FC00207F
:105A880070BD90F83C602DF097FE014620463246E6
:105A98002DF026FF0028F2D0C0680028EFD08368D8
:105AA8001D42EDD10068F8E7EE380590607E04905D
:105AB8002DE9F04F83B00E468146904600AF4C6802
:105AC8007B6097F830303B602DF076FEA368014686
:105AD8001B6B33B96FF0150420460C37BD46BDE883
:105AE800F08F204698470028F4D0051F002406F1BF
:105AF8000C0A55F8041F09B10B782BB9002C0CBF00
:105B08006FF03C040024E7E74B78042B0ED1002CFF
:105B18003CD18B787A689342EBD1CB783A68934240
:105B2800E7D10B79002BD7D00124E2E7052BE0D190
:105B3800002CDED0B8F1010F91F802B009D0B8F10D
:105B4800020FF1D152465946D9F818002DF0ECFF52
:105B580004E05246D9F818002DF0CBFF044600287F
:105B6800E2D06D468AB0F3686A4609495062C2E9D4
:105B780007B30623C2E9051842F8103F00234FF483
:105B880041510448FDF7B0FBAD46A5E70024A3E763
:105B98001E390590887E04902DE9F0410B7E05465C
:105BA8000C465E0638D119062DD52DF00AFE40B1F7
:105BB8001B4801211B4A2DF0F9FB4FF0FF30BDE8CF
:105BC800F0812846D5F87480268AEF8D2DF0F4FDF3
:105BD800F8B1421E534253419B01228A9AB1BE42F8
:105BE8003246E98D28BF3A4691420CD9B2FBF3F10F
:105BF80003FB11223AB994F91830002BBEBF637E1B
:105C080043F0080363762146A869BDE8F0412EF009
:105C18002BBB98F80730E0E76FF01500CFE700BF1F
:105C2800807E04905A39059070B5064680690C4606
:105C38002EF0BEFA054638B10A4A234602210A4820
:105C48002DF0BDFB284670BD14F0800F4FF0010207
:105C5800B36B1CBF24F080041034A2401A43B26313
:105C6800F0E700BF6E390590807E049070B5054658
:105C780080690E462EF0C7FA044638B1064A334604
:105C8800022106482DF09BFB204670BD314605F1E8
:105C980038002DF020FFF7E785390590807E0490C5
:105CA80070B50646EFF31181102282F31288BFF314
:105CB8006F8F1D4C236881F31188BFF36F8F5B686A
:105CC80093F87030DB0705D40A220023BDE8704042
:105CD80005F026BBEFF3118382F31288BFF36F8FB1
:105CE800256865B983F31188BFF36F8F2368D3B133
:105CF800304600220023BDE8704005F0DDBA616837
:105D08002A688D42226008BF626083F31188BFF35E
:105D18006F8F686805F10801C369984729460348E9
:105D28002FF0F9FFE2E770BD18200024F40B0024DF
:105D380030B585B00546002316486C4684E8060051
:105D4800002203A904F0AEFE0246E8B9039B94E8DA
:105D580003005D60083383E80300EFF3118010232C
:105D680083F31288BFF36F8F039B1A600A4A516846
:105D780061B9C2E9003380F31188BFF36F8F002245
:105D88000023064805F098FA05B030BD0B60536053
:105D9800F1E700BFF40B00241820002400000024C1
:105DA800D3B50026002704460648CDE900672DF044
:105DB800ABFC20B1230604765CBF0023038202B04B
:105DC800D0BD00BFD40C00242DE9F04383B00023DC
:105DD8001D4C4FF00108056902AF1C4E05F124095E
:105DE80028602B7785F82030B442234601D3002061
:105DF80019E095F820201034CAB16C4688B01B68A9
:105E080002AA1349C2E905134FF400739383114B97
:105E180042F8103F104800234FF4E251FDF764FAAE
:105E28006FF00B00A5460437BD46BDE8F08385F842
:105E38002080484654F8043C009354F8101C54E958
:105E480003232EF01BF8CFE7C8B00590C8B0059023
:105E5800AF39059003000001987E04901FB5CDE985
:105E6800010103924FF0FF324FF0FF3301A90348BD
:105E78002FF0B4FF002005B05DF804FB380C0024B7
:105E880013B514464A780369FE2A14D14A8892B990
:105E9800CA8882B193F820300BB1013BDBB20122F2
:105EA8000DF1070104F10C008DF807302DF051FCBD
:105EB800002002B010BD034B6FF08502FEF784FA94
:105EC8001A50F5E70C0000001FB500230190CDE93A
:105ED80002334FF0FF324FF0FF3301A902482FF091
:105EE8007DFF05B05DF804FB380C002408B54B783D
:105EF800FF2B07D14B882BB9CB881BB9FFF7E4FFE1
:105F0800002008BD034B6FF08502FEF75DFA1A50BA
:105F1800F6E700BF0C0000002DE9F04103680446D5
:105F280017460E461B695B6893F80B804046FFF7DF
:105F380037FFD4F87B2005460146D21B2068C4F8F9
:105F48007B202DF007FE88B10B4A434601210B4800
:105F58002DF035FA314620462DF0D6FE2846FEF7BC
:105F6800C3FD2046BDE8F0412DF08ABEA37F013372
:105F7800A377BDE8F08100BFC6390590987E0490EC
:105F88002DE9F8430368054630274FF024081B69BC
:105F98005B689E7CEB7F012B20D82B68D3F8109090
:105FA80099F8614017FB04844C4420462DF08CFF7F
:105FB800B0F5007F636A044628BF4FF4007499F86F
:105FC8001F2024F03F047BBB3AB1041BB4F5007FCB
:105FD80028BF4FF4007424F03F040CB9BDE8F883DF
:105FE80028462DF0EDFD2246014681463046FFF752
:105FF800D7FE0446014628682DF0ACFD80B1134A4F
:106008003346012112482DF0DAF92046FEF76CFDDF
:10601800494628462DF078FEBDE8F8432DF030BEFD
:10602800EB7F0133EB77B5E7B4FBF3F45C43002A6D
:10603800D3D0001BB0F5007F28BF4FF4007020F0CC
:106048003F00B0FBF3F000FB03F4C6E7C639059048
:10605800987E04902DE9F04FDFF8EC9287B04FF06E
:10606800FF324FF0FF3303A9B84804F0B9FDDDF85B
:106078000C80049DD8F81040002D40F0978004F162
:106088002406257794F820309D42C0F2898004F1D7
:106098001803BFF35B8F53E8002F22F0020243E896
:1060A80000210029F7D1BFF35B8FBFF35B8F53E863
:1060B800001F21F0040143E80012002AF7D1BFF3C2
:1060C8005B8FBFF35B8FA369BFF35B8FDB07C6D51D
:1060D800237F022B00F07781032B00F0708143BBF4
:1060E800DDF80CB0DBF81050EB7F13BB6B6828466B
:1060F80093F812802DF064FD402201460646404682
:10610800FFF74EFE0746014658462DF023FD0028AE
:1061180000F051818E4A434601218E482DF04FF9F7
:106128003846FEF7E1FC314628462DF0EDFD2DF00E
:10613800A7FDA37F002B92D1237F012B40F068811C
:10614800302394F8615004F1630694F8621003FB5D
:1061580005453046243500F04FFA3146024623699A
:10616800284600F067FA0646C4F8840028462DF051
:10617800A1FE804628462DF0A2FE074628462DF0AF
:10618800A3FEE26D3044002A40F02681002840F04A
:106198001E8128462DF0BFFE003818BF012017E1E8
:1061A8003046013530362DF07CFE6BE7059AD8F87D
:1061B80004B02B7E3AB3298A71326648009107BF32
:1061C8000221654A0121654A2DF003F9D8F810200B
:1061D8002B7E5268917C994240F0DF80E37F5A1E03
:1061E800E2776A680AB1023BE377696920462DF0D5
:1061F8008BFD6B6813B159692DF086FD2946584609
:106208002DF0C0FC5DE76168887C984240F0918081
:10621800227FEF68B5F810A0002A48D1BAF11F0F05
:1062280041D13B684B453ED1394604F1540307F14F
:106238001C0251F8040B914243F8040BF9D10A8867
:106248001A808A7842219A705523E26D84F8733057
:106258005323C4F87B2084F8743084F87630A36D17
:1062680084F87510C4F877300023C4F8803094F8A7
:1062780060309A060FD194F8612094F820309A4241
:1062880009D294F86230013B0F2B04D8012384F81B
:106298007F3023779AE720682DF0A6FC022384F844
:1062A8007F300423F5E720462DF0EAFC8EE7032A29
:1062B8008CD1302294F8616002FB0646D4F8802025
:1062C80052442436C4F88020BAF1000F15D0304665
:1062D8002DF0FAFD88B13946524630462DF007FEBA
:1062E800074628B91E4A534602211A482DF067F876
:1062F800D4F87B30DB1BC4F87B30D4F88020E36D06
:106308009A420DD230462DF0DFFD00287FF45EAFB3
:10631800D4F88020E36D9A4202D220682DF06AFCFE
:1063280030462DF0F8FD003818BF012084F87F00B2
:10633800B7E7C97A99427FF449AF237F298A052BA9
:1063480010D1227742E700BF55534243380C00244E
:10635800C6390590987E0490EB3905900F3A059060
:10636800303A0590022B7FF431AFD4F880302068A2
:106378000B4494F86160C4F880302DF041FC00288B
:106388007FF424AFD4F87B3013B120682DF02CFCB7
:10639800302303FB06402430C3E7D27A9A427FF4C5
:1063A80024AFA37F5A1EA2776A68002A3FF41DAF64
:1063B800023BA37719E7EB7F0133EB77B9E6204679
:1063C800FFF7DEFDB5E620462DF0AEFCB1E6022073
:1063D80084F87F0004231AE094F9601040B900297A
:1063E800206802DA2DF000FCD3E62DF003FCD0E69D
:1063F800002914DA904202D8B8F1000F06D12068BB
:106408002DF0F2FB022384F87F30E3E702232377A1
:10641800237F022B0CD120462DF086FC1FE69042EC
:1064280000D81FB920682DF0E5FBEBE70323EEE762
:10643800032B03D12046FFF7A3FD10E6042B7FF4BE
:106448000EAEA37F2BB11E4A01211E482CF0AEFFD1
:1064580005E6236820461B695B68DF7A2DF0B0FBF0
:1064680004F173030546024604F17F0153F8040B57
:106478008B4242F8040BF9D11B7829463846137031
:106488000D22FFF78DFC0646014620682DF062FBC1
:1064980078B10D4A3B4601210A482CF090FF30465E
:1064A800FEF722FB294620462DF02EFC2DF0E8FBB6
:1064B800D5E5A37F0133A37705232377CFE500BF75
:1064C800563A0590987E0490C6390590802938B5CB
:1064D8000D46144621D083290DD019BB80230320F3
:1064E80011715371832393710023E0700430657038
:1064F8002370A37038BD0223137101235371002345
:1065080093710A23D37108224168A01841F0F8F862
:10651800064B0E201B882382E6E7044B02201B88CB
:106528009380E1E76FF08500E4E700BF279A0590C4
:106538002DE9F04187690446D0F82480BA4228BF83
:106548003A46B2FBF8F5C2692B4600682DF073F89D
:10655800064648B9B7FBF8F7AF4207D0E3692B44C2
:10656800E361606A684312E00025012600220521E4
:106578002068FDF7D5F960B1094A012109482CF0D6
:1065880015FFE3692B44E361074B0020A362BDE8D4
:10659800F081E3692B44E361002EF5D1E1E700BF08
:1065A800773A0590987E04900203000C81420B46CE
:1065B80007B509D30D4A02210D482CF000FF6FF0F2
:1065C800150003B05DF804FB6AB10139114481423A
:1065D80001D28B4207D90221009305481346054A88
:1065E8002CF0F7FEEBE70020EBE700BF8E3A0590B2
:1065F800987E0490A53A05900C290346084616D1C2
:106608001B78252B12D009D8122B10D8084A42FA29
:1066180003F313F0010F08BF0620704703F0FD02D3
:10662800282A03D05A2B08BF0A2070470A2070472F
:10663800F6FFFBFF2DE9F0411E4690F82C30062AA4
:1066480086B023F00C030446884680F82C304FF0BF
:1066580000038361C0E904330B7840F00C81D3B99F
:106668004D7915F0040540F0168290F82C309B0700
:106678000AD402234FF468521D4684F82950002595
:1066880084F8283062853AE02DF07CFB0028F0D1B0
:106698002B462A46F1E7032B35D14F7917F004072B
:1066A80040F0F98190F82C308DF8077043F004031E
:1066B8008DF808708DF8097080F82C3070230D79EA
:1066C80001A9ADF8043090F82930122D8DF80A7020
:1066D80003F00F0328BF122503978DF806300A230D
:1066E8002A46ADF812708DF80B30438D3046ADF860
:1066F80014705BBAADF8103040F0A3FFA7622846CB
:1067080006B0BDE8F081122B4BD14B795F0700F141
:10671800C28190F82C3043F0040380F82C304B7879
:1067280013F0020723D113F0010F8B7819D0B1F8B9
:106738000350324619466DBAFFF7C8FEADB285421E
:1067480006DAB8F8030040BA80B200231A4613E00C
:10675800324698F802102046FFF7B8FE0028F4DA0F
:1067680005E083B1AB4A0221AB482CF028FE022396
:1067780005274FF410520020054684F8283084F885
:1067880029706285BBE7B1F8035031462DF02DFB27
:106798006DBAADB28542D4DB314620462DF025FBDB
:1067A800DCE71A2B27D14D7915F0040540F07381E9
:1067B80090F82C3043F0040380F82C308B783F2B72
:1067C80014D1CF7897B90D79032301A93046042D48
:1067D800019328BF04252A4640F033FF3A463B463A
:1067E80084F8282084F82970638588E70222052721
:1067F8004FF41053F4E71B2B23D14D7915F0040502
:1068080040F04981097990F82C200809C2F3400327
:106818000AD18E0708D5C80711D402F00302032A4B
:1068280000F03E81002301E0002BF6D094F82C20E4
:1068380063F3410284F82C2000231A461DE7012344
:10684800F4E71E2B40F022814D7915F0040540F045
:1068580022810B7913F0030306D0012BECD190F8B9
:106868002C3043F0010303E090F82C3065F300036B
:1068780084F82C30E0E70A2A40F00881232B40D125
:106888004B7A13F0040340F0068190F82C20ADF801
:10689800043042F004028DF80630082380F82C20DA
:1068A8008DF807302DF06EFA002801A93046ABBFED
:1068B800236A4FF0FF3302220322A8BF1BBA8DF8C8
:1068C8000C200293636A1BBAC3F307228DF80D30BC
:1068D800C3F307438DF80E208DF80F3094F82C3051
:1068E80043F0040384F82C30B8F807506DBAADB201
:1068F8000C2D28BF0C252A4640F0A3FE0023A362D6
:10690800FDE6252B2ED14F7A17F0040740F0C380FF
:1069180090F82C3043F00403990780F82C3006D403
:1069280002274FF46853002584F828705AE72DF0A1
:1069380029FA0028F4D1236A93B1013B1ABA1B063D
:1069480022F07F4294F82C001A43616A002340F039
:106958000400082509BA84F82C0032607160E3E766
:106968001A46EFE7282B2BD14D7A15F0040540F095
:10697800928090F82C30D1F8027043F00403B1F8FB
:1069880007609A0780F82C307FF573AE2DF0FAF97E
:1069980000287FF46EAE76BA3FBA206AB6B239469E
:1069A8003246FFF703FE20B1022305254FF40452B7
:1069B80063E61A4BE7612361636A7343A36167E681
:1069C8002A2B2FD14D7A15F0040564D190F82C307C
:1069D800D1F8027043F00803B1F8076080F82C3052
:1069E8009B077FF546AE2DF0CDF900287FF441AE28
:1069F80076BA3FBA206AB6B239463246FFF7D6FDB4
:106A08000028D1D1064BE7616361636A7343A361D0
:106A180012E700BFCF3A0590987E0490573E039046
:106A2800396500905A2B31D14D7A15F0040532D1D1
:106A380090F82C3043F0040380F82C308B783F2BEF
:106A480019D1CF78E7B94FF4C0633046CDE90135A5
:106A5800B1F8075001A96DBAADB2082D28BF0825B5
:106A68002A4640F0EEFD00231A4684F8283084F8C0
:106A78002970628543E6022305274FF41052F4E794
:106A8800022305274FF410520025EEE7074A01219B
:106A980007482CF094FC022305254FF41052ECE52E
:106AA8000223052545F20232E7E500BFEC3A0590DE
:106AB800987E049007B5094A6B4692E8030083E87C
:106AC800030007488268126822B11946904703B04C
:106AD8005DF804FB6FF05700F9E700BFB87E04903B
:106AE800F879049000F01F0201215F2801FA02F2F0
:106AF80008B5034605D90C480C4A2CF060FC002068
:106B080008BD1F284FF0B04106D8D1F888309A4305
:106B18000CBF01200020F3E73F2802D8D1F89830B5
:106B2800F5E7D1F8A830F2E7B87D0490073B059067
:106B380000F01F0201215F2801FA02F208B503469E
:106B480006D90B480B4A2CF03AFC6FF0150008BD2B
:106B58001F284FF0B04103D8C1F888200020F6E77D
:106B68003F2802D8C1F89820F8E7C1F8A820F5E72F
:106B7800B87D0490073B0590044B03EB40000023CD
:106B8800013320F8022B9942FADC70475C06002496
:106B98002DE9F041054600260F4F4FF00108F4B2E9
:106BA8006B78A34201D8BDE8F0812B781C442046BD
:106BB800FFF798FF68B12046FFF7BAFF57F834305F
:106BC8003BB107EBC40204F01F04516808FA04F053
:106BD80098470136E3E700BF20200024034680B130
:106BE800B0FA80F2C2F11F02D2B2074931F912009D
:106BF8004FF0B042D2F880100B43C2F88030FDF756
:106C08001BBBFF22F1E700BF5C06002430B5B0B122
:106C1800B0FA80F3C3F11F03DBB20B4850F83340DE
:106C28008C4204D100EBC3056D68954205D044B988
:106C380040F8331000EBC3004260002030BDFF2352
:106C4800EBE76FF00F00F9E72020002460B1B0FAFD
:106C580080F3C3F11F03DBB2044A002142F833106A
:106C680002EBC30251607047FF23F5E720200024A0
:106C780000F003020F23043292009340094A43EACA
:106C8800900000F00303023352F82320030C93FA18
:106C9800A3F3B3FA83F302EA104003F01F03D840CA
:106CA800704700BF000400582DE9F04705468946A3
:106CB80090461F46D0F808A02DF02CFA0446D0B113
:106CC800067FF3070AD590F8203018480121184AA2
:106CD8002CF075FB6FF07700BDE8F0873B46424625
:106CE80049462DF0D1F948B994F82030114A0121CC
:106CF8000E482CF064FB6FF01200EDE79DF8203091
:106D080026F0060684F8218021466784284684F800
:106D180024302677DAF818309847B0FA80F3227FC3
:106D28005B0963F300022277D6E700BF487E049030
:106D3800553B05906F3B059070B5054686682DF06C
:106D4800E9F90446D8B1037FDB0709D490F820306D
:106D58000C4801210C4A2CF032FB6FF0770070BD13
:106D68000146F3692846984738B1237F03F00103A9
:106D7800227F63F300022277F1E70346F8E76FF01A
:106D88001200ECE7487E0490913B0590064B1B6986
:106D980003F03803102B05D0182B044818BF002027
:106DA800400870470248FBE70044025800389C1C22
:106DB80040787D01354B10B518680B88C3F30B0379
:106DC800132B38D813B96FF0850033E0013B122B31
:106DD800F9D801A454F823F06B6E00902D6E009042
:106DE800CF6D0090816E0090CF6D0090CF6D0090B8
:106DF800CF6D0090716E0090756E0090756E00906A
:106E0800CF6D0090CF6D0090CF6D0090716E0090A7
:106E1800796E00907D6E0090CF6D0090636E00904B
:106E2800636E00904FF4004010600B68B3F5805F0C
:106E380024D2002010BDD42B0FD003F62873C3F33F
:106E48000B031C2BBFD8012404FA03F3104C234274
:106E580005D140F211142342B5D04008E4E7800878
:106E6800E2E7FFF793FFDFE70A48DDE70A48DBE7D9
:106E78000A48D9E70A48D7E70A48D5E7C3F31333DE
:106E88000133B0FBF3F01060D3E700BFB003002478
:106E98000010111100389C1C001C4E0E006CDC0206
:106EA800C9F6930040787D0137B5984CD4F8E030A6
:106EB80043F00073C4F8E030D4F8E03003F0007316
:106EC8000193019B236843F480232360236843F4E0
:106ED8008033236023689803FCD5FBF7E9FE236F12
:106EE8008A4A23F018032367236F43F001032367BB
:106EF800136F9907FCD5FBF7F9FE854B9A6942F4A5
:106F080040429A619A699204FCD5804B1A6902F052
:106F18003802182A16D11A68550706D41A6842F09A
:106F280001021A601A685407FCD5784B1A6922F0D6
:106F380007021A611A6912F0380FFBD19A6922F018
:106F48000F029A61714B1A6822F080721A601A68EF
:106F580022F080621A601A6822F080521A609A6AD7
:106F680022F0030242F002029A629A6A22F47C72C8
:106F780042F050029A62DA6A22F00C0242F00802E9
:106F8800DA62DA6A22F00202DA621A6B22F4FF721B
:106F980022F0010242F0BF021A63DA6A22F001020B
:106FA800DA621A6B22F47E4242F400721A63DA6AD9
:106FB80042F48032DA621A6B22F4FE0242F4403262
:106FC8001A63DA6A42F40032DA621A6B22F0FE427D
:106FD80042F040721A63DA6A42F48022DA621A686E
:106FE80042F080721A601A689001FCD59A6A474C80
:106FF80022F07C7242F4A0029A62DA6A22F44062B9
:1070080042F40062DA62DA6A22F40072DA621A6C16
:1070180022F4FF7222F0010242F0BF021A64DA6A17
:1070280022F48072DA621A6C22F47E4242F4007210
:107038001A64DA6A42F48002DA621A6C22F4FE02F6
:1070480042F498121A64DA6A42F40002DA621A6C9C
:1070580022F0FE4242F0C4421A64DA6A42F08072B8
:10706800DA621A6842F080521A6023689900FCD5E7
:10707800FFF78CFE05462748854201D202F070FAD8
:10708800A369224A23F47063A361A36923F00F0361
:1070980043F00803A361E36923F0700343F040035E
:1070A800E361E36923F4E06343F48063E361A36984
:1070B80023F0700343F04003A361236A23F07003B5
:1070C80043F040032362236923F0070343F00303DB
:1070D8002361136903F03803182BFAD10D48854250
:1070E80001D302F03DFA0A4B9A6942F440429A6190
:1070F8009A699204FCD5054A0020136923F40043D9
:107108001361054B054A1A6003B030BD00440258AC
:1071180000480258001C4E0EB003002400389C1C86
:10712800132808D8054BC34013F0010F14BF0020E3
:107138006FF0850070476FF08500704716C70D0027
:1071480008B507482EF051FD38B10648FDF788FB11
:107158000448FBF765FD002008BD6FF01200FBE74F
:10716800D47B0490717100900A2838B50446074D05
:1071780004D1AB680D2128465B689847AB68E1B23B
:1071880002485B689847204638BD00BFD47B04900E
:1071980098B5406800AF046B0369DCB133BB204687
:1071A8002EF023FD034640BB21686C4688B06A4632
:1071B8001548C2E905014FF400719183134942F85B
:1071C800101F13484FF4E251FCF78EF86FF01200CD
:1071D800A54602E01BB96FF05700BD4698BD214691
:1071E80010302DF063F900EAE070F6E70021103066
:1071F8002DF05CF90028D2DAEFE7A3681B68002BB2
:10720800E9D020469847E8E7BD3B05900300000118
:10721800B07D049098B5406800AF046B0369DCB199
:1072280033BB20462EF0E1FC034640BB21686C4688
:1072380088B06A461548C2E905014FF40071918388
:10724800134942F8101F13484FF4E251FCF74CF869
:107258006FF01200A54602E01BB96FF05700BD465B
:1072680098BD012110302DF021F900EAE070F6E711
:10727800012110302DF01AF90028D2DAEFE7A368BF
:107288005B68002BE9D020469847E8E7BD3B0590AE
:1072980003000001B07D04902DE9F8431C46D0F8A6
:1072A80004809B88D8F800500B440669089FAB42BD
:1072B800D6F8B80005D8E388D8F804C01344634565
:1072C80008D919480121194A2CF070F86FF01500F7
:1072D800BDE8F88396F8A93005FB02114FF00009C4
:1072E80001FB0305E2881FFA89F39A4201D80020BE
:1072F800EEE7A388294696F8A92038465A4340F075
:10730800A0F9A18896F8A9305943384609F101092E
:10731800FDF7B8F896F8A930D8F8002002FB035515
:10732800228903FB0277DDE7B07D0490D93B059005
:107338002DE9F843D0F804801D46B3F804E0046949
:107348000EEB0103D8F80000089F834205D8EE88A9
:10735800D8F804C09319634508D930480121304A48
:107368002CF024F86FF01500BDE8F88352EA010903
:1073780094F8A93029D1704527D1B44525D12E8953
:10738800864222D10CFB06F1384604F1BC0559436C
:10739800FDF778F8284603F0DFFD23680122C4F8DA
:1073A800B470DA632268536B43F0010353634FF000
:1073B800FF324FF0FF33284603F0A8FD2268536BD5
:1073C80023F0010353630020CEE75843D4F8AC60A0
:1073D8004B434FF0000902FB00321644EA881FFABB
:1073E80089F39A42EFD9AB88394694F8A9203046F8
:1073F8005A4340F026F9A98894F8A93059433046F1
:1074080009F10109FDF73EF894F8A930D8F80020F1
:1074180002FB03662A8903FB0277DFE7B07D04904D
:10742800D93B05902DE9F743476806460569BB68CF
:1074380083B14FF4D01107F108002DF01CF8041E99
:1074480008DA3D4A01213D482BF0B0FF204603B041
:10745800BDE8F0833B694BB14FF4B01107F1100060
:107468002DF009F8041E01DA354AEBE701AA0021DC
:10747800B86A2DF048FC041E07DB019B002219792D
:10748800186801F055FA041E01DA2E4ADAE7DFF827
:10749800B880B969D8F80890D9F800302BB14046BF
:1074A8009847041E04DA294ACCE76FF05704FAE734
:1074B800FB69012B0ED9B969D9F81830083133B1F5
:1074C800002240469847041E04DA214ABAE76FF0C2
:1074D8005704FAE7D7E908018368DB6803B19847DE
:1074E8004FF40473A5F8A8300122002105F1BC006F
:1074F8002EF05AFDFB6A30469847164A284613680C
:1075080023F00D0313602DF069FE044600289DD179
:10751800024605F1380128462DF0BEFE0446002833
:1075280094D12A68D2F8043123F00103C2F8043157
:10753800094B18648AE700BF013C0590B07D0490B0
:10754800353C05906C3C0590F8790490863C059094
:10755800AD3C05900040005200100050064A1168EA
:107568000B6823F004030B60044B506819688368A8
:107578005B6803B11847704734020024A002002456
:10758800094B10B5D3E90040084B196883681B689C
:1075980003B19847236843F004032360236843F04A
:1075A8000803236010BD00BF34020024A002002499
:1075B80008B5EFF31181102383F31288BFF36F8F9F
:1075C800084B012093F8482083F8480081F311887C
:1075D800BFF36F8F22B9FFF7D3FF5020FCF72CFEC3
:1075E800002008BD34020024F8B51646837890F8C8
:1075F80003C0EFF31182102484F31288BFF36F8F56
:10760800077890F801E0DB1B3C4603EA0C039E4236
:1076180088BF9EB2BD190CEA0505057082F3118872
:10762800BFF36F8F8A198A421AD177450CD1EFF3CD
:107638001182102181F31288BFF36F8F0178417096
:1076480082F31188BFF36F8F02799B1B9A4205D38F
:107658002EF025FD60B1084803F0BEFD3046F8BDA8
:10766800051901346D7904EA0C0401F8015BDAE7C5
:10767800FFF79EFFF2E700BF6C0200242DE9F843F4
:10768800134F0D46144607F1560807F1180914B9A7
:107698002046BDE8F8834FF0FF324FF0FF333846FD
:1076A80003F034FC224629464046FFF79DFF064674
:1076B80030B94FF0FF324FF0FF33484603F026FC55
:1076C800A41B3846354403F0E5FBA4B2DFE700BF4E
:1076D8003C02002438B54368046922486060196890
:1076E80083681B6803B19847012204F1080011461A
:1076F8002EF05AFC0122002104F1200000252EF072
:1077080053FC04F1380018492EF09DFC07232A4643
:10771800294684F861300423502084F85E5084F8A8
:1077280062300F2384F85F5084F84C300C2384F8BF
:10773800605084F84D3084F8495084F84A5084F8F1
:107748004B502BF0A2FF094B1B681A6842F0040249
:107758001A601A6842F008021A60FFF729FF2846E3
:1077680038BD00BFF8790490C14503903402002465
:10777800164B014610B51A68EFF31184102383F3F2
:107788001288BFF36F8F53685B0605D45368D80718
:1077980013D46FF00A000BE06FF0400353600C2322
:1077A800013B9068FCD153685B06EFD56FF004008D
:1077B80084F31188BFF36F8F10BD506810F040003C
:1077C800F4D193680B60002BF2D1E2E73402002475
:1077D8002DE9F347D8070F46144605D42E48FFF77E
:1077E80003FF02B0BDE8F087002A37D0EFF3118518
:1077F800102383F31288BFF36F8F5020FCF73EFDF0
:1078080006465020FCF726FD85F31188BFF36F8FDD
:10781800DFF88880FFF7B4FED8F800305A685107BF
:1078280014D45B685A0611D4DFF874904FF4803A88
:107838002546C9F888A1D8F800305B68DB070FD463
:10784800BFF34F8F20BF40BF20BFF4E7002401A83B
:10785800FFF78EFFE6B15020FCF7EEFC2046C0E7AC
:1078680001A8FFF785FF0028C9F888A1E3DB6A1E95
:10787800291F019B17FA82F289B2013D02F80139EA
:107888001B0AADB2002DE5D08D42F6D10193D2E7A7
:10789800FFF764FEE2E700BF7D0200243402002403
:1078A80000E100E02DE9F74301A8FFF761FF002898
:1078B80044DB284C0021019A042794F84B30884671
:1078C80094F84CC0084694F84AE0A3EB0E055FFA1A
:1078D80082F93CEA05051ED194F8600094F85F60CF
:1078E80094F86150861B35EA06062AD109B184F856
:1078F8004B30B8F1000F00D001925020FCF7AAFCE1
:10790800FFF72CFE002384F84830134803B0BDE885
:10791800F04303F0BFBAE118013381F84E900CEA46
:1079280003030121013F4FEA12224FF00108CCD195
:1079380009B184F84B3001920028E6D103B0BDE8C4
:10794800F08326180130054086F86390012084F8FA
:107958006050E7E73402002454020024C3780F2B58
:1079680014D9C96B0B480B0E00EA911013708B02E7
:10797800090603F47C0301F0FE41034310680B433E
:107988000549014000200B43136070476FF08500E4
:10799800704700BF00FF0300FF00008000487047E9
:1079A800E8810490F0B5154602681E468FB013684A
:1079B80004460F4602A823F040030021136030223A
:1079C8003FF067FE5A23082141F288322046CDE96C
:1079D80000374FF4005303934FF48073CDE9051338
:1079E8004FF48063694607934FF08073CDE90936F9
:1079F8002DF095FD034668B10D4A0E4801212CF083
:107A0800E2FE6FF004002268136843F0400313603D
:107A18000FB0F0BD41F28832294620462DF006FE0F
:107A2800034608B1044AE8E7C4F89000EBE700BF52
:107A3800133D0590C87D0490373D059038B58B629D
:107A4800002304461546C0F890302DF0ACFD0346DF
:107A580038B10D4A0D4801212CF0B5FE6FF0040035
:107A680038BD294620462DF042FE034608B1084A93
:107A7800F0E74FF0FF324FF0FF3304F1640003F0FA
:107A880045FAD4F89000EBE74F3D0590C87D049087
:107A9800733D0590002310B5C0F8903004462DF0D2
:107AA80082FD034638B109480121094A2CF08BFEB2
:107AB8006FF0040010BD4FF0FF324FF0FF3304F1B8
:107AC800640003F023FAD4F89000F3E7C87D04902B
:107AD8004F3D059038B58B62002304461546C0F823
:107AE80090302DF060FD034638B10D4A0D48012154
:107AF8002CF069FE6FF0040038BD294620462DF0B1
:107B08002EFE034608B1084AF0E74FF0FF324FF067
:107B1800FF3304F1640003F0F9F9D4F89000EBE7BF
:107B28004F3D0590C87D0490733D05902DE9F04FB9
:107B38000D1E91B0064614467CDBD0F80490AA18B6
:107B48004FEAE5734FF00001D9F80C0043F1000348
:107B5800904271EB03036DD3002C39D0382202A870
:107B6800D6F810803FF095FD4FF480724FF4806393
:107B7800DFF8C8A04FF0FF3B4046CDE9082398F84E
:107B8800BF3013F0010F0CBF4FF400534FF44053B4
:107B980005932CF028FE514630690395FFF77AFFCC
:107BA800D9F80C300027A34216D1C72302A930699F
:107BB80002930997FFF76EFFD9F80C30E41A3046A4
:107BC8002CF082FE002CE6D130694C302CF0F9FD07
:107BD800204611B0BDE8F08F08F1840308F18C004D
:107BE80045EA040C5A785AB10BFA02F13CEA010151
:107BF80006D117B17978914202D21A781F460292BB
:107C080002339842EED147B102A93069FFF742FF2B
:107C18007A78012393401D44D0E7094A234601217D
:107C2800084800956FF015042BF0D3FB30462CF074
:107C38004BFEC9E76FF01504CAE700BFF081049056
:107C48008B3D0590C87D04902DE9F0470D1E8EB040
:107C5800074690461E4665DB4068AA194FEAE57359
:107C68004FF00001C06843F10003904271EB030339
:107C780058D3002E59D0342201A83FF00AFD3869A4
:107C88004FF48073DFF8A890069390F8BF3013F094
:107C9800010F0CBF4FF400534FF44053039390F877
:107CA800BC30322B009314BF4FF440634FF4806311
:107CB80007934FF0407309932CF095FDB6F5007FBC
:107CC800B2464FEA5522494628BF4FF4007A386930
:107CD8000AEB0503013BB2EB532F1CBFC5F3080A9F
:107CE800CAF5007AFFF7D6FE044698B953464246CD
:107CF800694638690195FFF7A1FE044650B9384630
:107D0800A6EB0A062CF0E0FDD0445544044608B919
:107D1800002ED3D138694C302CF053FD20460EB0DC
:107D2800BDE8F0876FF01504F8E73446F6E700BFC2
:107D3800F08104902DE9F04FB5B047680669044614
:107D480020AA0021B8692CF0DEFF051E07DB209B66
:107D580000221979186800F0EBFD051E06DA2B469B
:107D6800AB4A0121AB482CF02EFD08E0DFF8A882D1
:107D7800D8F80890D9F800302BB96FF004052846D8
:107D880035B0BDE8F08F394640469847054600288B
:107D9800F3D1D9F80C30002BEFD008AA3946404669
:107DA80098470028E9DB089A2846034601303D69D0
:107DB800B2FBF0F18D4203D2B0F5807FF5D10346D6
:107DC80073604025FA68304692FAA2F3002AB3FAA3
:107DD80083F308BF4FF0FF33013B33613B7D013B29
:107DE80073610023C6E9073501F018FA80460028B8
:107DF800C3D1012206F14C0011462EF0D5F801221C
:107E0800414606F1640066262EF0CEF8BB6820468F
:107E180098473422414621A83FF03BFC4FF4407379
:107E280020A9206926932096FFF734FE034628B13F
:107E38007A4A012177482CF0C6FC1CE0992520A934
:107E480020692095FFF726FE034608B1744AF0E73B
:107E58004FF4807320A9206926932096FFF71AFE15
:107E680003460028E4D120A920692095FFF712FED7
:107E780003460028EAD10A202DF090FE18230CAA08
:107E880000212069FFF78EFD054610B10346654ABB
:107E980067E70C9B644A934207D0644A01215D4816
:107EA8006FF015052CF08FFC69E79DF836300EAAA7
:107EB8004FF0010B012B164697BF01331023DBB29D
:107EC800DB00D3180293029B2069B34200F0F280D2
:107ED800F279337843EA0223B3F57F4F40F0DD812E
:107EE800F37871799B00B27909023779502B41EA0E
:107EF800024120AA28BF50233943FFF753FD824689
:107F0800002840F0D180219A2769002A616807F18A
:107F1800840973DA22F000420123A2F1200AC2F197
:107F2800200003FA02F203FA0AFA23FA00F04AEAF6
:107F3800000AD208C96842EA4A72B1EB420F4FEA16
:107F4800420304D03A4A012132482CF03CFC002379
:107F58004FF0010AC7F88430C9F804304A46514640
:107F680020A82CF0B1FB20B999F80130013389F829
:107F780001300AF1010A09F102095FFA8AFABAF135
:107F8800050FEBD1F3780A2B89BF2A9B4FF4807336
:107F9800C3F303130BFA03F35B00A7F88C30209BA1
:107FA800C3F34143012B49D10AAA20A93046FFF760
:107FB800D5FC002844D19DF82830980740D099076F
:107FC800206904D51B49FFF765FD8246C0B93422F4
:107FD800002113A83FF05DFBB72312A92069129373
:107FE8004FF480731893FFF755FD824640B997F810
:107FF800BF3043F0010387F8BF3021E0013298E732
:1080080053460D4A012103482CF0DDFB4CE000BF2C
:10801800A43D0590C87D0490F8790490C33D05906F
:10802800DF3D0590FC3D059053464450113E0590B8
:10803800293E0590F0810490433E0590022BD6D04E
:1080480040F204730DF1140A4FF00009ADF8143032
:10805800FF2387F88F301AF8012B07AB20A9304689
:1080680003922CF0C3FA002810DB039A9DF81C3009
:1080780087F88F2087F8BD309DF81D209DF81E30A9
:1080880087F8BE3012B1134487F8BE30B9F1000F3B
:1080980037D097F88F30FF2B36D16FF0850A854A95
:1080A800012185482BF082F95346844A01218248F0
:1080B8002CF089FB22696368B2F88C0002F108068B
:1080C800D968134693F884403CB193F88540B8F1D9
:1080D800000F01D0444500D2A04602339E42F1D1A0
:1080E800B8F1000F00F0DB80012303FA08F35C1EEF
:1080F800044208BF0346C2F88030B1FBF3F3D367EC
:108108003DE64FF00109A6E709AA20A930462CF060
:10811800EFFA031E10DA6A4A022167482CF053FB73
:10812800236993F88E30062B00F2B480DFE803F061
:10813800B58C0B908C8C8C009DF82430C3F34203D3
:1081480087F88E30ECE740274FF0010906AA494628
:1081580020462CF09CFBB0F1000A7EDB9DF818202D
:108168009DF81930174202D03B4240F096803A43BE
:108178003B43544920698DF818208DF81930FFF7D2
:1081880089FC8246002865D112AA012120462CF0DC
:108198007EFB824600285DD19DF848309B07F3D5C9
:1081A8009DF849309807EFD50021342213A8D4F858
:1081B80010A0CDE90A113FF06CFA0123B9F1010FC3
:1081C800BDF8182012934FF4807318934FF0807302
:1081D8001B939AF88E3043D1012BADF8282053D148
:1081E8000DF12A02022120462CF051FBB0F1000AC1
:1081F80033DB0AAA042312A92069FFF71FFCB0F198
:10820800000A2ADB20462CF05FFBB0F1000A24DBD1
:1082180006AA494620462CF03AFBB0F1000A1CDBBE
:108228009DF818209DF81930174201D03B4234D1EF
:10823800BDF81830244A012100934B461E486FF0C0
:10824800040A2BF0C6F808E002274FF002097DE780
:108258008027FAE7BAF1000FA6DA53461B4AD1E69F
:108268003121012BADF82A20129102D0043B012BB9
:108278000DD80AAA012120462CF009FBB0F1000A0A
:10828800EBDB01231293B4E70AAA0223B3E70DF14B
:108298002A02FAE76FF0850ADFE7083613E66FF07F
:1082A80085030B4A012104486FF012052CF08BFA64
:1082B80065E500BF603E0590C87D0490F13E0590DD
:1082C800833E0590F0810490AE3E0590D23E059025
:1082D800053F05900048704728820490044BB3F886
:1082E80080389B020B60002318464B60704700BF24
:1082F80000E0F11F064B186828B94FF0010C4FF445
:108308000030C3E900C0012010600B60704700BF57
:10831800A02000240B4A5369DB0312D5002910DD85
:1083280000F1006300F01F000144BFF34F8F2039B4
:10833800C2F85C3220330029F9DCBFF34F8FBFF35A
:108348006F8F704700ED00E037B505682C6914F0B1
:10835800C06F0AD02B6EC3F30E030C4A02210C48DF
:108368005B01009301232BF034F80A480A4B2040A4
:108378006B6108D001230648084A194600942BF07F
:1083880028F86FF0040003B030BD00BF463F0590E9
:10839800D07D04900000EE150F00EF1F613F05909F
:1083A80070B5054610461A46EFF31186102383F37D
:1083B8001288BFF36F8F012383F31388104C63690E
:1083C80043F480736361BFF34F8FBFF36F8F01F185
:1083D80000613FF036F9002383F31388636923F4BF
:1083E80080736361BFF34F8FBFF36F8F86F311887C
:1083F800BFF36F8F2869BDE87040FFF7A5BF00BFC6
:1084080000ED00E0F7B517461A4606460D461C462D
:108418002CF08FFA50B90B482B460B4A01210094D7
:108428002AF0D7FF6FF0150003B0F0BD44B1234622
:108438003A462946304603B0BDE8F040FFF7B0BFE2
:108448002046F1E7D07D0490773F059007B50BB142
:10845800CB0604D103B05DF804EB2CF06ABA2023F4
:10846800054A064800930B4601212AF0B2FF002076
:1084780003B05DF804FB00BFA13F0590D07D0490D8
:10848800D3B50446154A002368462DF08CFF2069B1
:10849800DDE90067FFF758FF00280EDB002223699B
:1084A8001B68186910F0040009D052B14FF4FA5350
:1084B8000B4A01210B482AF082FF6FF0040002B03A
:1084C800D0BD32463B4668462DF092FFDDE90032CA
:1084D80013430CBF01220022E1E700BF80380100EE
:1084E800F33F0590D07D04902DE9F84FB1F5003F9A
:1084F800036907460D4690461E6809D32F480B4668
:108508002F4A01212AF05BFF6FF01500BDE8F88FB4
:10851800F46814F0010402D06FF00400F6E7FFF7E6
:10852800AFFF0028F2DB05F1006505F120022B46BC
:10853800D3E90001B1F1FF3F08BFB0F1FF3FEBD134
:1085480008339342F4D1F36843F00203F360BFF3B6
:108558004F8FDFF868B008EB040158F804204B6827
:108568002919C1E90023BFF34F8F2DF01AFF0A2202
:108578000023F9F7B3F810F1640941F1000A3369EF
:108588005B070FD52DF00DFF0A220023F9F7A6F897
:1085980081457AEB0101F2DA64230A4A012158463F
:1085A8002AF00DFF0834202CD5D13846FFF768FF94
:1085B800F36823F00203F360A8E700BFD07D0490BE
:1085C8000740059021400590013A2DE9F041074602
:1085D8000D4600205618DFF87080AE420CD33B6978
:1085E800B5F5003F1C6809D318482B46184A0121E5
:1085F8002AF0E5FE6FF01500BDE8F081E368DB07BF
:108608001ED43846FFF73CFF0028F5DBE36823F467
:10861800E063E360E36843F00403E360E36843F086
:108628008003E360BFF34F8F3846FFF729FFE36805
:10863800002803EA0803E360DEDB05F50035CCE734
:108648006FF00400D8E700BFFBF8FFFFD07D04906F
:10865800074005902DE9F743012306460F461446C7
:10866800FFF7F4FE60B96FF015053B46224A012179
:10867800224800942AF0ADFE284603B0BDE8F083F6
:10868800002C36D030692CF04DF933691B68DA6854
:10869800D20723D4224604F5FF34DFF86490394624
:1086A80004F5FF743046FFF78FFF07EA09083C44DA
:1086B8000546404604EA0901A1EB0801FFF72AFE36
:1086C800336930461C68FFF7DBFE68B1002D08BF30
:1086D80005463069043002F0DDFBCDE7094A5A60EF
:1086E80002F188325A60D5E7E36843F00103E3609A
:1086F800ECE72546C0E700BF32400590D07D0490E6
:108708000000FEFF230167452DE9F041044600699A
:1087180015461F460E462CF005F923691B68DA68D2
:10872800D2071BD43B462A46314620462CF016F980
:10873800236905462046D3F80080FFF7A1FE98B1CB
:10874800002D08BF054639463046FFF7E3FD20698E
:10875800043002F09FFB2846BDE8F081064A5A60C3
:1087680002F188325A60DDE7D8F80C3043F0010393
:10877800C8F80C30E4E700BF23016745F7B51C468D
:1087880017460123064622460D46FFF75FFE50B9FD
:108798000B482B460B4A012100942AF01AFE6FF071
:1087A800150003B0F0BD44B123463A462946304689
:1087B80003B0BDE8F040FFF7A7BF2046F1E700BFD0
:1087C800D07D04905D4005902DE9F843D0F80490E1
:1087D800904607460D46D9F808001E462BF0E7FBE1
:1087E800B8F5001F044616D1D9F808402846FEF708
:1087F8003FFA84420CD129462BF0D9FB04462BF0D2
:10880800DBFB2046FEF722FA002120462BF0DDFB99
:108818000020BDE8F883B8F5800F20D0B6F1806F4E
:1088280019D0B6F1C06F18D0B6F1007F1AD1022660
:108838003A460F492046FEF7E9F9B0B9D9F80810C9
:1088480028462BF0EBFB204631462BF0BEFB20469A
:10885800FEF7C4F9DCE70126EAE70326E8E76FF04C
:108868008500D6E76FF01500D3E76FF00F00D0E76B
:10887800CF4B039008B5416805480C3183681B68E5
:108888001BB1984700EAE07008BD6FF05700F9E7A0
:10889800F87904901FB50C4B0C29D3F8082828BF89
:1088A8000C2112BA0C460192D3F8042812BA02928B
:1088B8000A46D3F8003801A91BBA03933EF0C1FE5B
:1088C800204604B010BD00BF00E0F11F37B5456871
:1088D80001AA0021E8682CF016FA041E07DB019BA8
:1088E80000221979186800F023F8041E08DA0C4AE7
:1088F800234601210B482AF062FD204603B030BD13
:108908000948696883681B682BB19847041E05DA13
:10891800064A2346EDE76FF05704F9E70024ECE731
:108928004E410590F87D0490F87904906C410590CB
:108938002DE9F047044600EBC10600251C4FB44260
:1089480001D1002014E02068C30600F01F0911D4EB
:10895800656845F02005C0F3481AC0F3442019287B
:1089680023D857F82080B8F1000F0DD16FF012000E
:10897800BDE8F087B9F1100F04D0B9F1110FEAD1B1
:108988006568E8E73025E6E740462DF02EF900282F
:10899800ECD04B462A460AF00F0140462CF029F944
:1089A800002804F10804CADAE2E76FF01500DFE7EF
:1089B800C084049043681B6803F1080252E8002F42
:1089C80042F0010203F1080040E800210029F3D138
:1089D800154A93421BD0A2F54C42934217D002F598
:1089E8008062934213D002F5806293420FD002F561
:1089F800806293420BD002F54442934207D0A2F51D
:108A08001C42934203D002F58062934203D15A6814
:108A180042F040025A6053E8002F42F4807243E863
:108A280000210029F7D170470010014043681B68F6
:108A380003F1080252E8002F22F0010203F10800B6
:108A480040E800210029F3D1154A93421BD0A2F532
:108A58004C42934217D002F58062934213D002F53C
:108A6800806293420FD002F5806293420BD002F5E8
:108A78004442934207D0A2F51C42934203D002F528
:108A88008062934203D15A6822F040025A6053E848
:108A9800002F22F4807243E800210029F7D17047A3
:108AA800001001402DE9F04182B080460D46436830
:108AB80000AF1E68002936D0586819698368DB68DA
:108AC8006BB13A1D9847041E0CDA1A4A01211A485C
:108AD8002AF06CFC20460837BD46BDE8F0816FF0EF
:108AE8005704F2E7336823F4004333607B6803EBF1
:108AF8005503B3FBF5F30F2B18D86C468AB0D8F89A
:108B080000306A460D49D561C2E905134FF4007378
:108B180013840B4B42F8103F00234FF411510648C1
:108B2800FAF7E2FBA5466FF01504D3E79BB20024E1
:108B3800F360CFE7D8410590407E04900642059047
:108B480004000001F8B50C46036941681D682379E3
:108B5800012B15D09F1E7E427E41B6026279022A01
:108B680096BF464F4FF4005737F81270A279022A81
:108B780009D0042A30D0003B18BF01231B0306E0AC
:108B88004FF4C066EAE7B3FA83F35B091B07E2799F
:108B98000968012A14BF4FF0000C4FF4407CA5422D
:108BA8001DD10A6822F0805222F4B05232431A438F
:108BB8000A604B6823F440533B434B6043681A6890
:108BC800936823F4407343EA0C0393602968FFF722
:108BD80069FF00EAE070F8BD4FF48053D7E7D1F899
:108BE80000E00EF4C06E764506D0D1F800E02EF411
:108BF800C06E4EEA06060E6041680E68716801F4A0
:108C080040518F4204D0716821F44051394371605A
:108C180041680E68316801F010218B4204D0316838
:108C280021F010210B433360436819688B6803F403
:108C380040739C4505D08B6823F4407343EA0C03CA
:108C48008B6043681B689968490405D5032A09D0D5
:108C58009A6822F4804204E0032A03D19A6842F415
:108C680080429A6021682B68994205D0FFF71AFF65
:108C78000028B0DB23682B600020ACE7782805903B
:108C88002DE9F04383B00546466800AF7068316946
:108C980083681B685BB96FF057046E4A01216E4800
:108CA8002AF084FB20460C37BD46BDE8F083984780
:108CB800044630BB3A1D0021706A2CF024F8041ECB
:108CC800F0DB7B68002219791868FFF731FE041E73
:108CD800E8DBD5F804802B69D8F80040D3F8009079
:108CE800236823F001032360D8F808002CF07DFFE7
:108CF80078B95A4A012158486FF012042AF056FBF5
:108D0800D0E7544A012154482AF050FB002CC9DB13
:108D1800D0E7D8E902018368DB6803B1984754E8D3
:108D2800003F43F00C0344E80032002AF7D14946DB
:108D38002846FFF707FF002802DA6FF01504B1E7AD
:108D480098F818301BB1A36843F00803A36098F89B
:108D580019301BB1636843F40043636098F81A3014
:108D68001BB1636843F48033636098F81B301BB110
:108D7800636843F40033636098F81C30002B53D0C9
:108D8800374B9C4233D0A3F54C439C422FD003F57C
:108D980080639C422BD003F580639C4227D003F567
:108DA80080639C4223D003F544439C421FD0A3F523
:108DB8001C439C421BD003F580639C4217D0294B6F
:108DC8009C4214D06C4688B02B686A462649C2E992
:108DD80005134FF400739383244B42F8103F00238C
:108DE8004FF4E2511C48FAF77FFAA546A5E76B68ED
:108DF8001A68936843F480439360236898F81D20A9
:108E080023F0787343EA42532360236898F81E20BE
:108E180023F4F81343EA0243236098F81F301BB188
:108E2800A36843F40043A36098F820301BB123687B
:108E380043F000532360236843F001032360E36990
:108E48009A02FCD5E3695B02FCD5B36A2846002484
:108E5800984727E71D420590407E04903D420590C3
:108E680000100140000C0058584205900300000112
:108E7800F8B5436802460E4691F805E01C68036998
:108E880008791D6801288B7913D1BEF1020F6CD9BE
:108E9800022B1F464FF4C0614FF4005C7DD0042BB9
:108EA80076D000287ED0C31E012B73D86FF08500C2
:108EB800F8BD02280AD1BEF1020F62D9022B1F4663
:108EC8004FF480610BD04FF4005CE8E7BEF1020F6D
:108ED8005AD9022B1F4659D100286ED00021C31E33
:108EE800012BE3D90020022703237345DED12BF0A1
:108EF80056FFB842DAD1F3791BB3012B65D1344B55
:108F08009C421ED0A3F54C439C421AD003F58063C3
:108F18009C4216D003F580639C4212D003F580630F
:108F28009C420ED003F544439C420AD0A3F51C434F
:108F38009C4206D003F580639C4202D0254B9C429C
:108F4800B4D123683146104623F001032360FFF7AC
:108F5800F9FD0028AADB236843F00103236096E8A3
:108F6800030085E803000020A2E74FF4C0611A4F10
:108F7800022B37F81EC01F4691D170B94FF08050B0
:108F880010E04FF48061F2E70021F0E700219AE752
:108F980000288BD14FF4805004E0C31E012B85D9E3
:108FA80002270020BCF5805F0BD0BCF5405F0AD0DB
:108FB800BCF1000F98D1012397E701464FF080508C
:108FC80092E7002391E702238FE7032B97D06DE701
:108FD80000100140000C0058782805904FF0E0235D
:108FE8000F4910B59C691A6908689B6902F48032B8
:108FF8000C4934B993B903464AB90A681044C01AEF
:1090080010BD002B08BF03460AB9A342F5D90A6868
:1090180002440A604FF0E0221269EEE70446F3E7E3
:109028005C21002458210024094B1022002083F8D9
:1090380023204BF68032074B1A604BF67F32064BE3
:1090480018604FF0E0235A61072298611A6170474F
:1090580000ED00E05C21002458210024684620F03F
:1090680007018D4619B5FFF7B9FF1149114B08687B
:10907800D3E90042001942F10002C3E900020E4A96
:1090880000230B604BF68033D2E90041001BB0FB94
:10909800F3F043431B1941F10001C2E9003102F02A
:1090A8008DFEFAF739FDBDE819408546704700BFC7
:1090B80058210024E81A0024E01A00242DE9F04180
:1090C800DFF8E08099B1421C0BD14FF0E022136920
:1090D80023F0010313614FF07F43C8F80030BDE867
:1090E800F081D8F80060012807DC00270BE0431C5A
:1090F800D8F80060F7D14FF4AE7040F25D13984293
:10910800A8BF1846471EEFF31185102383F3128872
:10911800BFF36F8FFFF762FF234C4FF0E02399698D
:10912800D4E9002380184FF0000243F10003C4E99A
:1091380000031E4B1A601E4B1A68831A2ED44BF676
:10914800803C0CFB073303F53B437F33B3FBFCF751
:10915800131A40F6B8320CFB0733934238BF134654
:10916800144A934228BF1346C8F800304FF0E02253
:10917800013B90695361002381429361A1EB000395
:10918800D4E9001238BF9B195B1842F10002C4E908
:10919800003285F31188BFF36F8FA0E740F6B8332C
:1091A800E2E700BF5C210024E81A002458210024CB
:1091B800E01A002400E2FE0038B5EFF31185102311
:1091C80083F31288BFF36F8F084B1C68084B1B682A
:1091D800E41AFFF703FF85F31188BFF36F8F4BF68F
:1091E80080332044B0FBF3F038BD00BFE81A0024F8
:1091F800E01A002438B5EFF31185102383F31288A1
:10920800BFF36F8F044B1C68FFF7E8FE85F31188E6
:10921800BFF36F8F204438BDE81A002437B50446E1
:109228002AF011F80546002C41D094F841302BB9AA
:1092380020462CF073F941F28833A3642168204654
:10924800A3680A68013B22F4F85242EA03220A6042
:109258000022A36C202100932B462CF038F920BB68
:109268002168E569E3680A682B43256A22F07F4292
:109278002B43656822F0D00243EA056313430B6071
:109288002168D4E905324D681343226943EA024351
:10929800084A2A4013434B602268136843F00103CD
:1092A80013600123606484F8413003B030BD0120AD
:1092B800FBE700BFFEF8E0FF38B50368044699688D
:1092C8001A68480734D5550332D594F84120122A34
:1092D80014D122689168480703D420462CF09AFAE2
:1092E80038BDE16AF9B1626A127883F82020626AAF
:1092F80001326262E26A013AE262EAE794F84120E6
:10930800222AEAD1226891684907E6D5A16B51B1B2
:1093180093F82010226B1170226B01322263A26B2A
:10932800013AA263EEE7136823F480231360D4E7BD
:109338008D076CD590036AD50222DA60226813681B
:1093480023F4E023136094F84130122B14D12368DE
:109358001A68510709D51A6822F004021A60E36BEB
:109368001A68D36823F00103D3600123204684F8E8
:1093780041302BF0C6FAB3E794F84130222B27D1BD
:1093880023681A6852071DD51A6822F004021A6069
:10939800E36B1A68D36823F00103D36001232046E6
:1093A80084F841302BF0AAFA9AE7A26B002AF5D08C
:1093B80093F82010226B1170226B01322263A26B8A
:1093C800013AA2632268926812F47C5FEDD1E5E766
:1093D80094F84130022B06D10123204684F841300D
:1093E8002BF089FA7CE794F84130082B7FF478AFAA
:1093F80022682046536923F040635361012384F8AF
:109408004130636C002B3ED12CF003FA68E70D075E
:1094180012D5100310D50822DA6023681A6855029D
:1094280006D51A6822F410221A60012384F8413004
:1094380020462BF069FA53E7C80727D5D50325D569
:109448000125DD602268136823F470231360636CC0
:1094580043F00203636423681A68500710D51A683A
:1094680022F004021A600F4AE36B9A65E06B2BF056
:1094780061FF00283FF434AF636C43F00403636476
:10948800204684F841502BF030FA29E7C9067FF5C9
:1094980027AFD2027FF524AF10222046DA602BF0E6
:1094A80036FA1DE7E157039038B50D460446F0B18A
:1094B80090F82C3003F0FF021BB980F82D202CF017
:1094C800AAF90223211D206884F82C3000F014F832
:1094D8006268294620682CF0D6F9064A00201368ED
:1094E80043F000431360012384F82C3038BD012079
:1094F800FCE700BF0040005230B50A684D6AD1E968
:1095080007342343154C92B902682B432240134376
:109518004A6813438A681343CA6813430A691343A2
:109528004A6913438A6913430360002030BD026807
:109538002B4322F4F8421343036043684A682340EC
:1095480013438A681343CA6813430A6913434A6971
:1095580013438A6913434360E7E700BF0080FFFFB6
:10956800002854D02B4A936903F44043B3F5404F85
:109578001FD1294B294A0344934242D9284B294AEF
:10958800034493423FD9284B984240D80020274AA9
:10959800136823F00F0303431360136803F00F03EA
:1095A800984232D0136803F00F03C01A18BF012085
:1095B8007047936903F44043B3F5004F0ED11C4A3A
:1095C8001C4B02449A421AD91B4A02449A4218D99F
:1095D8001A4A02449A4216D90133D5E7184A194B58
:1095E80002449A4209D9184A02449A4207D9174AAA
:1095F80002449A4205D9164AEBE70420C7E703203C
:10960800C5E70220C3E70120C1E70346CDE70120F3
:10961800704700BF00480258FFC4A7F7FFE0F505F0
:109628007FE2D3FB7F1D2C04801D2C0400200052F8
:10963800BF4C2AF6BF3B47037F8871F93FC4B8FC8B
:10964800FF6A45F53FA5AE023F10F4F77FB5A2FAD1
:10965800BF5A51FD10B50A46044619B1024B002104
:109668001B68984710BD00BFB403002403460A4A8C
:1096780000209A6002F18832DA6002F12942A2F5EC
:109688009612A2F68B621A61A2F188325A61034AD5
:10969800C3E900009A61704701234567F0E1D2C32E
:1096A8002DE9F04F4B68AFB0D1F800E01BBA8E68D7
:1096B800CD689EFA8EFE089336BA0B692DBA0190D2
:1096C80093FA83F84B6993FA83FA8B691BBA0A9366
:1096D800CB691BBA12930B6A93FA83FB4B6A1BBACA
:1096E8000B938B6A1BBA0C93CB6A1BBA0D930B6B4B
:1096F8001BBA0E934B6B1BBA03938B6B1BBA049369
:10970800CB6B1BBA059383680F93C36802930369F5
:109718000F9906934369029F10938369109A1393D4
:10972800069B83EA0200029B1840E04B5040139AC4
:1097380003EBB7071A442F4402EBF1620299104475
:10974800069A82EAB1020F9970448EEA060E0A4020
:1097580006998EEA0B0E4A40109919440A44089952
:109768000A440F994FEAB10C029902EBF0628CEAB5
:10977800B104044084EAB10406991944314486EAE4
:1097880008060C448CEAB001114004EBF2644FEA7D
:10979800B20281EA0C019C4482EAB409394482EAA3
:1097A800B007C444274001EBF46187EAB00709EA2F
:1097B800010967440AEB030C89EA020907EBF16720
:1097C8000CEBB00C0A984FEAB101E144184481EA65
:1097D800B40C104409EBF7690CEA070C129A8CEAEE
:1097E800B40C1A44844481EAB70002EBB40200EADC
:1097F80009000CEBF96C484010444FEAB9020BEB36
:10980800030982EAB704894400EBFC6004EA0C040B
:1098180084EAB70404EB090182EABC04DDF82C9061
:10982800044001EBF06199444FEAB000544009EB61
:10983800B7090C9F4C4480EABC091F4409EA010996
:1098480004EBF16417440D9A89EABC091A44B94437
:1098580080EAB10702EBBC02DDF838C0274009EB0B
:10986800F4694FEAB4049C444740844484EAB9004C
:10987800174484EAB10202EA090207EBF96782EAAF
:10988800B10238406244DDF80CC060409C4402EBF1
:10989800F7624FEAB7070CEBB10C0499604487EA0A
:1098A800B90C19440CEA020C00EBF2602144059C47
:1098B8008CEAB90C1C448C4487EAB20104EBB90465
:1098C80001400CEBF06C4FEAB0007940214480EA8B
:1098D800B20401EBFC69039904EA0C048EEA010165
:1098E80084EAB20403EBF17E07910899BE4481EA49
:1098F80005070B99744485EA0A054F40049904EB5F
:10990800F964794080EABC0703EBF17E07EA0907AE
:1099180008914FEAB9010EEBB20E0C9A4740564037
:10992800059A7744564007EBF46703EBF67E4FEA57
:10993800F67286440D98149281EABC024540079855
:10994800224085EAF07082EABC0211904FEAF0707A
:10995800119D7244159081EAB40003EBF573384009
:1099680002EBF76203EBBC0348404FEAB707184421
:109978000A9B87EAB40988EA03080E9B89EA020968
:1099880000EBF26088EA0308089B88EAF3730993FE
:10999800099D474B03EBF57C039D8C4412998AEA99
:1099A8000101E14487EAB20A6940129D8AEA000A85
:1099B80009EBF06981EAF6714FEAB00003EBF17C3C
:1099C8000CEBB40C0A9C84EA0B08049CE24488EA79
:1099D8000408119C0AEBF96A88EAF47803EBF87C2E
:1099E8004FEAF874BC440B9F169480EAB20485EAE7
:1099F800070E059D84EA09048EEA050E099D644454
:109A080080EAB90C8EEAF57E04EBFA648CEA0A0C5B
:109A180003EBFE774FEAFE7507EBB2070C9A129537
:109A28004FEABA0A079D8BEA0202BC448AEAB907E0
:109A380082EAF57267400CEBF46C82EAF17203EB90
:109A4800F27B0A920B9A83440D9D07EB0B0082EA86
:109A58000507089A0E9D00EBFC6087EAF27787EA13
:109A6800F8728AEAB4070B9203EBF27B0C9A87EA46
:109A78000C070BEBB90B82EA05090D9A5F444FEA14
:109A8800BC0C89EAF6768CEAB40986EAFE7689EA9D
:109A9800000907EBF0674FEAF67503EBF67B1795BD
:109AA800039DD34482EA050A04E000BF9979825AEB
:109AB800A1EBD96E119AD9448AEAF2750A9A8CEA0E
:109AC800B00A85EAF2758AEA070A09EBF76903EB37
:109AD800F57B4FEAF5720BEBB40B0D924FEAB70723
:109AE8000E9A0AEB0B04DDF810A004EBF96482EA85
:109AF8000A0A099A8AEAF27A0B9A8AEAF27287EAD9
:109B0800B00A03EBF27B0C928AEA090A039AE3444F
:109B18000AEB0B0CDDF814A082EA0A0A0CEBF46CD1
:109B28008AEAF17A8AEAF67287EAB90A03EBF27BE3
:109B380003928AEA040A049A0BEBB00B0798DA44FA
:109B48004FEAB40B82EAF0748BEAB90084EAF8743D
:109B580080EA0C000AEBFC6A84EAF57403EBF478FB
:109B68004FEAF472B8440E9200EB0807059A089879
:109B780007EBFA6782EAF0700C9A80EAFE708BEACB
:109B8800BC0E80EAF2708EEA0A0E4FEABA0A03EBBC
:109B9800F0784FEAF07208EBB9081192C644149AAB
:109BA800DDF81C800EEBF76E82EAF8780A9A88EAEC
:109BB800F278039A88EAF2728AEABC0803EBF2792F
:109BC800049288EA0708159AD944C844DDF8209019
:109BD80082EAF9790B9A08EBFE6889EAF27989EA50
:109BE800F4728AEAB70903EBF27B059289EA0E0957
:109BF800149A0BEBBC0B4FEABE0E09EB0B0CDDF80D
:109C0800249082EAF9790CEBF86C89EAF6798EEA05
:109C1800B70689EAF07986EA08064FEAF97203EB93
:109C2800F97B1492D344159A06EB0B0A82EAF17673
:109C3800049A86EAF5768EEAB80586EAF27685EA27
:109C48000C050AEBFC6A4FEAF67203EBF67B1592F9
:109C58004FEABC0C169A0BEBB70B099F5D4482EADE
:109C6800F7770C9A05EBFA6587EAF277059A87EA9F
:109C7800F2728CEAB807079203EBF27B129A87EA32
:109C88000A07F3448CEABA0E82EAF171039A5F4438
:109C98008EEA050E81EAF271169A07EBF56781EAFA
:109CA800F97B4FEAB50503EBFB7101EBB8018E4474
:109CB8000A9982EAF1710EEBF76E81EAF47485EA8B
:109CC800BA0184EAF67479404FEAF47203EBF47847
:109CD8001692E044129ADDF82CC0414482EAFC7CDA
:109CE800079A01EBFE618CEAF07085EAB70C80EA0E
:109CF800F2708CEA0E0C01EABE0803EBF0734FEA2F
:109D0800F07203EBBA0312929C440A9A179B0CEB6D
:109D1800F16C83EAF272049B82EAF37282EAFB73C3
:109D28000893089AE74B03EBF272154441EABE0226
:109D380002EAB70205EBFC6542EA0802DDF82C806E
:109D48002A440D9D85EAF875DDF8148085EAF875D2
:109D58004CEAB10885EAF47508EABE0809950CEAE8
:109D6800B10548EA0505DDF8248003EBF87808EB2F
:109D7800B70805EB0807179DDDF8308007EBF26799
:109D880085EAF87888EAF97802EABC0988EAF0787E
:109D98004FEAF8750B9503EBF87505EBBE0E42EA32
:109DA800BC050EEBF76E05EAB10545EA0905DDF8D5
:109DB8000C90AE440D9D85EAF97547EAB20985EA2B
:109DC800F676089D09EABC0986EAF5764FEAF67543
:109DD8000D9507EAB20549EA050503EBF67909EBA3
:109DE800B1090E994D44DDF8309081EAF971DDF83A
:109DF8001C9005EBFE6581EAF971DDF8249081EA93
:109E0800F9710EEAB7090A9103EBF17101EBBC0C89
:109E18004EEAB7010CEBF56C01EAB20141EA09011F
:109E2800DDF80C906144DDF844C08CEAF97C45EA21
:109E3800BE098CEAFB7C09EAB7098CEAF87CCDF804
:109E48000CC005EABE0C49EA0C0CDDF80C9003EBDB
:109E5800F97909EBB2090E9ACC44DDF8109082EA40
:109E6800F9720CEBF16C82EAF47401EAB50984EA40
:109E7800F6744FEAF4720E9203EBF47202EBB70732
:109E880041EAB50207EBFC6702EABE0242EA0902B0
:109E9800DDF814901744119A82EAF9724CEAB10974
:109EA80082EAF0700A9A09EAB50980EAF2704FEA84
:109EB800F07211920CEAB10249EA020203EBF0795E
:109EC80009EBBE09DDF850E04A44DDF810908EEA4F
:109ED800F97EDDF8209002EBF7628EEAF97EDDF874
:109EE8000C908EEAF97E03EBFE79CDF810E007EAD4
:109EF800BC0E09EBB50947EABC0509EBF26905EAAE
:109F0800B10545EA0E05DDF814E0A944159D85EA7A
:109F1800FE75DDF824E085EAFE7502EAB70E85EAEB
:109F2800F475059542EAB70505EABC0545EA0E0E43
:109F3800059D03EBF57505EBB1051499AE44079D36
:109F480081EAF5710EEBF96E81EAF87809EAB20553
:109F580088EAF0784FEAF871149103EBF87101EB95
:109F6800BC0C49EAB2010CEBFE6C01EAB7012943CB
:109F78000EEAB9058C44159981EAFB7A04998AEAB4
:109F8800F67A079E8AEAF17A4FEAFA7115914EEA53
:109F9800B90101EAB2010D4303EBFA7101EBB70114
:109FA8000D44169981EAF6710A9E05EBFC6581EA73
:109FB800F671059E81EAF671089E03EBF177079129
:109FC8000CEABE0107EBB2074CEABE0207EBF567E5
:109FD80002EAB9020A4305EABC011744129A82EA66
:109FE800FB7B039A8BEAF27B45EABC028BEAF87B9F
:109FF80002EABE02114303EBFB7202EBB902114401
:10A00800169A82EAF67601EBF76186EAF47686EA32
:10A01800FA764FEAF67203EBF674169247EAB5023F
:10A0280004EBBE0402EABC0207EAB50E04EBF164D5
:10A0380042EA0E02DDF824E01444129A82EAFE7223
:10A0480041EAB70E82EAF070079A0EEAB50E80EA86
:10A05800F2720C924FEAF2720C98129201EAB7026D
:10A068004EEA020203EBF07E08980EEBBC0E02EB00
:10A078000E0C0B9A04EAB10E82EAF07204980CEB0B
:10A08800F46C82EAF0720D9882EAFB72089203EB94
:10A09800F27202EBB50244EAB10502EBFC6205EA92
:10A0A800B70545EA0E050CEAB40E2A44099D80EA74
:10A0B800F575059885EAF07585EAF6704CEAB405F9
:10A0C80002E000BFDCBC1B8F099005EAB10545EA38
:10A0D8000E0E03EBF07505EBB705AE44DDE90A504B
:10A0E8000EEBF26E80EAF5750C984EEAB20985EA35
:10A0F800F87502EABC0885EAF075039809EABC0914
:10A108004FEAF577179703EBF57707EBB10742EAC4
:10A11800BC0107EBFE6701EAB40141EA08010EEA57
:10A12800B2080F440D9949EA080881EAF0710898C5
:10A1380081EAFA714FEABE0A81EAF0718AEAB20E40
:10A1480003EBF1734FEAF1708EEA070E03EBB403E9
:10A158000D9008EB03040A980E9B04EBF76483EA5E
:10A16800F073079883EAF073099883EAF0730A9307
:10A178000A98DF4B03EBF078119808EBBC08DDF880
:10A188000CC080EAFC7CC6448AEAB7088CEAFB7CEF
:10A198000EEBF46E88EA04088CEAF5704FEAB40412
:10A1A80003EBF07C0B9004980CEBB20C0E9A82EA4D
:10A1B800F079E04484EAB70C059889EAF6798CEAE4
:10A1C8000E0C08EBFE6889EAF1794FEAF9720E92F3
:10A1D80003EBF97252449444119A82EAF0760C9A8D
:10A1E8000CEBF86C86EAF2760A9A86EAF2764FEA7F
:10A1F800F67203EBF6700C9284EABE0200EBB7002D
:10A20800149F82EA080202444FEAB800DDF8108081
:10A2180080EABE0A87EAF877DDF820808AEA0C0A25
:10A2280002EBFC6287EAF877DDF82C8087EAF8779A
:10A238004FEAF777039719971F442744159CBA44A8
:10A24800059F84EAF774099F0AEBF26A84EAF774B7
:10A2580084EAF9744FEAF4740494049F1A9480EA27
:10A26800BC041F4454404FEAB20207EBBE070592F4
:10A278003C44149A079F04EBFA6482EAF778059A3B
:10A2880088EAF57882EABC05159A88EAF67885EABC
:10A298000A054FEAF87808EB0307CDF86C80074405
:10A2A8003D4482EAFB77059A87EAF177039982EAC7
:10A2B800BA00169A4F4005EBF46560404FEAB404C3
:10A2C8004FEAF77784EABA0EF9181C978EEA050E5A
:10A2D80001EBBC010844079982EAF1710A9A00EB84
:10A2E800F56081EAF271049A5140059A4FEAF171DA
:10A2F80001EB030C1D919444129AE64482EAFB7226
:10A30800DDF82CC00EEBF06E82EAFC7284EAB50C24
:10A3180082EA08028CEA000C4FEAB0004FEAF272B7
:10A3280002EB030B1E920BEBBA0BDDF858A0DC44D2
:10A33800DDF820B08AEAFB7A0CEBFE6C8AEAF97A3F
:10A348008AEA070A4FEAFA7980EAB50ACDF8149042
:10A35800CDF87C9099448AEA0E0AA144129CCA441A
:10A36800DDF8249084EAF9740AEBFC6A84EAF6744E
:10A3780080EABE064C4086EA0C064FEABC0C4FEA5F
:10A38800F4748CEABE09079420941C4489EA0A09EB
:10A3980004EBB504039D2644179C84EAFB7406EB82
:10A3A800FA666C4054404FEAF474E5182194054469
:10A3B8000D98A944099D80EAF570049D09EBF6699A
:10A3C8006840059D68408CEABA054FEAF070754010
:10A3D8004FEAB60600EB030B22900BEBBE0BDDF841
:10A3E8005CE05D44DDF828B08EEAFB7E05EBF9659C
:10A3F8008EEA080EDDF81C808EEA080E86EABA0896
:10A408004FEAFE7E88EA09080EEB030BCDF88CE0D4
:10A41800E344DDF834C0D844DDF82CB08CEAFB7C8A
:10A4280008EBF5688CEA070C8CEA040C86EAB90498
:10A438004FEAFC776C404FEAB50507EB030C24970D
:10A448000CEBBA0CDDF828A06444DDF838C08CEABF
:10A45800FA7C04EBF8648CEA010C8CEA000C85EABF
:10A46800B9004FEAFC7180EA080001EB030C259162
:10A47800B4440C9E86EAFB766044564085EAB802EE
:10A4880000EBF46086EA0E0662404FEAB4044FEA35
:10A49800F6762D9426961E4406EBB9063244039EA2
:10A4A80002EBF06C0E9A5640059A56400C9A7E4084
:10A4B80084EAB8074FEAF67647404FEAB000279695
:10A4C8001E442C902E44049D5540079A374455400D
:10A4D8004FEABC0207EBFC674D4084EA00012A976B
:10A4E80018954FEAF57581EA0C012B9202E000BF3E
:10A4F800D6C162CA28951D4405EBB8054B190F99BA
:10A5080003EBF76329930B4401998B60029B1F446B
:10A51800069B1A44109BCF601844139B0A611C4485
:10A52800486118A88C615821FFF794F800202FB0D3
:10A53800BDE8F08F03460846C1B90E4ADFF838C0B7
:10A54800C3E910110D49C3E912120D4A0D49C3E9B7
:10A5580014C20D4AC3E916120C4A1A6602F1745263
:10A56800A2F52302A2F692425A6670476FF0730072
:10A57800704700BF85AE67BB72F36E3C67E6096A39
:10A588003AF54FA57F520E518C68059BABD9831FB6
:10A598002DE9F04FCFB0044600F1480300F16806FA
:10A5A80046AD03911868083353F8041C2A46B34291
:10A5B80003C21546F6D1DDF834B104AA4A984FF023
:10A5C800000CDDE94883DDE94B9601933D4BDDE95D
:10A5D80046150293BCF10F0F5CD8039B53F82C303F
:10A5E8001BBA4FEAF02E86EA0907DDF808A00CF13D
:10A5F800010C8EEAB01E07409360BCF1400F8EEA52
:10A60800706E87EA060702F1040277445AF804EBF1
:10A61800774445EA010ECDF808A005EA010A3B4453
:10A628004FEA71370EEA080E87EAB1075B444EEA33
:10A638000A0EB34687EAB1577744DDF804E0CDF84F
:10A6480004809E443B441ED1CDE94631CDE9043710
:10A6580045A904F144036434CDE94C96CDE94AE0B8
:10A66800CDE9485853F8042F51F8040FA342024487
:10A678001A60F7D104A84FF49471FEF7EBFF00209D
:10A688004FB0BDE8F08FA8464E460D4681461946A4
:10A6980070469FE7136852F834AC4FEAF34E52F80D
:10A6A800387C8EEA734E8EEA932E52F8143C3B4463
:10A6B8004FEABA4787EAFA17734487EADA073B444E
:10A6C8008FE700BFD485049070B5044688B103783D
:10A6D800C3B10D4D0D4EB54201D3002409E02968E0
:10A6E800A14208D128462BF080FA002814BF2C4636
:10A6F8000024204670BD2046F7F70AF80028F1D05C
:10A708001C35E8E71C46F4E7F8790490607C04906F
:10A7180010B50446F8F718FD03480121034A28F04C
:10A7280045FE20462BF06CFA207E0490A542059049
:10A738002DE9F843044600AF0D46EFF311881023C6
:10A7480083F31288BFF36F8F0428294AE9468AB039
:10A7580098BF284B9668117C6A4694BF53F82030FE
:10A76800254BC2E9073140F2013324489384244B36
:10A77800C2E9050442F8103F00234FF43151214843
:10A78800F8F7B2FDCD4645B1EB69C3F3080323B131
:10A798001D4A01211B4828F009FE2EB130462BF036
:10A7A80087FC08B1037803B91848E9468AB06A46B5
:10A7B800174BD061C2E9053640F201331384154BBB
:10A7C80042F8103F00234FF411510E48F8F78CFD62
:10A7D80029462046CD46FFF79BFF88F31188BFF333
:10A7E8006F8F3046F9F7BCFCBD46BDE8F88300BF63
:10A7F80060210024D4860490B4420590CA42059092
:10A8080005000001207E0490F2420590C2420590A6
:10A81800134305900400000138B50A4B53F8204053
:10A82800013053F82050A54200D838BD606830B1D7
:10A83800037EDB0701D42BF0C0F90834F3E7236863
:10A848009847FAE7E88604902A4B0122032070B55E
:10A85800294C86B0294D1A70FFF7DEFF01F038FC4D
:10A868000420FFF7D9FF26463034AE4210D3224CDD
:10A8780000F082FF224EAC4226D300F091FF27F071
:10A8880090FE204A938923F00103938106B070BD9E
:10A8980054F80C3C059354F8103C049354F8143CB9
:10A8A800039354F8183C029354F81C3C019354F851
:10A8B800203C009354E90A2354E90C0100F036FDCA
:10A8C80054F8303C5E65CEE7D4E90A23B3F1FF3F84
:10A8D80008BFB2F1FF3F05D052EA0301206803D157
:10A8E80001F030F83034C6E73146183001F0D6F9B7
:10A8F800F8E700BFA2280024607C0490907C0490B4
:10A9080099610390901B002470B5A023154E86B062
:10A91800012203FB00660023134D044601931349EB
:10A92800CDE904230F22CDE9023214234FF4A0729B
:10A9380003FB00554FF4C0700D4B00FB041130466B
:10A94800009500F0F3FC337C0A4A23F00403EE6020
:10A958002C7433744FF4046304FB033313446B60A7
:10A9680006B070BDF01A00246021002400430024C2
:10A978008F5D0390C03A0024BFB50020FFF74CFF5D
:10A98800274B83F30888274D0024F023264F85F8AA
:10A998002230EC772C766C76AC7685F820406B6AA2
:10A9A80043F4E0236B62F9F7EFFAF9F7E9FC4FF0AB
:10A9B800FF33AB62EB62F9F763FE1C4DF9F7A8FDB4
:10A9C800F8F724FB1A4800F043FDF8F7C9F901200D
:10A9D800FFF722FF0220FFF71FFF00F015FF154BBE
:10A9E80015494FF4BE425D612846144B0094059307
:10A9F8000123CDE90144CDE903433B4600F096FC31
:10AA08002A7C0646284622F004022A742BF08CFB86
:10AA18002046FFF779FF3A4631462846F9F790FC79
:10AA28000043002400ED00E051A80090901B002492
:10AA3800301C00246021002480440024A02F0590AD
:10AA480038B5064C064DAC4201D3002038BDD4E9D8
:10AA58000112204614342BF01DF9F4E7100C0024E1
:10AA6800240C002430B585B0044BDDE90845029379
:10AA7800CDE900452BF0CCF805B030BD832A039012
:10AA880038B50020054C064DAC4200D338BD2046F1
:10AA98002BF024F90028F9DB1C34F5E7F40B00242B
:10AAA800100C002473B50C46EFF31181102585F3C3
:10AAB8001288BFF36F8FC5685DB125602B68C360CE
:10AAC800836901338361002081F31188BFF36F8F9D
:10AAD80011E052EA030603D16FF00B002560F3E79B
:10AAE800CDE900230246083000F08CFD18B9034B6D
:10AAF8009B685B69236002B070BD00BF60210024C1
:10AB08002DE9F34104460E469DF8200004F108089B
:10AB1800EFF31187102181F31288BFF36F8F256A35
:10AB2800E1688D4246D22568AC4218D0BDB12846AE
:10AB38002BF034F905F118002BF007FCA268314618
:10AB480068693CF07EFD00232846C5F898302BF054
:10AB5800EBFA4046394600F0E9FD002037E0A268EC
:10AB6800D8B13146E0693CF06CFDE369A268134452
:10AB780062699342E36101D12369E361236A102189
:10AB880004F12400013323622BF0BEFC0028E0D13D
:10AB980087F31188BFF36F8F19E0A1692369994280
:10ABA800314604BF6369A361A069801AA0613CF0C3
:10ABB80048FDE3E752EA03010CD00849404689689A
:10ABC8004E613946CDE90023224600F01BFD02B054
:10ABD800BDE8F0816FF02200DAE700BF60210024B1
:10ABE800F7B50446084604F10807EFF3118610216B
:10ABF80081F31288BFF36F8F216A00293AD0A268C7
:10AC0800A1693CF01EFDA369A26825681344626926
:10AC18009342A36104BF2369A361AC42236A03F191
:10AC2800FF33236234D02846002D32D02BF0B6F8FB
:10AC380005F118002BF089FBA2686969E0693CF00E
:10AC480000FDE369A2682846134462699342E36100
:10AC580004BF2369E361236A013323620024C5F832
:10AC680098402BF061FA3846314600F05FFD2046E7
:10AC780003B0F0BD52EA030110D00A49896848615F
:10AC880031463846CDE90023224600F0BBFCEFE709
:10AC9800002086F31188BFF36F8FE9E76FF0220079
:10ACA800F7E700BF602100242DE9F3410446174669
:10ACB8001E46EFF31188102383F31288BFF36F8FBA
:10ACC800C368314A7BB180689168884219D057EAD5
:10ACD800060318D188F31188BFF36F8F6FF00F0048
:10ACE80002B0BDE8F081916891F90E10013321613D
:10ACF800E3609368A36088F31188BFF36F8F002027
:10AD0800EEE72169F2E790F90E3091F90E109942B9
:10AD1800A8BF19468B422DDD2BF0AAF8054622461E
:10AD280041461A48CDE9007600F06CFC0028E6D0D0
:10AD3800EFF31186102383F31288BFF36F8FA06897
:10AD4800D0B1236821699C420AD04BB193F90E30E7
:10AD58009942A8BF19466FF07F039942B8BF1946B8
:10AD68002BF086F840B13146084800F0DFFC6FF060
:10AD78000A00B5E70025D2E7002DF4D186F3118843
:10AD8800BFF36F8FF3E700BF60210024A3280024DE
:10AD9800F8B583680546002B40D0234A9268934251
:10ADA8003FD1C368012B03D9013BC3600020F8BD24
:10ADB800EFF31187102383F31288BFF36F8F0169B4
:10ADC80080682BF055F82C68AC4207D10023C5E900
:10ADD800023387F31188BFF36F8FE7E7002CF5D0B4
:10ADE800002604F11800D4E9003213605A60237C6D
:10ADF800A66023F00203C4E9006623742BF0A5FAC9
:10AE0800AC6094F90E3020462B61C4F898602BF0A2
:10AE18008BF93946054800F089FCC7E76FF0150043
:10AE2800C5E74FF0FF30C2E760210024A3280024C3
:10AE380037B51146EFF31185102282F31288BFF35C
:10AE48006F8F04689CB123680121426823F00303D3
:10AE58009442036008BF436020462BF08FF80446F5
:10AE680085F31188BFF36F8F204603B030BD51EAD8
:10AE78000302F5D000F10802CDE900131046294677
:10AE880000F0C0FB0028EFD1014B9B685C69EBE741
:10AE98006021002470B5EFF31186102383F3128824
:10AEA800BFF36F8F0468A0421BD0D4B1002504F112
:10AEB8001800D4E9003213605A60237CA56023F09F
:10AEC8000203C4E9005523742BF03FFA2046C4F866
:10AED80098502BF029F931460B48BDE8704000F036
:10AEE80025BCD0E90232022110309A4218BF013342
:10AEF80040F8083C2BF008FB0028ECD186F31188B9
:10AF0800BFF36F8F70BD00BFA328002413B5EFF304
:10AF18001181102484F31288BFF36F8F846844B1C1
:10AF2800013C846081F31188BFF36F8F002002B069
:10AF380010BD52EA030406D181F31188BFF36F8F65
:10AF48006FF00F00F3E7CDE900230246014800F057
:10AF580059FBECE7A32800242DE9F8430546EFF355
:10AF68001188102383F31288BFF36F8F00266FF0C8
:10AF78000A0937462C68A54216D0ACB104F118006E
:10AF88000126D4E9003213605A60237CA76023F0BD
:10AF98000203C4E9007723742BF0D7F92046C4F8DC
:10AFA80098902BF0C1F8E5E70023022105F1100085
:10AFB800AB602BF0A9FA30B92EB988F31188BFF32A
:10AFC8006F8FBDE8F88341460248BDE8F84300F0BA
:10AFD800ADBB00BFA32800242DE9FF41044610277C
:10AFE8004E4EEFF3118887F31288BFF36F8FD4F8B2
:10AFF800A450F5B9022104F1BC002AF0E5FF0028AD
:10B0080068D004F1B4050022012128462BF032F95A
:10B018000028F8D100234FF0FF3241464048029300
:10B028004FF0FF33CDE9002304F1AC0200F056FDE8
:10B03800D7E7D4F8A8202B689542C4F8A43008BFF5
:10B04800C4F8A830D4F8BC3043F00203C4F8BC30CC
:10B05800EB6823F0040343F00103EB606B6888F3AB
:10B068001188BFF36F8F28469847EFF3118887F34D
:10B078001288BFF36F8FEB68D80623F0010236D42D
:10B08800EA60EB689A0716D523F002033068EB6094
:10B0980088B10368002170B14268954235D10368D0
:10B0A80069BB72683360824200D17360002340F844
:10B0B800083BFFF7EFFED4F8BC3023F00203C4F8D6
:10B0C800BC3088F31188BFF36F8FDB0589D400F09B
:10B0D800B9FB86E7D4F8BC30D9069BD5C4F8BC00C8
:10B0E80088F31188BFF36F8F04B0BDE8F08123F0B7
:10B0F8001103EB6005F11000FFF7CCFEC1E70B6010
:10B108007368834208BF7160D0E723B11A680146AB
:10B1180018461346BFE71A46F9E700BF8421002402
:10B12800A3280024F8B5C36804460F469A07C3F35A
:10B1380040062DD45B071BD40B680BB983680B60E2
:10B14800E368DD0745BFA368022601263B603D682A
:10B15800002D3CD01F4B9A68D5F8A0309A420AD0EF
:10B16800D5F8BC30D807C3F3800214D46FF01206A8
:10B1780000233B6025E02AF092FFD5F8BC30002878
:10B18800F0D1D907C3F3C002F0D552B15B0708D498
:10B198006FF00F06ECE7002AFAD1C3F3C003002BC7
:10B1A800F6D100232360D5F8A83063B9C5E929444E
:10B1B80028462AF023FFE36843F00403E3603B6872
:10B1C800A3603046F8BD1C60C5F8A840F0E76FF0F2
:10B1D8001506CDE760210024014601482AF04FBF3B
:10B1E800F01C0024F0B50446002089B0C4E9290009
:10B1F80004F1AC000E9DC4E92B0004F1B400C4E9CD
:10B208002D0055B32879002840F2011008BF01200D
:10B21800C4F8BC0000204FF0FF364FF0FF37009411
:10B22800CDE90330CDE901000D4B2046CDE9066795
:10B2380000F0E2F855B1296811B120462AF035FF2F
:10B248006B791BB1A38943F00103A381204600F069
:10B2580079FBC4F8A04009B0F0BD0120D8E700BFD1
:10B26800E1AF009037B501900846EFF31184102143
:10B2780081F31288BFF36F8FC16811F01E0F17D1C9
:10B2880053EA020508D101A9FFF74CFF84F311889E
:10B29800BFF36F8F03B030BD41F00801103040F8A4
:10B2A800041C01998161034900F0F8FC0120EDE7D5
:10B2B8000020EBE71360039001460148FFF7D2BF77
:10B2C800F01C0024F7B50C4616461D460190EFF316
:10B2D8001187102383F31288BFF36F8F08462AF073
:10B2E8007EFE55EA060309D101A92046FFF71AFF99
:10B2F80087F31188BFF36F8F03B0F0BDE368324660
:10B30800064904F1100043F00803E360019BA362BF
:10B318002B4600F0C3FC0120EAE700BF136003904E
:10B3280001460148FFF7CEBFF01C0024073222F087
:10B3380007022DE9F04F7F3285B01F4600F1580310
:10B34800044622F03F020E4604213F2AA2F1400B98
:10B3580006F14008C0E91633129B4FF00000217433
:10B36800A381119BA060A373E073DDE90EA9C4E972
:10B37800060005D880F31188BFF36F8F084602DFF7
:10B38800B51820462946F8F7A7FB0730109B314629
:10B3980020F007002D1AC4F8880020462A46C4E980
:10B3A800208BCDE90193CDF800A03B46F8F798FF34
:10B3B8000023C4F874906365109BC4E91B7AA367E3
:10B3C800EFF31182102383F31288BFF36F8F094BB9
:10B3D800196A1C62E16782F31188BFF36F8F9B685B
:10B3E8000BB1D3F88C302846C4F88C3005B0BDE8D2
:10B3F800F08F00BF60210024F0B5002587B0044617
:10B408000595109D04950F9D03950E9D02950D9D24
:10B4180001950C9DDDE912760095FFF787FFB6F1DF
:10B42800FF3F08BFB7F1FF3F05D056EA070305D134
:10B43800204600F087FA204607B0F0BD3A4633466A
:10B4480004F11800014900F029FCF4E79961039020
:10B458000123037483810023C0E92033C0F88C30B2
:10B46800014B9860704700BF602100240A4A6FF0C2
:10B478000A019368C3F898100849C3F894004B6808
:10B4880043F080534B60002383F31188BFF36F8F21
:10B498009368D3F8980070476021002400ED00E01D
:10B4A80070B590F91020037C002A36DBD90634D118
:10B4B8001B4C63F07F0322460374E16952F8183F7E
:10B4C800934207D1C0E900210860E06111E0994288
:10B4D800F8D01B68002BF5D090F90E5093F90E6048
:10B4E800B542F4D0AE42F2DD5968C0E900310860D7
:10B4F8005860A569954200D005B9E568A3681A7C2B
:10B50800D20604D1DA897F2A01D9AA6932B1AB42BD
:10B5180002D0284600F024FB656170BD6361FCE73A
:10B528006021002438B590F910200146037C002AD8
:10B5380004DA03F07F0303742AF0BCFD0D4D2A469C
:10B54800AB6852F8184F944200D004B9EC688B42AB
:10B5580007D01A7CD20604D1DA897F2A01D9A269D8
:10B568002AB1A34202D0204600F0FAFA23466B61C2
:10B5780038BD00BF60210024B3F1FF3F08BFB2F11E
:10B58800FF3F03D00249183000F088BB704700BF66
:10B598009961039038B5194CA168E0690B6881423C
:10B5A80014BF1A46002249680B605960A368E16914
:10B5B8002AB9134AC3E900210B60E3610CE093F94F
:10B5C8000E0092F90E50A84214D0854212DD51683F
:10B5D800C3E900210B605360A569094B9D4200D067
:10B5E80005B9E568A3689D4202D0284600F0B8FA7C
:10B5F800656138BD9142DCD01268D9E7602100242A
:10B6080078210024F8B50E4B0C4611460D4A98686F
:10B61800DDE906671060EFF31182102282F31288C9
:10B62800BFF36F8F9D6828462AF056FD284632469C
:10B638003B46FFF7A1FF2046BDE8F840FFF716BFDD
:10B64800602100248C210024F8B50446EFF311870B
:10B65800102383F31288BFF36F8F037C49B203F082
:10B668001F02002A0CBF0126002639D103F07F03F0
:10B678002D4D03742AF01EFD037C2A46817363F066
:10B688007F03037452F8183F934227D1E869C4E94D
:10B6980000200460EC610FE09842F8D01B68002B92
:10B6A800F5D093F90EC06145F6D08C45F4DD5968A4
:10B6B800C4E900310C605C60AC69944200D004B904
:10B6C800EC68AB689C4202D0204600F049FA6C61F5
:10B6D80087F31188BFF36F8F3046F8BDE869DEE75E
:10B6E8009B071ED585682AF0E5FC81732B689D426F
:10B6F80009D16B68C4E900531C606C60E8E76A68AC
:10B708009342F6D01B68002BF3D093F90E20914298
:10B71800F5D08A42F3DD5A68C4E9003214605C60EF
:10B72800D6E78173D4E700BF6021002449B9EFF35D
:10B73800058030B9054B5A699B689A4201D0FFF7DA
:10B7480095BE81F31188BFF36F8F70476021002485
:10B75800034648B9EFF3058232B9064A516992683F
:10B76800914201D0FFF782BE83F31188BFF36F8F38
:10B77800704700BF60210024EFF31181102383F389
:10B788001288BFF36F8F054B9A68D37B013BD37345
:10B7980081F31188BFF36F8F704700BF60210024C9
:10B7A80070B5EFF31186102383F31288BFF36F8F00
:10B7B800144DAB68DA7B0132DA732A4652F8184F17
:10B7C800944200D004B9EC681A7CD20604D1DA8914
:10B7D8007F2A01D9A2692AB1A34202D0204600F0EB
:10B7E800BFF923466B6186F31188BFF36F8FEFF3C0
:10B7F8001180102383F31288BFF36F8FBDE8704068
:10B80800FFF7A6BF60210024024B03F11802C3E929
:10B81800062270476021002408B5FFF715FF70B1B4
:10B82800074B9B68DB7B53B9EFF31180102383F33D
:10B838001288BFF36F8FBDE80840FFF789BF08BDC6
:10B848006021002470B5EFF31186102383F312886A
:10B85800BFF36F8F1B4CA168E0690B68814214BF6E
:10B868001A46002249680B605960A368E1692AB941
:10B87800154AC3E900210B60E3610CE093F90E005F
:10B8880092F90E50A84218D0854216DD5168C3E9D6
:10B8980000210B605360A5690B4B9D4200D005B990
:10B8A800E568A3689D4202D0284600F059F9304661
:10B8B8006561BDE87040FFF7D9BD8A42D8D01268EB
:10B8C800D5E700BF6021002478210024F8B550EAAC
:10B8D800010306460C4603D1FFF7B4FF0020F8BD6C
:10B8E800EFF31187102383F31288BFF36F8F124D84
:10B8F800124BA8681860FFF715FEA8682346324661
:10B908000F49183000F0CAF9AA6804463846137C73
:10B9180043F004031374FFF7A9FDAB68D3E90A23C6
:10B92800B3F1004F08BF002AD8D12AF036FD201AFB
:10B9380020EAE070D3E700BF602100248C210024B6
:10B948009961039038B50446EFF31185102383F30A
:10B958001288BFF36F8F037C5B070FD518302AF06E
:10B96800F4FC237C204623F004032374FFF798FD9E
:10B9780029460548BDE83840FFF7D8BE85F3118849
:10B98800BFF36F8F38BD00BFA3280024014B986810
:10B99800704700BF602100242DE9F84304468789D9
:10B9A800EFF31185102383F31288BFF36F8F037CA5
:10B9B800190705D585F31188BFF36F8FBDE8F883A4
:10B9C800D90943F0080260D10274A36813B1204674
:10B9D8002AF078FB04F1180004F158082AF0B5FCA5
:10B9E800A66DB04511D04FF0000976B130462AF067
:10B9F80069FB06F118002AF0A8FC3046C6F89890B2
:10BA0800FFF74EFDA66DB045EFD1DFF8C480D8F83A
:10BA180008309C4241D1EFF30589B9F1000918BFFC
:10BA28004FF00109D8F818602A4A964200D00EB99A
:10BA3800D8F80C60B34202D0304600F091F82046A6
:10BA4800C8F8146027F029FE204600F0DBF8B9F1A9
:10BA5800000F02D02048FFF7FBFCD8F808309C42C2
:10BA680031D1EFF3058373BBA289D20718D42846D6
:10BA7800FFF7FCFCFB07A1D5002383F31188BFF374
:10BA88006F8F0423184602DF98E703F07F0343F023
:10BA9800080303742AF00EFB97E74FF00009C1E78B
:10BAA80085F31188BFF36F8F83F31188BFF36F8F0E
:10BAB8000423184602DFEFF31180102383F3128862
:10BAC800BFF36F8FD4E785F31188BFF36F8FD1E78A
:10BAD8006021002478210024301C0024D3B5DDE93E
:10BAE8000667089CCDE90067FFF78CFD1CB1034B86
:10BAF8009B685B69236002B0D0BD00BF6021002451
:10BB0800027C034612F01F0210D10A4988420DD068
:10BB18000949086868B1D9897F2909D893F90E209D
:10BB2800064B1B689A42B8BF002070470020704738
:10BB380010467047F01A0024B8030024902100240E
:10BB4800044B0122C01A044BC0105843034B1A542B
:10BB5800704700BFD01C0024ABAAAAAAA3280024BF
:10BB68000D4B70B51E7CFFF7CBFF0C4D044606EB62
:10BB7800460305EBC30528462AF0E7FB084B0022DD
:10BB88009A553CB1621E28460649D317BDE8704055
:10BB980000F084B870BD00BF60210024D01C0024D0
:10BBA800A328002449BB009038B5EFF31185102372
:10BBB80083F31288BFF36F8F0F4B104A9C6810688D
:10BBC800A04206D1FFF7CCFF85F31188BFF36F8F32
:10BBD80038BD00211B7C1160094AD35C002BF3D0CF
:10BBE8002046FFF78DFF0028EED0237CDB0601D12D
:10BBF800FFF7D0FC2046E5E7602100248C210024D3
:10BC0800A3280024EFF31181102383F31288BFF3D4
:10BC18006F8F0A4A136A834207D1DB6F136281F37D
:10BC28001188BFF36F8F70471346002BF7D0DA6F78
:10BC38008242F9D1C26FDA67F1E700BF60210024C0
:10BC4800024B1868984208BF00207047BC030024C4
:10BC5800034B1B680BB9FDF7AFBA0020704700BF54
:10BC68009421002430B570B10B4B5B6898420AD020
:10BC7800036843B1D3E90421D0E90445121941EB23
:10BC88000501C3E90421D0E9003213605A6000239A
:10BC9800C0E9003330BD00BFBC030024B3F1FF3F4F
:10BCA80008BFB2F1FF3F2DE9F84F04469946154603
:10BCB8001F467AD08160EFF31188102383F312882E
:10BCC800BFF36F8FB9F1000FDFF8E4A020DBFFF7B7
:10BCD800BFFF0135064649F100092D18DAE90027AA
:10BCE80049EBE0734FF00109C4E90453AD1843EB85
:10BCF8000707FFF7A5FFDFF8BCE00346DEF804A05E
:10BD0800EBB9C4E900EACAF80040CEF8044028E0DC
:10BD1800DAE900126FF001035B1A4FF0FF3161EBB3
:10BD280002025B1B62EB0902012B4FF0000972F162
:10BD38000001BCBF01230022C0E90432D9E7D3E9DE
:10BD4800041CD4E904208A4270EB0C0B24DA891A0B
:10BD58005A686CEB0000C3E90410C4E900321460AF
:10BD68005C60FFF76DFF84420ED1134B1B685BB913
:10BD7800B9F1000F02D1FFF76BFF064630462AF0F3
:10BD8800CDFA0021FDF79AF988F31188BFF36F8F78
:10BD980028463946BDE8F88F521A60EB0C009A45E0
:10BDA800C4E90420ADD01B68AAE700252F46EFE7B9
:10BDB800E81C0024BC030024942100242DE9F0474A
:10BDC800EFF31185102383F31288BFF36F8FDFF829
:10BDD800A4900026DFF8A0800027C9F80000FFF72C
:10BDE8002FFFD9F80030D8E900ECD91750B1D0E9C5
:10BDF8000442A34271EB020A1CDAE41A62EB010264
:10BE0800C0E9044213EB0E034FF000044CEB0101B0
:10BE18002046C9F80040C8E900312AF07FFA2146D7
:10BE2800FDF74CF985F31188BFF36F8FBDE8F04734
:10BE3800FFF7BABE14EB0E024CEBE473C0E90467DB
:10BE4800C8E90023FFF70EFF85F31188BFF36F8F52
:10BE580083689847EFF31185102383F31288BFF3A3
:10BE68006F8FD9F800301B1BC9F80030FFF7E8FEC8
:10BE7800B7E700BF94210024E81C002410B5EFF3B5
:10BE88001184102383F31288BFF36F8FFFF7E0FE4E
:10BE9800054A0346D2E90001181841EBE37184F31F
:10BEA8001188BFF36F8F10BDE81C0024F8B5064653
:10BEB800EFF31187102383F31288BFF36F8F0268A3
:10BEC80022B187F31188BFF36F8FF8BDD0E90A5408
:10BED800691C44F10003022973F1000334D3013DC6
:10BEE80044F1FF34002CBCBF15462C462AF059FA01
:10BEF800013041F10001401944EB0101012871F1C1
:10BF080000014ADB2AF04DFA01306FF0020341F1DB
:10BF18000001401944EB010183426FF000438B415B
:10BF280040DB2AF03EFA01306FF001024FF0FF3398
:10BF380041F10001401944EB0104121A63EB0403B8
:10BF48001A493046FFF7AAFE336B01333363336A6D
:10BF58006BB187F31188BFF36F8F336A3046984708
:10BF6800EFF31187102383F31288BFF36F8F3346E3
:10BF780053F8184F9C42A4D0002CA2D020462AF097
:10BF8800E2F80023C4F8983087F31188BFF36F8F65
:10BF98002046BDE8F8402AF0C7B86FF001024FF01C
:10BFA800FF33CDE700224FF00043C9E7B5BE00904C
:10BFB8002DE9F04105461C4690461F46EFF31186D1
:10BFC800102383F31288BFF36F8FB4F1FF3F08BFCC
:10BFD800B2F1FF3F05D186F31188BFF36F8FBDE83B
:10BFE800F081002C09DB012A74F10003BCBF012297
:10BFF800002412F1FF3844F1FF3728462AF0A5F94A
:10C00800002342462B633B46DDE90601C5E90A01E8
:10C0180028460249FFF742FEDDE700BFB5BE0090A3
:10C0280038B50346EFF31185102282F31288BFF367
:10C038006F8FC160012181600068834206D185F35A
:10C048001188BFF36F8F0024204638BDD0E9003235
:10C0580013605A600023C0E900332AF012FA294617
:10C0680004460248FFF762FBEEE700BFA42800245D
:10C07800F8B507460C4616462AF011F808B1002014
:10C08800F8BD0E4B9B68D3F88C50002DF7D0221DBD
:10C09800F5D2EFF31184102383F31288BFF36F8F67
:10C0A80047F004012846B04784F31188BFF36F8F27
:10C0B8000028E4D040F8045BE2E700BF60210024D8
:10C0C8000146024A0020FFF7D3BF00BF7D2A039034
:10C0D800014826F039BE00BF75430590074B07B5E8
:10C0E8004FF48062009306494FF0FF330548FFF78D
:10C0F80079F8002003B05DF804FB00BF00870490C6
:10C10800C0A30024F01C00240428F0B504468BB01A
:10C118002BD0344D286818B112F0BAFF00232B60D9
:10C128001CB3314B9C4220D001AB0026214602A80B
:10C1380002932E4B019603932EF0FAFA019831469A
:10C14800013012F085FF0246286070B106AF0199F0
:10C15800384630F055FD264B214604A80593049730
:10C168002EF0E6FA2A68019BD654224D02F04CFBC9
:10C1780030F0CAFE2AF0FFFA01F076FC1E4B0022CE
:10C18800D5F8F0401A7084B1204611F073FF30B32F
:10C19800A06804F04FFBD5F8F040002CF4D1D5F896
:10C1A800F0301C46DB68002BFBD1C5F8EC400025BD
:10C1B800124C02F05FF804F0F5FB12F04DF820681D
:10C1C80012F066FF25600E4C206812F061FF2560B2
:10C1D8002AF0F0F90BB0BDE8F0402AF06ABAE4683A
:10C1E800DBE700BFF0220024842300246D65039060
:10C1F80081CB03900C230024A4280024D4210024FC
:10C20800D021002470B5164B0022044600EB8105AE
:10C218009A60C3E900222646043430682CF0FEF9FF
:10C22800022818D130680F4C206098B10E482AF0C7
:10C2380083FC20682AF0E6F90C4802F017F901F0AF
:10C2480059FC074920682AF0D8F90023236001F037
:10C2580051FC012070BDA542DDD10020E3E700BFFD
:10C268009C210024CC21002404450590AB9705901F
:10C2780010B5044608482AF0C5F901F095FD40B10B
:10C28800064802F0F3F834B10548BDE8104002F062
:10C29800EDB80448F5E710BD044505909A9505905A
:10C2A80078900590C795059073B506462AF001FA6F
:10C2B8000CF0C6FE12F0CAFD054612F0D3FD044686
:10C2C8000CF0C6FE641B0025A4F58060244C0CF01D
:10C2D800C5FE01F0C9FB00F053FC6B464FF4006249
:10C2E8002049304600952AF041F91F4B0146186055
:10C2F800009B194404F0EAFF4FF4005201AB1B49BC
:10C30800304601952AF032F9194B01461860019B15
:10C31800194411F081FE06F0CDFB2946D4F8E80057
:10C328000DF01EFE1621D4F8E8002EF036FE662128
:10C33800D4F8E8002EF031FE40F6B651D4F8E80003
:10C348002EF02BFE294604F1D8000DF009FE09480D
:10C3580003F0AEFE084B01221A7002B070BD00BF98
:10C368000C230024AC430590D0210024C34305903E
:10C37800D421002473300590A428002409282DE92D
:10C38800F0470446A4B000F08B8001F087FB00283A
:10C398007DD0002C7BD1444BD3F8F030002B76D0E5
:10C3A80002AD2046DFF80481FFF77EFF01F00CFCA8
:10C3B8004FF400712846DFF8F8A030F006FCC8F802
:10C3C800005001F073FB0121064600F180072AF0B6
:10C3D80090F9384B384A06AD384939482EF003FBF6
:10C3E800DFF8DC9006A800F035FB364934482EF01B
:10C3F8001FFB013415F8012B514648462EF018FB57
:10C40800202CF6D130492E482EF0EDFA30F07DFD83
:10C4180002212E48FFF7F6FE0023C8F8003001F08D
:10C42800D9FB01232A4A0EA9384631F00AFDA0B9E2
:10C4380002982CF093F9039A0446014601AB0132A5
:10C448000EA831F024FE40B9039A019B9A4204D108
:10C45800214604983BF025F9A0B14FF47A702AF0F0
:10C468009CFB0A231A4A0EA9384631F0EAFC01ABB4
:10C478000EA8DDE9032131F0BCFE0EA832F021F848
:10C4880001F0F2FA002130462AF033F902E02046A2
:10C49800FFF70AFF0F4C6068FFF736FE0023636062
:10C4A80024B0BDE8F08700BF0C23002498210024A5
:10C4B80099970590DD430590EE4305904544059016
:10C4C800C8CC0490688F0590108205903C87049032
:10C4D800554405909C2100242DE9F04F89B007466A
:10C4E8002AF005FB804640B1B0482AF025FB3846C3
:10C4F800FFF7BEFE384601F07DF9DFF8B492CDF8BB
:10C508000880002F40D0D9F80030B3F5007F40F004
:10C51800D580002520262C464FF002094FF4401BF9
:10C528002AF037FB4FF4C873039003FB09F3049315
:10C5380003F59C5308330093002C40F07481A24605
:10C548004FF0010901F064FE01F034FC054601904A
:10C55800002800F0BB8046F0100601F0FDFB954C6A
:10C56800206828B103781E4002D112F091FD2660A0
:10C57800BAF1000F04D0002001F04AFB01F042FBA1
:10C58800284609B0BDE8F08F01F06EFA01F030FCE2
:10C598000546002840F08480864EFFF785FE336804
:10C5A800002B5DD01A7822F020021A7033689A683E
:10C5B8001C78127892B1586808B103F079FD336895
:10C5C800012107A89B680793FFF71CFE98B93368F9
:10C5D80098682AF0B1FA784801F048FF04217748B2
:10C5E800FFF710FE38B908217548FFF70BFE10B1A8
:10C5F800744801F03BFFD9F800301B0532D501F033
:10C6080009F801282ED1704801F030FF4FF0000AD8
:10C618006E4BD9F8040083F800A0FFF775FD326867
:10C62800C9F804A02AB11378980644BF43F0200340
:10C638001370D9F80030190516D500F0EBFF441E29
:10C648004FF0300618BF0124D9F80030DA051AD5A2
:10C65800B3F5007F4FF001043FF45EAFA1462AE036
:10C668003C46BBE75A48CFE71BB904F0010424262F
:10C67800EAE714F002044FF028061CBF83F4806335
:10C68800C3F38024E0E7B3F5007F254615BF4FF0DC
:10C6980001094FF002094FF4405B4FF4401B3FE79C
:10C6A800D9F80030B3F5007F3FF433AF3D463C4640
:10C6B80020264FF001094FF4405B31E70025202682
:10C6C8004FF00309DFF80CB12C4629E72AF00FFADE
:10C6D800059080B12AF028FA68B101F089FB054677
:10C6E80048B92AF011FA04287FF439AF032000F082
:10C6F80097FF059D33E7CCB92AF0F9F90546A8B1AB
:10C7080001F076FB90B9B8F1000F02D13846FFF777
:10C71800AFFD029B13B9384601F06CF823482C464C
:10C728002AF00AFA2C4801F0A1FE02952AF0DFF956
:10C738000546002814BF45462C46B9F1000F05D020
:10C7480001F056FB10B902F0C1FD81462AF021FA2A
:10C75800039B049A8046C31A9A423FD94FF4C87182
:10C76800B3FBF1F201FB1238B8F1630F11D9BAF13A
:10C77800000F04D0002001F04BFA01F043FAC8F58D
:10C78800C870B9F1000F47D112F090FB12F0D8FB36
:10C798002CE0BAF1000F04D101F054FA584601F028
:10C7A80037FA0123C8F164000193EAE77F45059051
:10C7B8009C210024EC220024B19705902C8704903A
:10C7C8000C870490998E05900D8E0590A42800245E
:10C7D800268E059000303000F5900590009A9A4218
:10C7E80008D22AF0D6F9CDF804A00390DDF804A009
:10C7F800A846A7E6BAF1000F04D0002001F008FA15
:10C8080001F000FA009B039A1344A3EB0800B9F166
:10C81800000F05D00028E9D0484528BF4846B3E7AF
:10C828000028E3D0B0E74FF0000A98E607B5114AB0
:10C83800114B1068596820B103B05DF804EB2AF079
:10C848007BB91A6892050ED59A68002A0BDD51B19A
:10C8580009680C330948C988009109492EF0C3F8C2
:10C8680003B05DF804FB074803B05DF804EB01F082
:10C87800FDBD00BFCC2100249C210024C8CC04901D
:10C8880063440590339405902DE9F74312F0C2FAFA
:10C8980000F01EFF29F08EFE12F074FB29F068FFED
:10C8A80001F04EFC524829F0ADFE00F00BFF18B91C
:10C8B80000F014FF00F00CFF29F05EFF01F094F97E
:10C8C80000F000FFB0FA80F00021400901F014F8F0
:10C8D80010B9082000F0FCFE30F016FB29F04BFFE1
:10C8E80000F0D0FE02F0DCF8414829F08BFE002071
:10C8F80000F096FE00F0E6FE08B901F033FA0120D8
:10C90800012501F0C5F8002001F0BCF84FF480744F
:10C9180000F0D8FE374EFFF731FD374F29F0CAFE39
:10C92800012001F0DBF8DFF8D480284614F4106900
:10C9380055D015B9384601F099FD3578002D3CD110
:10C9480000F0C0FEFFF7C8FD0028EFD100F0BAFEE6
:10C95800044601F089F82046FFF7A6FC012001F003
:10C9680013FA00F0AFFE28B9254B012101A8019365
:10C97800FFF748FC01F066F9404601F049F901F07B
:10C9880041F93378012B1AD101F01EF900F0BEFCF1
:10C99800044601F01FF90420FFF7B6FB01F052F935
:10C9A800002001F035F901F02DF9012001F0F4F92A
:10C9B800032000F035FE0020B8E70025C6E7114B3C
:10C9C800DFF84490C9F8003001F094F800F02EFD2B
:10C9D80000230446C9F8003001F08CF8DBE7002C8E
:10C9E800B2D02CF0A7FA484603B0BDE8F08300BFE8
:10C9F80004450590A528002457860590303030005E
:10CA08006C44059074440590CC21002408B511F0BD
:10CA180041FB00F035FB0421064830F0F4F92AF018
:10CA280006F901F05BFC01F075FFBDE8084011F064
:10CA380045BB00BFFC230024014B1878704700BF9A
:10CA4800A42800240048704700389C1C0048704700
:10CA58003333534038B505462021FBF71BFF041E2E
:10CA680011DA21460024094826F06EF921462022D1
:10CA7800074826F069F9C4F1200228190021BDE809
:10CA880038403AF006BE1F2CF0DD38BD0D45059044
:10CA9800274505900428034607B506D801460F48E0
:10CAA80003B05DF804EB01F073BC06210C4A68463C
:10CAB80023F0BCFB011E0DDD052901DD26F015FE66
:10CAC80001F108034422013168466B4403F8082C3D
:10CAD80001F05EFC03B05DF804FB00BF4E45059015
:10CAE80053450590F8B5244DAB7DDB0732D52E684C
:10CAF800706801282ED9B168431ECA5C0A2A29D158
:10CB08004A1E002B01DC1A4608E0D45C0A2CFAD035
:10CB1800013BF6E78C5C202C02D101329042F9D817
:10CB2800002B0CDD541CA04209D15C1E0C44A14210
:10CB380005D014F8017D0A2F0CD0202FF7D001441E
:10CB4800D21A0E4F11F8023C94083A2B08BF013450
:10CB5800013C00D2F8BD04223946304630F00CF8CA
:10CB68000421384601F014FC2B6904332B61AB7D9A
:10CB780043F00203AB75EBE7D8210024259A059012
:10CB88002022002101483AF084BD00BFC4230024BC
:10CB980038B500220B4C05460846A2606B686275E2
:10CBA8004FF0FF3263602560A161C4E9032329F0D7
:10CBB80029FD6B680BB90123A375BDE83840FFF761
:10CBC80091BF00BFD8210024F8B503780446DBB133
:10CBD8000E4FD7F8B80018B12146F4F799FD98B16F
:10CBE8002046F4F7A7FD461C30462BF0BAFD054653
:10CBF80050B1324621463AF024FD05491C22081D51
:10CC08003AF02DFDC7F8B850F8BD00BF0C2300243A
:10CC1800C42300242DE9F347AB4C06462368D3E927
:10CC280001102BF0C8FEA5680746002D40F038819A
:10CC3800731E042B1AD8D4E900325B689A4278D064
:10CC4800012E15D1236865689868D4F8108000EB28
:10CC580008012844A8EB0508002529F0B6FC06467B
:10CC6800A845A56040F3BA80A946A8E00D2E13DCBC
:10CC7800022E40F3B380F31E0A2B00F28F80DFE808
:10CC880013F058008D00CD018D008D005F008D00E0
:10CC98008D008D003D004D001B2E4ED07F2E4FD0B5
:10CCA800A37D99077FD41F2E40F3988020682169BF
:10CCB80083685A5C06F0C003802B16BFF2B2237D4E
:10CCC800002302F1400508BF0133EDB208BFDBB213
:10CCD800372D194423759BBFD208E525002502F09E
:10CCE800060298BF1541324698BF05F0030530F09B
:10CCF8002DF8237DAB4271D1013596E0734829F0B8
:10CD080081FCA06929F07EFC22686368216990682B
:10CD1800C91A184401F03CFB002586E06C4800263F
:10CD280029F070FC20682FF0A0FF63681844FFF713
:10CD38004BFF304602B0BDE8F0870123A3604DE009
:10CD4800226961688A4249D92068561A0023D0F8B6
:10CD580008E0B34203EB010C17D1032BCCBF042628
:10CD68000126961B33461EF803C01946013B0CF0FA
:10CD7800C00CBCF1800FF6D0A2EB0108761A42462F
:10CD88002FF0F1FF4FF0010919E01EF80CC0BCF1BB
:10CD9800200F01D10133DCE70126E2E7A37D9A07E2
:10CDA80023D5092E18D0202E7FF47DAF00264FF012
:10CDB800030803212068B146A6752FF0CDFFA8EB24
:10CDC8000600FFF767FE2369A3EB08032361B9F1A7
:10CDD800000F00F0298128E00023A375A37D4FF000
:10CDE800FF3623F00203A375A3E7092E7FF45BAF98
:10CDF80022682169D2E90123002A40D00B4413F8A4
:10CE0800010C04F093FA002839D0324B0425019321
:10CE18000026019B21695A1C206831440136019281
:10CE28001A782FF08DFFB542F3D12368D3E90110AA
:10CE38002BF0C1FDB84203D20321274801F0A8FA1C
:10CE480023682769D3F80880D3F80490781908EB89
:10CE58000901404429F0B9FBA9EB0701064608EB94
:10CE6800070001F095FA236822695B689B1A5B1B2F
:10CE7800981BFFF70FFE23692B442361AEE7236855
:10CE880060689D6801AB2169144A091A284410F0AA
:10CE98007BFC05460028A1D0431C3FF432AFB7E71E
:10CEA800013D032D00F2E880DFE815F004001A00C8
:10CEB800A000E1004F2E04D05B2E40F0DD8002235D
:10CEC8003CE704233AE700BFD821002458450590E1
:10CED8007F450590259A059061450590C8CC04903A
:10CEE800A6F13003092B03D803236675A36075E701
:10CEF8000023412EA3602ED1E368062B3FF76EAFC7
:10CF080003F1010A5D4D2D3305EB8305AB68002B5A
:10CF18003FF464AFD4F80080D4F80490D8F808003F
:10CF280021690144484429F050FBC8F8049006469A
:10CF3800A9684046C4F80CA02FF0F5FE6368226982
:10CF4800A2EB03082268B8F1000F5568A5EB0305AA
:10CF58007FF76BAF16E7423E062E3FF63FAF01A3C1
:10CF680053F826F089CF0090CFCF0090DFCF009004
:10CF7800E5CD009025D00090E5CD00904DCC0090F7
:10CF8800E568002DFFF62AAFD4F80080013DD4F8FB
:10CF98000490D8F8080021690144484429F015FB99
:10CFA800D8F8041006464046A1EB0901E5602FF0C9
:10CFB800D3FEE268002AC1DB304B206803EB820312
:10CFC800D3F8B810B8E7236822695B689A42BFF4BF
:10CFD80005AF01252BE0226963689A427FF6FEAE11
:10CFE80000254FF00108A9462E46E8E67E2E43D1DB
:10CFF800637D312B3FF426AE333B052B3CD801A291
:10D0080052F823F047D0009025D0009081D00090AE
:10D0180081D000904DCC009025D0009023685D68A9
:10D028002369ED1A0023A360002D7FF7D7AE23688C
:10D03800294698682369184401F0AAF91BE7206873
:10D0480021694368994217D285685B1A01220D4409
:10D0580015F8016F06F0C006802E01D19A4204D15E
:10D068002FF081FE0023A36056E60132F0E7462E3A
:10D07800D4D0482E3FF4E6AD00235FE60C2300240D
:10D088002DE9F04F0B4B8BB019686846CDF820C0DE
:10D09800091ACDF824D08908CDE90045CDE9026701
:10D0A800CDE90489CDE906AB2FF0ADFE0BB0BDE8A4
:10D0B800F08F00BF0C23002470B5067804461EB11B
:10D0C8004FF0FF35284670BD29F0B2FDC31E054656
:10D0D800012B0CD801210C48217001F059F9032DBE
:10D0E800EED10A48836E60309E6010F0E1F9A388A3
:10D0F800013B9BB2A380002BE4D10121044801F03D
:10D1080047F96388A380DDE7654505900C23002473
:10D11800834505902DE9F04391B017461D4600233D
:10D12800044603A80493884607F0010610F0ACF9FA
:10D13800034600285BD1F90641D5DC20D4E901215A
:10D148002DF08AFA0446B8F1010FD4F8009007D1FF
:10D158004FEA091140F20A3041F0060105F012FDCC
:10D168002146424601A80DF037FDC7F38002494623
:10D1780001A808F027FFB8F1010F044601D1FFF715
:10D1880045FC380602D4032000F0FCF914B120460F
:10D198002BF008FF4FF0FF3000F0F4F9012004F005
:10D1A8007BF809F0ADFEEEB9CDB900241EB101211E
:10D1B800474801F0EDF8204611B0BDE8F0837A0643
:10D1C80005D5DC2094E80E002DF0FEF9BAE7BB0681
:10D1D800B9D520462BF070FA2DF04CFAB2E70023AF
:10D1E8002B60E2E701213A4801F0D2F8DCE74FF082
:10D1F800FF3000F0C7F9022004F04EF8790602D596
:10D20800A368206898471EB10121314801F0C0F891
:10D21800049C20460AF056FA2E4905F0E5F9002844
:10D2280041D004982DF07BFC0E283AD0C20705D4D3
:10D2380083072BD10268284B9A4227D12BF0B5FCE3
:10D2480040F48074002DB1D0049F4FF0FF332C6060
:10D2580038466F60AB602DF04DFC0028A6D001AABF
:10D26800694638462DF075FC019B002B9ED05A6804
:10D27800AA60002285F82C2018682BF03DFA20229D
:10D28800014605F10C003AF03BFA8FE7014600220F
:10D2980012480AF033FA124910482DF021FB0120F8
:10D2A800CEE70020CCE70F4B9C420DD004990B48E9
:10D2B8002DF03EFA049B0C49186805F095F908B161
:10D2C8008224BFE70124BDE74FF40064BAE700BF3A
:10D2D8006545059098D10490A4CB0490C8CC0490DF
:10D2E800108205908423002474D1049008B5037833
:10D2F8004BB901210170044801F04AF829F098FC63
:10D3080003380128FAD808BD654505902DE9F04392
:10D318008BB0DFF8F48000263C4F202106A82FF0C0
:10D3280054FC404629F06EF93846079629F06AF908
:10D3380029F07EFC0128044635D107990229F0D14D
:10D34800089B1A78052AECD193F80190B9F1410F9E
:10D3580006D02F4801F01CF800232C480793E5E776
:10D3680080252C4801F014F803216846ADF80050D8
:10D378008DF8024001F00CF801AA0023214603A809
:10D388000392254A8DF804300492244AADF80650D9
:10D3980005924A46ADF80850FFF7BCFEC305DBD539
:10D3A8000BB0BDE8F083022809D11D4829F02AF9FD
:10D3B80006A82FF02CFC00201A4B1870F0E7032861
:10D3C80002D100230793B3E7042804D0C1B206A80A
:10D3D8002FF05AFCACE7144829F014F9079B43B91D
:10D3E8000F4829F00FF906A82FF011FC4FF48070B0
:10D3F800D6E700231122012106A8FFF78BFE10F4BF
:10D40800106F91D0CCE700BF674505900A80059062
:10D41800C07E049082450590C1D00090F5D200905E
:10D428007F450590A5280024854505902DE9F04104
:10D4380092B04B4EDFF82C81202101A82FF0C5FBBC
:10D448003046494F29F0DEF8484829F0DBF83046E5
:10D4580029F0D8F8BA8A002302B1BB8205A8029342
:10D46800069310F011F8044690B9414901A829F033
:10D47800BAF8012805462CD1394829F0C3F801A883
:10D488002FF0C5FB3B4B20461D7012B0BDE8F08164
:10D49800022003F001FF304629F0B4F80699364817
:10D4A8002DF046F9029B002BD4D001A82FF0DDFB0C
:10D4B80010F0A6F858B10A2101A82FF0E5FB414663
:10D4C80001A829F090F803280BD00428EDD10021F9
:10D4D8002CE0022803D1224829F094F8B0E7032869
:10D4E80001D1304619E0042808D11D4829F08AF8EE
:10D4F80001A82FF08CFB4FF48070C6E70528D1D126
:10D508001E4829F07FF802941D4C29F091FBC1B206
:10D5180003298DF8031003D1114829F073F899E70E
:10D5280004290CD10E4829F06DF801210023162298
:10D5380001A8FFF7EFFD10F4106F8BD0A5E701A845
:10D548002FF0A2FB9DF803300D2B03D1204629F0C4
:10D5580059F8DAE701210DF1030000F019FFD4E7CB
:10D568007F450590C44505900C230024EE430590A3
:10D5780088450590A5280024C8CC04908D450590C1
:10D58800BD450590014B1860704700BFC4030024D7
:10D59800024B986A003818BF012070470C230024FA
:10D5A8002DE9F04106460D4600270DB9BDE8F0818A
:10D5B80033780A2B16D1AFB9012401210F4800F0A6
:10D5C800E7FE06EB040843461FB998F800200A2A2C
:10D5D80001D0A54208D1304621462D1B464600F011
:10D5E800D7FEE2E70024ECE71F7808F101080134D0
:10D5F800A7F10D035F425F41E5E700BFC94505900C
:10D60800024B034819782CF0CEBE00BFA628002490
:10D61800D4AD0490014B1878704700BFA6280024A9
:10D62800014B1870704700BFA628002410B5064C9F
:10D6380020680E2806D1054B80220549054800F0D0
:10D64800B9FF206010BD00BFC8030024A72800242C
:10D65800D47B0490B01D002410B5064C20680E2819
:10D6680006D1054B80220549054800F0A3FF20603C
:10D6780010BD00BFCC03002427290024F07B0490B0
:10D68800001E002470B501F085F9044698B10A4BD4
:10D6980003600A48FDF718F8054660B128F0A5FAB6
:10D6A80048B1074B29462046002223600123BDE8E4
:10D6B800704002F0C7BF70BD08D90490D73C0590F0
:10D6C80050AE0490014B1878704700BFA72900247A
:10D6D800014B1870704700BFA72900242DE9F041BD
:10D6E8002FF015FC044620F47F00284B284E20F428
:10D6F8007F4098420AD114F47F4FC4F3072505D020
:10D708002FF004FC35702846BDE8F0810023337003
:10D7180028F059FF28B1062833D85423C340DB0723
:10D728002FD51C482FF0F2FBDFF86C8000F08AFA46
:10D7380029F020FA064600200F460146FA22002367
:10D74800F3F7CCFF7D2A73F1000334BF4046002075
:10D7580000F05EFA29F069FA054648B929F00AFA94
:10D76800801B61EB0701B0F57A7F71F10003E5D307
:10D77800002000F04DFA00F045FA25B920462FF0B8
:10D78800C5FB0025BFE71125BDE700BFAF0000AD11
:10D79800A7290024AF1100AD00303000024B43EA46
:10D7A80000202FF0B3BB00BFAF0000AD0D4D044605
:10D7B80008B52B78012B0FD901280DD90A4825F077
:10D7C800C3FA2146094825F0BFFA2978084825F008
:10D7D800BBFA25F06CFFFCE72046FFF7DFFF2FF0D0
:10D7E8008FFB00BFA7290024CB450590E145059094
:10D7F800ED45059010B50446002838D01C4800F0C7
:10D8080035FE631E112B12D8DFE803F02D1111111C
:10D818001111112B1129111127212523091F154831
:10D8280000F024FE1448BDE8104000F01FBE023C82
:10D83800124800F01BFEE4B20A2C16D8104B53F81D
:10D84800240000F013FE0F48EAE70F48E8E70F4806
:10D85800E6E70F48E4E70F48E2E70F48E0E70F483C
:10D86800DEE70F48DCE70F48DAE70F48E9E710BDC5
:10D87800B88D0590408E0590CC8D0590A9940590A3
:10D88800B8A50490DD8D05900593059065950590E4
:10D89800388F05904E8F0590399005901C90059013
:10D8A8000895059016910590F58E059010B5064CD3
:10D8B80023783BB1054B4FF47A721A6000F008FAEE
:10D8C8000023237010BD00BFA8290024D003002422
:10D8D800074B1A683AB11A68012A05D105490A7036
:10D8E8004FF47A721A6070471A68013AFAE700BF73
:10D8F800D0030024A82900242DE9F0414D4E4FF013
:10D908000008ADF5287D07464B4C30460D46A6F875
:10D91800048000F0EBF906F18000C4F8048030F0D0
:10D928008CFA0D2806D13FB935B900200DF5287DB0
:10D93800BDE8F081002D79D04FF400730022072153
:10D948003E48009328AB12F0C7FC0028EDD100F048
:10D95800BFF93B49394812F0D7FB0028E5D13949CE
:10D96800364831F05FF9384B03AA03F138071868D5
:10D97800083353F8041C1546BB4203C52A46F6D1A2
:10D988001B8812A9314A2B8039232C4802930A2379
:10D9980030F057FA02AB029A03A912A830F029FC1A
:10D9A80012A830F08EFD0A23294A12A9234830F024
:10D9B80048FA12A830F085FD264B03AA03F1100798
:10D9C8001868083353F8041C1546BB4203C52A4699
:10D9D800F6D1186899889B792860AB711623A980BD
:10D9E80012A91D4A02930A23144830F02AFA02ABFE
:10D9F80003A91A6812A830F0FCFB12A830F061FDE8
:10DA080016490E4831F00EF900288ED100F060F961
:10DA1800134B012523600023E360124BC4E9015630
:10DA2800C3E93B4429F0C0FF28467FE70028EFD030
:10DA38007BE700BF800D0024F4210024000E0024A1
:10DA4800824D059004460590394605900846059094
:10DA58001C460590734605902B4605903446059064
:10DA6800733005900C23002408B54FF47A72044BE8
:10DA78001A6000F02DF9BDE8084011F07DB800BF2C
:10DA8800D00300240146014828F016BE800D00246A
:10DA98000146014828F023BE800D0024024B586837
:10DAA800003818BF01207047F4210024034B0448B4
:10DAB8005B68002B08BF0020704700BFF4210024DA
:10DAC800800D0024034B1B7813B9034829F034B8A0
:10DAD800704700BFA92900248A46059010B1034B5E
:10DAE80001221A70024800F06FBB00BFAA29002467
:10DAF80004220024F8B5254B1D7825B10120BDE886
:10DB0800F840FFF7EBBF224B22481D702AF093F82C
:10DB180020482AF076F858B91E4801272AF083F8D9
:10DB280080F00104012000F03FFB0546E4B20AE062
:10DB380028F0DDFF0028EFD016482F462AF073F8AA
:10DB480080F00104E4B2F4B1012000F035FB064690
:10DB5800114828F0F1FF114828F0EEFFFEF766FEA5
:10DB68000F4828F0E9FF0F4828F0E6FF0E4828F094
:10DB7800E3FF17B1284600F017FB34B13046BDE883
:10DB8800F84000F019BB2646E2E7F8BDA9290024B1
:10DB9800AA290024D80300249146059096460590AA
:10DBA8009B4605909F4605908E460590044B1B7832
:10DBB80023B9044B1B780BB1FFF79CBF704700BF1C
:10DBC800A9290024AA290024014B01221A707047B0
:10DBD800A9290024024B002202481A7000F0F4BA66
:10DBE800A929002404220024034B044A04481A608B
:10DBF80000225A602AF019B804220024B5DB0090EC
:10DC0800D8030024014829F072B800BF1822002464
:10DC180038B5094D04462B6883420CD0074B197858
:10DC280028F08FFDB0FA80F12C6049090448BDE85E
:10DC3800384000F015BD38BD14220024B506002474
:10DC48001822002438B50B4D2C7894B901230A49C1
:10DC58000A482B7000F0E8FC22462146074829F0C4
:10DC68006EF8074B4FF0807218681A60FFF7D0FF04
:10DC78002C7038BDAB290024D097049018220024BA
:10DC880014220024014B1870704700BFB506002409
:10DC9800014B1878704700BFB5060024F8B50E464A
:10DCA8001C4615466AB1094F3B781BB900F04AFB80
:10DCB80001233B702246691E3046BDE8F84010F04B
:10DCC800E5BF012B94BF00200120F8BDAC2900243A
:10DCD80010B5054C10F038FF23780BB100F044FB69
:10DCE8000023237010BD00BFAC2900240F4B10B5D2
:10DCF80003600446838843F0050383802FF0F4F81B
:10DD080001230E220A4984F88430231D61612361AE
:10DD18000849A060C4F88040E260A162C4E9082311
:10DD2800C4E90D23044BE36310BD00BF68E1049010
:10DD380087670390A5DC0090E968039008B5FFF7B2
:10DD48006FFC044B03F178029A62BDE8084011F0B9
:10DD580077B800BF0C230024014B00221A607047DB
:10DD680024220024034B01221A700022024B1A605D
:10DD7800704700BFAD29002424220024014B002253
:10DD88001A707047AD290024024A136803431360D0
:10DD9800704700BF28220024024A136823EA0003C0
:10DDA8001360704728220024014B1878704700BF81
:10DDB800AD29002410B50C4C206890B10B4B1B68A2
:10DDC80083B928F0E6FE236883422368A0EB0300AA
:10DDD80040F2EE2388BF00F1FF30984294BF002044
:10DDE800012010BD0020FCE7242200242822002462
:10DDF800024B1868003818BF0120704724220024FD
:10DE08000129024610B50C4617D9042915D00B492B
:10DE18000B482CF00DFE022C03D0052C0BD0094921
:10DE280000E0094906482CF003FE08490448BDE80B
:10DE380010402CF0D8BD0649F4E710BDD3950590E5
:10DE4800C8CC049016930590C69205901082059050
:10DE5800D19205902DE9F04F9DB080460C46924630
:10DE680000AFFFF723FE28B9012528467437BD46C1
:10DE7800BDE8F08F01239F4A07F1180180302FF089
:10DE8800E0FF0028F0D1D7E91402D7E90A139A4233
:10DE980008BF884200F02B8197F84930002B40F0EA
:10DEA800268107F1180028F04AFD5B28064606D1AE
:10DEB80007F11800D7E90A2330F0D8FBE3E7002E72
:10DEC800F6D008F1FF3919F8015F2DBB304603F091
:10DED8002DFA20B107F1180028F031FD06463D2E35
:10DEE8001CD107F1180028F02AFD22280CBF0123B5
:10DEF80000238AF8003040F0CA8007F1180028F0A3
:10DF08000FFD22282AD016D830B30A2824D0C1B24F
:10DF1800204628F02CFDF0E7B54206D00A2EB2D0F4
:10DF280007F1180028F01AFDADE707F1180028F0EE
:10DF3800F7FC0646C7E75C28E9D107F1180028F086
:10DF4800EFFC7628E3D861281DD80A2804D0552884
:10DF580000F089800028DAD1052509E007F11800CA
:10DF680028F0EDFC0A2803D0232807D00028F3D195
:10DF7800EDB207F1180030F0A4FA76E707F11800BF
:10DF880028F0ECFCF4E7A0F16203142BBFD801A23F
:10DF980052F823F093E0009017DF009017DF00900D
:10DFA80017DF009001E0009017DF009017DF009066
:10DFB80017DF009017DF009017DF009017DF009041
:10DFC80017DF0090F5DF009017DF009017DF009053
:10DFD80017DF0090F1DF009017DF0090F9DF009065
:10DFE80005E00090FDDF00900D2090E70A208EE705
:10DFF80009208CE70B208AE70C2088E73B1D6E463A
:10E008004FF004099B46D84609EB0B0A07F11800A4
:10E0180028F086FC08F8010BD045F7D100233946D3
:10E02800102258460BF8093022F0A0F93B68014647
:10E03800434528D1B0F5881F22D27F281AD9B0F5D8
:10E04800006F19D3B0F5803F34BF03230423227B2C
:10E0580022B16268134422689A420FD920462EF0F2
:10E068001AFEB54649E707F10C036E464FF008095A
:10E078009B46C8E70123EAE70223E8E76360F0E785
:10E088000225B54674E7B54666E708203FE70A2843
:10E098003FF462AF00283FF45FAF00250D281CD085
:10E0A80009DC092819D00A2800D040B963685B1B2D
:10E0B800636000255CE720280FD0232805D0C1B273
:10E0C8002046002528F053FC0CE0636807F118008F
:10E0D8005B1B636028F042FCEBE70135C1B22046C8
:10E0E80028F045FC07F1180028F01AFCD6E70425AB
:10E0F8003FE700BF1C46059070B586B00E4610225B
:10E108000DF1070302A928F03DFC044648B99DF823
:10E1180007507DB9084902A8F3F7FAFA20B9012592
:10E128003570204606B070BD044902A8F3F7F0FA2E
:10E138000028F5D00524F4E7A6460590AB460590DF
:10E1480010B5054C23782BB928F0C1FC11F02AF83A
:10E158000123237010BD00BFAE29002473B5054606
:10E168000C4669B10D4B1B786BB90A4601AB0146E9
:10E178000B4829F073FE06460A4B1B782BB1344630
:10E18800204602B070BD0E46F6E72146284628F024
:10E19800A6FC2146284611F02DF8F0E7AF29002407
:10E1A800E0030024B0290024024B1A7818701046A6
:10E1B800704700BFB0290024024B1A781870104627
:10E1C800704700BFAF29002410B5044601F0C4FD14
:10E1D800E3681BB90C4A1168A14203D1BDE810409D
:10E1E80001F0D4BDA360094B1968E160196809B151
:10E1F80019688C60116801B914601C6001F0C6FDD3
:10E2080010F01EFE10BD00BF34220024302200246E
:10E218002DE9F041144E31F066FB33680BB3134D12
:10E2280001F09AFD2C681CB1BDE8F04101F0AEBDCB
:10E2380001230F4A2B603368346014601BB92B68C4
:10E24800013B2B60F0E7D3E900689F68C3E902440B
:10E2580001F09CFD0EB14046B04701F07DFD3B4604
:10E26800ECE7BDE8F08100BF342200242C22002412
:10E27800302200242DE9F7430025154E01AF019502
:10E28800A84601F069FD346854B9019B3360114B0D
:10E298001D60114B1C6003B0BDE8F04301F076BD72
:10E2A800D4F808902046C4F808800FF0E3FE18B1AF
:10E2B8000023E3604C46E7E760680FF0DBFE0028C8
:10E2C800F6D12B463C60254604F10807F1E700BF6C
:10E2D80034220024302200242C220024044B10B5C0
:10E2E8001C6804B910BD60682EF0C1FDA468F8E789
:10E2F8003422002408B531F0F3FA28F03FFA00F090
:10E30800E9F9FFF7D3FA31F0EDFA28F037FA0020EF
:10E318002EF0FFFD034BC3E90001BDE8084031F0D2
:10E32800E0BA00BF501E002408B5FFF7D1FA00225A
:10E3380002490348BDE8084028F008BCFDE2009007
:10E348003C22002410B5074C01F006FD23680BB9E8
:10E3580010F098FD236801332360BDE8104001F0F8
:10E3680015BD00BF3822002408B501F0F5FC074BA5
:10E378001A6812B11A68013A1A601B680BB910F0D2
:10E388008FFDBDE8084001F001BD00BF3822002420
:10E398002DE9F843DFF87C8000AF05460E4628F0EB
:10E3A800E9F9D8F8003043B31B4828F05AFCC0F507
:10E3B80000720446D8F8000043689919914223D99D
:10E3C8000734D21A2946E94624F007042EF0D4FB74
:10E3D8001148ADEB040DD8F80040694600F050F83C
:10E3E800014620462EF09FFC0A21D8F800002EF0A6
:10E3F8004BFC0023C8F80030CD4631462846FFF7CD
:10E40800ADFEBD46BDE8F883324629462EF0B4FB82
:10E41800F3E700BF98210024338E0590A1F1800313
:10E42800542B70B5064618D819460E480E4C0223D0
:10E4380010F8012B914205DA03FB0144E518A542C7
:10E4480005D870BD03FB0244891A0133F0E714F8BC
:10E45800011B3046FFF7E2FFF1E7BDE870402EF000
:10E468001ABC00BFB4460590BE4605900246024954
:10E4780002482CF0B8BA00BFB1460590F0D204901B
:10E488002DE9FF4105460A466846802415F8011B18
:10E49800274F0131DFF89C802EF0B2FB009E013E31
:10E4A800019B9E4205D868462EF0DFFB04B0BDE80C
:10E4B800F0810023184619461A4695F800C0520004
:10E4C800013114EA0C0FC9B214BF4FF0010C4FF020
:10E4D800000C64084CEA020204BF01358024824221
:10E4E80005D317F801C00CEB40006344E5E71B1A9D
:10E4F8004244D15C012917D10B2300202A7840001F
:10E50800144214BF01220022640840EA020004BF3A
:10E5180001358024013BF1D101302AF0EDF80146A4
:10E5280068462EF000FCBBE76846FFF777FFB7E7C1
:10E53800FE48059053480590F7B504460D46836894
:10E548005B6CD3B9A3685B6BE3B9194FA3689B698C
:10E55800B3B101220DF1070120469847012806466C
:10E568000ED19DF807203B689A4210D105F10800AA
:10E5780027F03BFC02F080FEE8E798470028E1D14D
:10E5880003B0F0BD204698470028DED1F8E795F89B
:10E598004830002BDAD1002200230DF1070105F1E4
:10E5A800080027F01BFC0028D0D085F84860CDE78C
:10E5B800C4030024F8B51E46174B04460D461746FB
:10E5C800C0E900318B68F3B19B6CE3B10246134993
:10E5D800284698473B460122314604F1080027F0B7
:10E5E800EAFB4FF0FF324FF0FF33C4E90E23C4E9D2
:10E5F8001023002384F84830AB689B6A0BB1284687
:10E6080098472046F8BD6FF05703054A0121054891
:10E6180024F0D5FEDEE700BFE4A5049041E50090B4
:10E628000B490590987D049038B50C460546084678
:10E6380027F0C4FF6C60606827F0D7FA20B9074854
:10E6480024F082FB012038BD4FF48032217A6068C3
:10E6580028F03CFB0028F5D12872F4E73A490590E8
:10E6680038B543680C460546012158681B7A99401D
:10E6780003691B68194214BF84F0010323464BB198
:10E688008368DB689847014610B1044824F05CFBB6
:10E698006C7238BD83681B69F4E700BF5149059067
:10E6A80038B501294368094A04460D4618BF4FF496
:10E6B8000032197A586828F009FB014620B104484D
:10E6C80024F042FB012038BDA572FCE706000200D9
:10E6D8006949059008B5FEF75BFF10B9FFF76AFBBB
:10E6E800A8B108BD114A934203D1BDE8084028F0FB
:10E6F80056BF0F4A934203D1BDE8084000F07EBDE3
:10E708000C4A9342EDD1BDE8084029F028BF0A48D9
:10E718000368002BE5D0094A9342E2D0084A9342A5
:10E72800E0D1BDE8084031F00EBC00BF48A9049014
:10E7380020A7049050AE0490581E002408D90490D5
:10E748000CF0049070B54FF0FF33244E244C336026
:10E7580023682BB933681BBBBDE8704013F072BF48
:10E76800204DAB42F6D0204A934204D1204631F0E6
:10E7780003FC2560EEE71D4A934203D1204600F0D2
:10E788006DFDF6E71A4A934203D1204601F0C8F816
:10E79800EFE7184A9342ECD1204602F01FF8E8E769
:10E7A800154C2368002BD7D00E4DAB42D4D0134A5A
:10E7B800934204D1204628F0CDFB2560CCE7104ACF
:10E7C800934203D1204601F023FAF6E70D4A93421B
:10E7D800F3D1204601F02CFDEFE700BFD40300245D
:10E7E800581E002408D904900CF0049020A7049027
:10E7F80048A9049050AE04904C220024C0A804906C
:10E80800C4AA049014AD0490F8B5374C374E236869
:10E818000BB1B3420DD1266035480368002B61D097
:10E82800B3425FD0334A934247D1BDE8F84015F070
:10E83800EDB9314A934216D16568A54203D304F174
:10E8480098039D42E8D928460FF014FC0028E3D02D
:10E858002A4B6C222946184638F0F3FE6060284699
:10E8680031F008FCD8E7264A93421FD16568A542D3
:10E8780003D304F198039D42CED928460FF0FAFB42
:10E888000028C9D01D4A2B4605F1200E9446186869
:10E89800083353F8041C1746734503C73A46F6D1A4
:10E8A8002846C4F804C031F026FDB5E7154A93425E
:10E8B800B2D1204629F0FAF8AEE7134A934203D1C1
:10E8C800BDE8F84000F0F6BC104A934203D1BDE819
:10E8D800F84001F037B80E4A934203D1BDE8F8403A
:10E8E80001F08CBFF8BD00BF4C22002408D9049069
:10E8F800581E00240CF00490C0A804905422002450
:10E90800C4AA049014AD049020A7049048A90490C8
:10E9180050AE0490174808B503681BB91648036839
:10E928004BB908BD154A9342F8D0154A9342F5D120
:10E9380029F050F9F2E7114A9342F2D0114A934272
:10E9480003D1BDE8084031F026BB0F4A934203D1FA
:10E95800BDE8084028F03CBE0C4A934203D1BDE80C
:10E96800084028F08DBA0A4A9342DAD1BDE8084037
:10E9780029F00EBE4C220024581E002408D9049009
:10E9880014AD04900CF0049048A9049020A70490BA
:10E9980050AE0490084B10B5084C1B68A34200D039
:10E9A80043B9074BB4220021184638F072FE40F8EC
:10E9B800044D10BD0020FCE7581E002408D904901F
:10E9C8005C1E002408B5FFF7E5FF10B9014804F004
:10E9D800FFF908BD868F0590084B10B51B68084CD9
:10E9E8000BB1A34208D1074B94220021184638F0F6
:10E9F80050FE40F8044D10BD0020FCE74C220024D6
:10EA080008D904905022002408B5FFF7E5FF10B993
:10EA1800014804F0DDF908BD8C8F0590094B1B688F
:10EA28005A1C0DD0002B0BDCB8225343064A981809
:10EA3800D358064A934203D0002B08BF0E207047D4
:10EA48000E207047D4030024581E002408D90490CF
:10EA58000E2807B513D00E4A9042136803D10D4A09
:10EA6800934200D093B908F02DFEC388E7224FF4F3
:10EA78008A7100934FF4AA73074804F0E5F94FF040
:10EA8800FF33064A136003B05DF804FB0023F8E780
:10EA9800581E002408D9049039970590D4030024FF
:10EAA800074A1368013304D1064B07491B688B4298
:10EAB80000D17047002BFCD000231360704700BFC3
:10EAC800D4030024581E002408D904902DE9F04FDF
:10EAD800044685B01F464FF0000800F15009CDE903
:10EAE8000212B84502D305B0BDE8F08F039B03EBD3
:10EAF800080694F8B530757896F901B0002B37D030
:10EB0800B57806F1030A484617F0FAF8A8B30123C6
:10EB180000210093334694F8B620206DD4F860C0E5
:10EB2800E0470095534694F8B6200121206DD4F8AB
:10EB380060C0E047484632F0DAFBBBF1000F23DB48
:10EB4800002029F019FB029B3BB1D4F88430164A07
:10EB5800934202D0204628F022F9FEF719FD00283A
:10EB6800C1D194F8B5304544DBB905F10208B8E7DE
:10EB780006F1020A05F07F05C5E7FEF709FD002842
:10EB8800C5D1FFF745FBBEE76B1C94F8B520DDB295
:10EB980056FA83F313445878FF2808BF4FF4FA70E5
:10EBA800CFE705F103089CE708D90490F0B54B6B53
:10EBB8008BB005460C46002B00F0C980012380F875
:10EBC8004030486B31F0D4FE85F83C00636B002B75
:10EBD80000F0C080A36B002B00F0BC804FF4807362
:10EBE800A5F84030A06B31F0C3FE85F83D00B4F8BD
:10EBF8005630002B16BF01230023042185F8B430BA
:10EC080094F8573085F8423094F8563085F84330F8
:10EC180008BF012394F8556018BF0026626B0CBF2B
:10EC2800194633460AB9A26B32B1228EB2F5807FFB
:10EC380002BF002602213346012205F10800002701
:10EC4800CDE90422CDE90222CDE90013638C228BA1
:10EC5800E18A32F064FA94F85930089705F15000C7
:10EC6800099394F85430CDE90673638D0593238D89
:10EC78000493E38C0393A38C0293B4F9203001939B
:10EC8800B4F91E300093628BA38B216816F0B0FF95
:10EC9800A38D3249A5F8AA3094F82E3085F8B03003
:10ECA800238EA5F8AC3094F8323085F8B130606C1A
:10ECB800F2F7A2FAF2F7A2FCA5F8A80094F84C30F3
:10ECC800264985F8AF3085F8B270206DF2F794FACE
:10ECD800F2F794FCC5F8900094F8543085F8B360C6
:10ECE80085F8B63063681D49C5F894302389A5F8BE
:10ECF800A030E068F2F780FAF2F780FCA5F8A600E9
:10ED08002369C5F89830A38AA5F8A230E36BC5F843
:10ED18009C30B4F84030A5F8A430114BC5F88430C5
:10ED280094F8583085F8B530A36C4BB128460D4B94
:10ED380040F8843FA16CFFF777FCA06C27F03CFCFF
:10ED4800094928460BB0BDE8F04028F06DB880F8B6
:10ED580040303BE7002385F8413048E700007A441B
:10ED680008D9049038F50490D405002410B50B6830
:10ED78000446C0F894304B680549A0F8A030104606
:10ED8800F2F73AFAF2F73AFCC4F8900010BD00BF67
:10ED980000007A4410B5038F04465A2B02D0B3F50D
:10EDA800877F19D15A2902D0B1F5877F19D104F18B
:10EDB800080032F073F90E4B9C4205D113F042FC67
:10EDC800E18EA08E13F0E0FAA06878B104F1180182
:10EDD800BDE8104031F081BC5A2902D0B1F5877FD7
:10EDE800E5D1A38EE28EE386A286E0E710BD00BFE0
:10EDF800581E00242DE9F04F97B0044690F8B23021
:10EE080002AFE3B1D0F88420B14B9A4217D18430D5
:10EE180027F078FF94F8AF30834204D100205437AC
:10EE2800BD46BDE8F08FFFF79FFA0021B4F8A23085
:10EE38002046D4F8982084F8B210FFF747FEA3685C
:10EE4800002B00F0BF81204627F0F7FF0028E5D10E
:10EE580004F1500A504632F03FFA0028DED094F808
:10EE68004810002900F099800023236304F1280347
:10EE7800FB6294F8B430002B40F0A080FEF788FBCA
:10EE880078610028CAD1204627F09BFF04F1080BBF
:10EE980007F13802F96A5846C7F810D032F0DDF9A0
:10EEA800002800F0848107F13800202532F005FCA5
:10EEB80094F83A30064607F13800B5FBF3F532F01E
:10EEC80001FC814607F138004FEAC51832F0FAFB19
:10EED800B0EBC51F00F2C98001231FFA89F03B621D
:10EEE80080239B0000254009BB610733013023F0D4
:10EEF80007037863ADEB030D7B6B9B000DF10808EE
:10EF0800073323F00703ADEB030D02ABBB62B4F884
:10EF1800AC30B3F5807F14BF02230123BB60BB690B
:10EF28004344FB6007F1380032F0C7FBB4F87A308D
:10EF38007862B3F5807F05D007F13802594650460C
:10EF480032F0D8F9B4F8AA3087F833301DB1B4F8E4
:10EF5800AC3087F83330504616F0D2FE002800F067
:10EF68002681012394F8B6200021009307F133038A
:10EF7800206DD4F860C0E047504632F0B8F900235D
:10EF88009946FB61BB8B3A6A9A4200F2A3806B1CDC
:10EF9800BA6801259A42C5D809E1A068002800F09E
:10EFA800118116F045F8F862002800F00B81B4F8DA
:10EFB8007A30B3F5807F7FF45CAF55E704F108063B
:10EFC800204627F0FEFEC7F828D0304632F00AF96E
:10EFD80005463046C5F34F0532F006F977218046DD
:10EFE800EB1D2A4623F00703ADEB030D0DF10809CD
:10EFF800484638F04EFBB4F8AA30504687F84430FB
:10F0080016F07EFE834688B12046D7F828D027F030
:10F01800F7FE94F8B230002B3FF430AFFEF7B8FAA1
:10F0280000287FF42BAFFFF7F3F8F2E7012394F8F9
:10F03800B6200146009307F14403266E206DB047C1
:10F04800504632F054F91FFA8BF39845DCD95046F4
:10F058000BF1010B16F054FE0028D5D094F8B62019
:10F068004B4600950121266EE8E707F1380032F09B
:10F078001FFBB8FBF0F0002808BF012086B207F19B
:10F08800380032F01AFBB0FBF6F083B207F1380013
:10F098003B6232F012FBB0FBF6F303FB160080B2C2
:10F0A80018B13B6A01339BB23B6207F1380032F07A
:10F0B800FFFA16FB00F080B2B0FBF5F293B205FB45
:10F0C8001202002A3FF40DAF01339BB209E700BFDB
:10F0D80038F504907B697A8F786AFB643B8F8642A7
:10F0E800B7F93C1007F14400A7F8443002EB0903D4
:10F0F80094BF92197A6A9BB2A7F8481098BF4A44FD
:10F10800A7F846308ABF9B1813B21BB2A7F84A303B
:10F118007B6A9B1B9BB27B6232F0D4FA94F83A303C
:10F1280008220021B2FBF3F3B0FBF3F37A6BB86A61
:10F1380092007B6038F0ADFABA690021404638F099
:10F14800A8FA94F8B43013B940F20713E387D5B19D
:10F1580094F8B33063B1062384F83E304346BA6A64
:10F1680007F14401584632F06BF894F8B13013E0D7
:10F1780094F8402012B184F83F30EFE7B4F84230F9
:10F18800002BF2D0EAE74346BA6A07F14401584631
:10F1980032F056F894F8B030B3B95046B14416F08E
:10F1A800AFFDFB691FFA89F90133FB61A8B9FB6A56
:10F1B800D7F810D09B68FB62002B7FF467AE20461F
:10F1C80027F01EFE01202AE64346FA689342E4D05F
:10F1D8001A68D24343F8042BF7E7BB88012194F857
:10F1E800B62000934346206DD4F860C0E0475046EF
:10F1F80032F07DF8FFF70CF8C4E600BF10B590F8C0
:10F20800B23004463BB3D0F88420134B9A4214D151
:10F21800843027F077FD94F8AF3083421BD0FFF796
:10F22800A3F80021B4F8A2302046D4F8982084F836
:10F23800B210BDE81040FFF749BC27F09BFCD4E9A9
:10F248000432C01AB4F8A83061EB020183424FF0CF
:10F2580000038B41E3D310BD38F5049010B590F846
:10F26800B230044693B1D0F88420104B9A4201D0B2
:10F2780027F095FDFFF778F80021B4F8A230204672
:10F28800D4F8982084F8B210FFF720FC04F10800A5
:10F2980031F0CAFFD4F88420054B9A4205D104F115
:10F2A8008400BDE8104027F022BD10BD08D90490A5
:10F2B80038F5049010B504490446083031F064FF6D
:10F2C800012384F8483010BDD405002410B50B4C38
:10F2D8000B4B22689A420ED1A2680A4B9A420AD175
:10F2E800204627F0AAFD28B92046FFF783FD80F0C5
:10F2F8000100C0B210BD0020FCE700BF581E00246A
:10F3080020A70490D4050024014808B503F058FD4F
:10F318000296059010B5044929F048FD044603F00B
:10F3280045F9204610BD00BF20A70490F0B50C4653
:10F3380089B00646174654F8040BFFF7EBFF03ABFA
:10F3480005463A46019321460A4B701E0093022354
:10F3580007F07EFC05A90522039808F05DFD0498D6
:10F3680008F060FB05A902462846FFF7FFFC0E20BF
:10F3780009B0F0BD10A7049008B5FFF7CBFFFFF761
:10F3880039FD10B9024803F023FD0E2008BD00BF67
:10F39800AE90059010B5FFF7BDFF27F04EFDA0B168
:10F3A8006430F1F7B7FA00220A4BF1F757FCF1F78E
:10F3B800C5FD01460446F2F7E5F840B924F003001C
:10F3C80040F00200A0F1FF4010BD0348FCE70348ED
:10F3D800FAE700BF00408F40020080800200400032
:10F3E8002DE9F04FCBB0084611461A462AAB0193D7
:10F3F8006A4B009320232BF032F82A9B05220AA996
:10F408002B98039308F008FD05220DA92C9808F005
:10F4180003FD40F25331409828F0DDF9339F5A221A
:10F42800049097FBF2F302FB137313B15C4803F0EB
:10F43800B1FCFFF7C7FA05463F9808F0F3FA834690
:10F44800429808F0EFFA8246489808F0EBFA3C9B9D
:10F4580080463A9805930E283D9B069300F08C80D1
:10F468002BF069F906463E9C09A99DF81C91204697
:10F4780008F05AFA002800F08280032029F076F973
:10F48800099B0446037000234370837009F102034B
:10F49800444A00210DF1560007932A60522238F0A1
:10F4A800F8F80A9A039B2846149213A90B9A139307
:10F4B800ADF854200D9ACDF8588017920E9AADF8F1
:10F4C8006E70ADF860202D9AADF862202E9AADF8D6
:10F4D80064202F9AADF86620309AADF86820319AEA
:10F4E800ADF86A20329AADF86C20349AADF87020E5
:10F4F800359AADF87220369AADF87420379AADF87F
:10F508007620389A059BADF878202093069B9DF8C5
:10F51800E420ADF87C608DF87A209DF8EC20CDF8D9
:10F5280090B08DF87E20CDF89CA08DF8A490CDE900
:10F538002134079BADF88C30049B25939DF804314A
:10F548008DF898309DF80C318DF8A0309DF8103169
:10F558008DF8A1309DF814318DF8A2309DF818313E
:10F568008DF8A3309DF824318DF8A530FFF71EFBE8
:10F5780028464BB0BDE8F08F4FF4807673E7012240
:10F5880010A9204608F048FC10B1DDE910437FE7D8
:10F5980040F29141044803F043FC00BF10A60490D8
:10F5A8003794059020A70490E792059070B58AB02B
:10F5B8000C460138043104AB01931A4B0093032322
:10F5C80007F046FBFF22002140F26F33049807F052
:10F5D800DBFB05228DF80F0007A90598246808F0C1
:10F5E8001BFC204627F073FDC0B19DF8186001256B
:10F5F8000DF10F03204632460021009527F087FDC4
:10F60800089B3246294620460093079B27F07FFD3A
:10F61800204627F0FDFD0E200AB070BDFEF7F8FD6C
:10F62800DFE700BFA8A8049070B58CB00846114663
:10F638001A4605AB0193184B009307232AF00FFFD6
:10F6480040F2E5421549059807F0D6FB0646FFF754
:10F65800DBF9134B044601220360002140F2724398
:10F668000A9807F091FB40F2674305460122002102
:10F678000B9807F089FB099BC0B231460193EDB2A4
:10F68800089B0390204600930295DDE9062327F0A6
:10F69800AAFC20460CB070BD70A8049050F20490EB
:10F6A800C0A8049008B527F082FC20B940F29D411B
:10F6B800024803F095FB0E2008BD00BF1992059083
:10F6C800436DDB6B0BB1006D18470148704700BFF5
:10F6D800000080BF10B5038F04465A2B02D0B3F543
:10F6E800877F19D15A2902D0B1F5877F19D104F142
:10F6F800080031F0D3FC0E4B9C4205D112F0A2FF5A
:10F70800E18EA08E12F040FEA06878B104F11801D5
:10F71800BDE8104030F0E1BF5A2902D0B1F5877F2B
:10F72800E5D1A38EE28EE386A286E0E710BD00BF96
:10F73800581E0024F8B590F8783004460D46174650
:10F7480043B100230126204684F8793027F070FD64
:10F758003046F8BD90F87960002EF2D14B1CF0D0FD
:10F7680027F008FA2369C31ABB4202D90D4803F0EF
:10F778002FFBA26E821A9542C4E91A01E8D3B3FBA3
:10F78800F5F205FB1233ED1A27F0F4F9D4E91A3231
:10F79800C01A61EB0201A84271F10001D1D2FEF753
:10F7A80037FDF1E78A9505902DE9F04F1F460023B4
:10F7B8000446016580F878308BB040F27A40904674
:10F7C80001F0A2FD6065C369002B00F09180206DF7
:10F7D800984786B2636D04F1080B206D1B69984742
:10F7E80083B2206D0793636D5B69984783B2089372
:10F7F800636D5B6A002B7DD0206D98478146636DF1
:10F80800DD6A15B1206DA8470546636D9B69002B1D
:10F8180077D0206D98475FFA80FA636D1B6B13B140
:10F82800206D98470346626D526B22B1206D099393
:10F838009047099B02465846CDE90432CDE9025A61
:10F848000023DDE90712CDE9006931F068FC636D3A
:10F858001B6A13B1206D984783B2A4F87430636DA6
:10F86800206D9B6B002B4FD1A38E94F83A20534305
:10F87800DB10A4F87630636D04F15801206D5B68E5
:10F888009847E28EB4F87610013AB4F87430E06D17
:10F8980001FB023394F83A20A18E514340F2D7324B
:10F8A80003EBD10107F080FA87F0010384F879307F
:10F8B800636D9B6A7BB3206D984780B24FF47A736F
:10F8C800A4F87000B3FBF0F3A4F87230B8F1000F9D
:10F8D80003D041462046FFF7FDFE1049584631F057
:10F8E80053FC394620460BB0BDE8F04F27F043BE25
:10F8F80010266FE7072E8CBF4FF000094FF0010963
:10F908007DE74FF0020A88E7984780B2A4F87600AE
:10F918000028B0D1A8E73C20D0E700BFD4050024D8
:10F9280010B50446002127F026FE04F1080031F046
:10F938007BFC636D206DDB689847014B236010BD2D
:10F9480008D9049010B50446006D07F0BBFE78B1E5
:10F958000A4B98420CD00121204627F00CFE08499A
:10F9680004F1080031F010FC012384F8483010BD80
:10F978002046BDE81040FFF7D3BF00BF08D9049068
:10F98800D405002408B5083031F0FEFB10B9024850
:10F9980003F000FA0E2008BD82930590014808B5CF
:10F9A80003F00EFA0296059010B5044929F0FEF905
:10F9B800044602F0FBFD204610BD00BF48A9049094
:10F9C80030B585B00C460138043102AB0193144BB5
:10F9D8000093022307F03CF92068FFF7E5FF039B3B
:10F9E80005460298002BCABF4FF47A744FF0FF34D3
:10F9F80094FBF3F40E280FD02AF09DFE4FF47A7191
:10FA080091FBF0F122462846FFF794FE00280CBF30
:10FA18001E203E2005B030BD4FF0FF31F2E700BF99
:10FA280038A9049010B5FFF7BFFFFFF749FE002182
:10FA38000446F1F77FFD10B1084803F0C9F92146E3
:10FA48002046F1F79FFD30B924F0030040F0020092
:10FA5800A0F1FF4010BD0248FCE700BF5695059095
:10FA6800020040002DE9F0418CB00C460138043109
:10FA780002AF07F1080301932B4B0093022307F011
:10FA8800E7F82068FFF790FF0622054607F1100106
:10FA9800D7E90286304608F0BFF9BB69012B02D0CE
:10FAA800224803F077F995F83A30102B01D0204816
:10FAB800F7E70023AC8E07F11C00FB61A7F81E8056
:10FAC80008F101087B623C846408A7F8228031F0C1
:10FAD800F9FDC30782B248BF0134D7E90431B1EB5D
:10FAE800840F1FD35209002101328C467A607A684C
:10FAF8009200073222F00702ADEB020D02AA88B28B
:10FB08007C68013184420AD807F11C0105F108001C
:10FB180031F096FB30462837BD46BDE8F08142F803
:10FB280020C0ECE70348BCE728A904904B95059052
:10FB3800499405903395059038B50C46FFF734FF86
:10FB480005460E2C0AD0204616F018FB014628461A
:10FB5800FFF718FF20B9034803F01CF90021F6E766
:10FB68000E2038BD8293059070B586B008461146C0
:10FB78001A4603AB01930F4B009303232AF06FFC43
:10FB88005A22DDE9036595FBF2F302FB135313B127
:10FB9800094803F0FFF8FEF715FF084B0446AAB220
:10FBA800036031469DF81430FFF7FEFD204606B08D
:10FBB80070BD00BF10A904903794059048A904901F
:10FBC80038B50C46FFF7F0FE0546204607F02AFF39
:10FBD80000210446F1F7AEFC28B94FF07E512046CB
:10FBE800F1F7C6FC30B10123002240F24B31064840
:10FBF80003F016F92146284627F0ACFC10B9034853
:10FC080003F0E6F80E2038BD6297059056950590EA
:10FC180010B50446406804F10803984201D130F059
:10FC280069FB0023A26A6360044B9A4205D104F180
:10FC38002800BDE8104027F05AB810BD38F50490E8
:10FC48000A4B10B5826A9A420ED000F128040021AE
:10FC58002046FEF705FD042027F0A9FD20460121D6
:10FC6800FEF7FEFC012010BD0020FCE708D9049037
:10FC78002DE9F04104460E4615461F467BB9154B43
:10FC88008362E9B2304630F037FBE0B9114B2046C9
:10FC98002360FFF7BDFF29460F4803F0C1F80F4B5B
:10FCA8008046394648F8283F4046FEF7BDFC00220A
:10FCB8000121404627F043F8384626F07DFC2046CF
:10FCC800FFF7BEFFDDE73046666030F0ABFBA58688
:10FCD800BDE8F08108D904901A8F059038F5049092
:10FCE80070B586B0084611461A4603AB0193104B0F
:10FCF800009303232AF0B3FB40F29D41059827F0B7
:10FD08006AFD4FF47F7206460A49039807F074F8B3
:10FD18000546FEF779FE084B04462946036033463C
:10FD2800BDF81020FFF7A4FF204606B070BD00BF45
:10FD3800ACAA0490CCF30490C4AA049008B5FFF7C9
:10FD48007FFF20B940F29D41024803F049F80E2098
:10FD580008BD00BF1992059010B50A4C23686BB90D
:10FD680026F09DF908B9FBF707FDEFF31182102380
:10FD780083F31288BFF36F8F034B1A602368013334
:10FD8800236010BDE4220024E822002408B50C4BAF
:10FD98001A6812B90520FDF709FD1A68013A1A60B8
:10FDA8001B6863B9074B1B6883F31188BFF36F8F18
:10FDB80026F075F918B9BDE80840FBF7F1BC08BD95
:10FDC800E4220024E8220024F7B5184CA568E66868
:10FDD80001950025ECB2019FA74215D8144CA568DF
:10FDE800E66801950025ECB2019FA7421CD906EBF5
:10FDF800C40C0135DCF80470B842F4D140F2394043
:10FE0800086040F269410AE006EBC40C0135DCF8F1
:10FE180004708742DED10020086040F2463111604C
:10FE280056F8342012091A6003B0F0BDAC8804906B
:10FE3800D489049010B54FF4307386B00446084650
:10FE480004AA0393059303A905ABFFF7BDFF039A23
:10FE5800059B3AB100932046049B06492AF0C3FD4E
:10FE680006B010BD049A2046034906B0BDE810400C
:10FE78002AF0B9BD86490590894905900A46014985
:10FE880006F0BABF14AB04901FB5044688B10E281B
:10FE98000FD026F094FB60B94FF4307301A92046C7
:10FEA80002AA039303ABFFF78FFF0399024802F0FE
:10FEB800B7FF04B010BD00BF9497059008B526F0B1
:10FEC80082FB01460248BDE808402AF06CBA00BF30
:10FED800F4AB04900E2373B50B600D4601A900F036
:10FEE800F5FC012804460FD9019E3046F1F722FCA3
:10FEF8000246012A03D9531EF15C2F2907D0314647
:10FF080004480BF065FD2860204602B070BD1A4613
:10FF1800EFE700BFF0C804900E2373B50B600D46E1
:10FF280001A900F0D3FC0128044609D9019E3046F6
:10FF3800F1F700FC3146024603480BF049FD286002
:10FF4800204602B070BD00BFF0C80490F8B5037831
:10FF580000AF06462F2B6BD0524CD4F8B45045B99D
:10FF6800022028F003FC05464F49F1F7DBFBC4F8F3
:10FF7800B4502846F1F7DEFB04463046F1F7DAFBC9
:10FF88002044023028F0F2FB04462846F1F7D2FB61
:10FF980029460246204637F054FB2846F1F7CAFBAB
:10FFA800054638B1231813F8013C2F2B1EBF2F2309
:10FFB800013523543046F1F7BDFB3146421C601928
:10FFC80037F03FFB2046F1F7B5FB002221461346E8
:10FFD800154690422ED145B39B002046651E073337
:10FFE80023F00703ADEB030DF1F7A4FB00236E46E6
:08FFF80020441A46194615F8D1
:02000004900169
:1000000001EF02F1010CBEF12F0F04F802E002D063
:10001000BEF1000F46D1012B30D115F8013C2E2B3B
:100020003BD14B1E56F8232000238542E7D1002305
:10003000A3542046BD46F8BD1E4D9EE711F801CBE6
:10004000561CBCF12F0F15D102F1020C0133604593
:1000500010D991F800C0BCF12E0F0BD191F801C05E
:10006000BCF12E0F06D10332904205D08A782F2A98
:1000700008BF01253246B0E70125FBE7022B0CD172
:1000800015F8013C2E2B08D115F8023C2E2B04D17B
:100090008B1E013956F82320C6E746F821C0624678
:1000A0000131C1E701336246BFE700BF0C230024E2
:1000B000733005908445059037B5134CFFF74AFF20
:1000C0006946C4F8B400FFF709FFC4F8EC00B0B902
:1000D000D4F8F0400CB903B030BD6568012D0CD1E7
:1000E00029460A480BF052FC01AB01902A4640F227
:1000F0005D31204627F0BBFBEDE7E468EAE76B469D
:10010000012240F25D31F5E70C23002473300590A5
:10011000084B10B5D3F8B4404CB12046F1F70EFBB4
:10012000214602460448BDE810400BF055BC66204D
:1001300010BD00BF0C230024F0C8049037B5FFF7B2
:1001400009FF01A9FFF7CAFE28B9144BD3F8F00044
:10015000A0B96623019301AB012240F2FF3127F0E1
:1001600086FB0021054608462BF02DF8044628465C
:1001700003F034FA38B9204603B030BD4368012B90
:10018000E7D0C068E4E70422012107F00DFE014634
:1001900020462AF006FFFEF73FF8E8E70C2300248C
:1001A00013B5FFF7D7FE01A9FFF798FE044610B973
:1001B000112003F093FD012807D001980CF022F9DB
:1001C0000649F1F7A9FA0028F2D001AB012240F26A
:1001D0003E41204627F04BFB02B010BD7330059026
:1001E00007B5FFF7B7FE01A9FFF79AFED8B9114B83
:1001F000D3F8F00080B901460A2008F0CDFA0122B8
:10020000031D00F1280143F8042F8B42FBD1C123C9
:10021000C36203B05DF804FB4368012B01D0C068E2
:10022000E8E76623019301AB012240F2EF4127F09A
:100230001EFBEEE70C23002410B50D4B04460268AC
:100240009A4214D1406804F10803984201D12FF07A
:1002500014FFA06F26F0B5F9D4F880000EF01CFF53
:10026000204698220021BDE8104037F016BA10BD94
:1002700014AD049070B58AB0084611461A4604AB16
:100280000193124B009306232AF0EDF840F25E3101
:10029000059827F09CFA40F2E5410646049813F0D1
:1002A000E7FF0546FEF7B4FB094B04463246036000
:1002B00029469DF824300293079B0193069B0093E7
:1002C000089B27F061FC20460AB070BDE4AC0490A6
:1002D00014AD049038B5437904460D468B4209D0DD
:1002E000837913B1044827F098FD6571BDE8384063
:1002F000FDF704BC38BD00BFE003002438B50C4650
:100300000F4D11461A460F4B9D4201D123F0F1F9D2
:100310000D4B9D42FAD00D4B9D42F7D00C4B9D42A8
:10032000F4D0A3070AD12368AB4207D130F0F3FD24
:1003300001462046BDE8384032F0D3B838BD00BF92
:100340009C01059040DC0490A4CB0490F0C804907C
:1003500008D90490F7B514460AB1002313701C4B5A
:10036000DFF870E0734501D123F0C3F91A4FBB42A7
:10037000FAD01A4EB342F7D0194DAB42F4D010F078
:10038000030210D1D0F800C09C450CD18DF8072095
:100390000DF1070231F08CFE14B19DF80730237087
:1003A00080B203B0F0BD0F4B7345DDD0BB42DBD054
:1003B000B342D9D0AB42D7D012B14FF6FF70F0E7BD
:1003C00002689A42F9D131F00FFDFF28E9D1F4E734
:1003D0009C01059040DC0490A4CB0490F0C80490EC
:1003E00008D90490CCFE049013B500230D4C0DF1F8
:1003F00007008DF807302CF090FDA0FB0432400878
:1004000040EAC17004FB012218189DF8073042EB46
:10041000510147F236725343C01841F1000102B056
:1004200010BD00BFB2E60E00014808B502F0CCFCDA
:100430000296059010B5044928F0BCFC044602F071
:10044000B9F8204610BD00BF50AE049030B585B05D
:100450000C460138043102AB0193144B0093022384
:1004600006F0FAFB2068FFF7E5FF039B05460298BC
:10047000002BCABF4FF47A744FF0FF3494FBF3F4AF
:100480000E280FD02AF05BF94FF47A7191FBF0F14E
:100490002246284600F0A0F800280CBF1E203E206F
:1004A00005B030BD4FF0FF31F2E700BF40AE049021
:1004B00010B5FFF7BFFF00F05BF800210446F1F72D
:1004C0003DF810B1084802F087FC21462046F1F7BC
:1004D0005DF830B924F0030040F00200A0F1FF40C5
:1004E00010BD0248FCE700BF569505900200400091
:1004F00038B50C46FFF79EFF05460E2C0AD0204665
:1005000015F040FE0146284628F04EF820B9034871
:1005100002F044FC0021F6E70E2038BD82930590DE
:1005200038B50C46FFF786FF0546204607F07EFAF1
:1005300000210446F1F702F828B94FF07E51204619
:10054000F1F71AF830B10123002240F24B3106488E
:1005500002F06AFC2146284627F0EAFF10B903485A
:1005600002F03AFC0E2038BD629705905695059032
:1005700000487047000080BF10B5038F04465A2B17
:1005800002D0B3F5877F19D15A2902D0B1F5877F00
:1005900019D104F1080030F085FD0E4B9C4205D1C5
:1005A00012F054F8E18EA08E11F0F2FEA06878B13E
:1005B00004F11801BDE8104030F093B85A2902D078
:1005C000B1F5877FE5D1A38EE28EE386A286E0E7D0
:1005D00010BD00BF581E0024F8B590F874300446D2
:1005E0000D46174643B100230126204684F8753096
:1005F00027F014FE3046F8BD90F87560002EF2D159
:100600004B1CF0D026F0BAFA2369C31ABB4202D9B8
:100610000D4802F0E1FBA26E821A9542C4E91A016C
:10062000E8D3B3FBF5F205FB1233ED1A26F0A6FA78
:10063000D4E91A32C01A61EB0201A84271F100013B
:10064000D1D2FDF7E9FDF1E78A9505902DE9F0415A
:100650001E46002386B0054617460C4680F87430C7
:10066000002943D16FF0120010F06CFC2C6505F1ED
:100670005408A368204641461B6A9847AB6DD806CC
:100680003AD4D9073AD41A073AD49C063AD4580631
:100690003AD419063AD49A073AD45B073AD495F873
:1006A000601095F8603085F864108B420DD0286D8D
:1006B00083685B6A03B19847286D414683681B6A6B
:1006C000984795F8603085F8643095F86440202CA0
:1006D0006DD0082C56D8002C51D0013C072C4DD899
:1006E000DFE804F06D5A4C5A4C4C4C1A084625F081
:1006F00080FA0028B6D0B9E71021D2E70121D0E76F
:100700000821CEE72021CCE74021CAE78021C8E7B5
:100710000221C6E70421C4E700244FF0040C202185
:1007200022462046234605F10808CDE9020CCDE912
:100730000013CDE904240023B5F85620B5F8541071
:10074000404630F0F0FC254B2B6786F0010385F81E
:1007500075301FB139462846FFF70EFF286D8368B4
:100760005B6803B198471E49404630F011FD3146A1
:10077000284606B0BDE8F04127F0E1BE002422463D
:10078000204607E0402C22D0802C4FF00004224667
:1007900020461FD023460EE0E86D01230024C0F35D
:1007A0004002C0439C46194600F00100BBE700220E
:1007B0000124104613464FF0020C1021B3E7002429
:1007C0004FF0030C1821224620462346ABE70024B5
:1007D00022462046012308219C46A4E73C00100045
:1007E000D405002410B50446002127F0A8FE04F12A
:1007F000080030F01DFD00232365014B236010BD70
:1008000008D9049010B50446006D78B125F0F1F9CF
:1008100060B10121204627F092FE074904F108004B
:1008200030F0B6FC012384F8483010BD2046BDE806
:100830001040FFF7D7BF00BFD4050024224B034070
:10084000062B2DE9F743064606D010F0030513D119
:1008500002681E4B9A4204D101A930460BF038FEC3
:100860000546DFF86C80DDF80490474657F8F04FF6
:1008700024B9162003F032FA0025F2E745B1636887
:100880004B4505D14A462168284636F00EFF18B17F
:10089000D4E90223B24213D1E3683B60D8F8EC30CC
:1008A0009C4202D10023C8F8EC30002340F22751CB
:1008B00020461A4627F07BFE0E2003B0BDE8F083E9
:1008C00004F10C071C46D3E70F0080FFF0C804902A
:1008D0000C2300242DE9F0410378064688462F2B8F
:1008E0000DD01A4BD3F8EC7057BB347884B127F095
:1008F00060F8164BD3F8F04024B9012408E0013623
:100900000127F2E76568013D05D1F71BC8F80070C3
:100910002046BDE8F08121682A463046013136F094
:10092000E1FE58B9735D72192F2B02D1C8F800206F
:10093000EEE71BB9064BC8F80030E9E7E468DBE7EF
:10094000C8F80000D3F8EC40E2E700BF0C23002415
:100950007330059010B586B0084B02AC00930423A9
:10096000019406F079F92146029827F03DFE2346CE
:100970000222762127F01BFE06B010BD80AF049046
:1009800008B50246084B586B13684168C1F31E0155
:100990008B4206D35B1A1360C268934203D322F0E2
:1009A000A8FE0068F1E708BD0C230024034B044AAD
:1009B0005A630022C3F8F420704700BF0C230024C0
:1009C000ACAF04902DE9F04781460F46002941D095
:1009D00027F064FE204B82465C6B0CB9204635E064
:1009E00094F907300025E668002B06F1FF3616DB88
:1009F000013604F11808B54215D32468EDE706EB7B
:100A000005083A4648464FEA580808F1060354F8E4
:100A1000231036F067FE0028CCBF45464646731BC0
:100A2000012BECD8E4E723695B5D9A4510D163693B
:100A30005B5D9F420CD13A46494658F8250036F096
:100A400034FE28B96068C0F31E002844BDE8F08772
:100A50000135D0E70120F9E70C2300242DE9F04708
:100A600080460E46FFF7AEFF0246002840F0918018
:100A7000FF2E03D94849494828F082FA484C751C92
:100A8000D4F8F40090B1D4E93E132B448B4229D919
:100A9000294427F080FE0746D8B90246D4F8FC1056
:100AA000D4F8F40027F077FEC4F8F470802D2F46B8
:100AB00038BF8027384627F060FEC4F8F400C0BB7A
:100AC000284627F05AFEC4F8F40088BB284602F0F6
:100AD00051F9D4F8F8302B44C4F8F830D4F8F43095
:100AE000002BE3D0D4F8FC304146D4F8F470324601
:100AF0001F442B4400253846C4F8FC3036F0A5FDD1
:100B000031463846BD5527F0C9FD636B8046D3E9B1
:100B100002A3534528D30C204FEA4A0900FB0AF0F0
:100B2000183027F022FE50B9C4F8F4004846CEE74A
:100B30002F460023C4F8F870C4F8FC30D2E700F167
:100B4000180202EBCA0202614A444261616B016011
:100B50004A68C968C2F31E02C5600A44416862F36C
:100B60001E01C0E901196063626BD2E9033202F829
:100B70000380991D626B5269D654626B42F82170F2
:100B8000616BCA680132CA60626B5268C2F31E02AE
:100B90001A441046BDE8F087D38705905CCE0490D8
:100BA0000C2300240346054A08460A601A7A0A7193
:100BB0005B688B600023CB60704700BFE8C5049082
:100BC000044B886008460B6001230B710023CB6047
:100BD000704700BFE8C5049010B5044904460C20D6
:100BE00029F073FD02224460027210BD00C6049019
:100BF0002DE9FF410C46054616461E4954F8047B74
:100C00008922384606F0FCF802AB214632460193B1
:100C1000681E194B0093022306F01EF8029C002266
:100C2000381D21469DF80C8008F0A0FF18B9214618
:100C3000124803F027F8D0E90065FC68B8F1000F0E
:100C400012D07A6800F1080122F007022244A2F1D2
:100C50000804521AD210D20036F005FD0E20C4E965
:100C6000006504B0BDE8F081021B214604F10800D4
:100C7000D210F0E7BCC604902CC5049058CF049065
:100C800010B50649044628F095F828B920460449CD
:100C9000BDE8104028F08EB810BD00BFBCC604905F
:100CA0008CC60490F0B5184B04460A7A85B00D4600
:100CB000012653F8221029F017FE14492046144F3C
:100CC00029F012FE134B00932B7A8DF804306B68D9
:100CD000029300230393684627F0A0FD054630B930
:100CE0000D49204605B0BDE8F04029F0FDBD1EB914
:100CF0003946204629F0F8FD0122294620460026E3
:100D000006F000FDE7E700BFDCC50490507F0590CA
:100D1000537F0590E8C50490034205902DE9F04FFC
:100D2000154685B004460846FFF7AAFF032D07467F
:100D30002CD00368364A93422BD1DFF8D890012596
:100D4000DFF8D4803549204629F0CEFD0023DFF8B6
:100D5000D0B003930123DFF8CCA003A93846019358
:100D600027F01DFD019B0646C8B92F49204629F0F2
:100D7000BBFD3A68264B9A4247D0032D45D02B49FC
:100D8000204605B0BDE8F04F29F0AEBDD4E9028998
:100D9000D8E7DA882046264929F029FECDE71BB995
:100DA0004146204629F0A0FD032D31682BD101EAF0
:100DB0000B03062B04D12A46204606F0A3FC17E0BD
:100DC0008B0708D10B681A7B2AB103EB82031A69DF
:100DD000184B9A42EFD05146204629F085FD3168E4
:100DE0002046032206F08EFC5146204629F07CFD69
:100DF0004946204629F078FD2A467168204606F0CB
:100E000081FC0023A9E70122D6E705B0BDE8F08FF9
:100E10008CC604902A9C0590537F05905A7F0590BC
:100E20000F0080FF5C7F05907E6E0590679C0590AB
:100E3000567F05901DCC0190F8B51446064608680B
:100E40000D46FFF71DFF07460CB127F004FD2246B3
:100E50006968381D08F08AFE034608B1406870B919
:100E6000022E05D1022C08D16968074802F00AFF5A
:100E7000A868012C00D15860F8BD0E20F9E7022CBB
:100E800004BF00225A60F7E758CF04901FB5FFF760
:100E9000F7FE044627F0DFFC6368072B04D84B22DB
:100EA0001249134828F07AF800222046019222794C
:100EB000510701A942BFC3F3DC0303F1FF330193E0
:100EC00027F06DFC08B922F014FC6368042202A923
:100ED000083B636003680293436803930023C0E9FF
:100EE0000023022007F058FC04B010BDC78605900F
:100EF00058CF049010B5044904460C2029F0E5FBB6
:100F000000224460027210BD00C6049010B504496E
:100F100004460C2029F0D9FB01224460027210BD66
:100F200000C6049010F003030CD10268117A31B1AD
:100F300002EB81021369044A9A1A5342534103F0A7
:100F4000010070470023FAE7811001902DE9F34773
:100F50001646074608680D46FFF792FE044627F03E
:100F60007AFC3168304A3846C90805F04DFE022F38
:100F700012D16F683846FFF7D5FF0146E8B12B68FC
:100F80009F4209D0002304F10408019301A9686875
:100F900027F005FC074640B9002504347368AB42CE
:100FA00031D80E2002B0BDE8F087012239684046F2
:100FB00008F0DCFD7B684360E8E7384604F1040A8A
:100FC00002F096FA8146484602F008FB0028E3D07A
:100FD000002102F08DFA804602F000FB07464046F1
:100FE00002F0FCFA0546404602F0F8FA0FB105B1EE
:100FF00010B10E4801F0D2FE01223946504608F0E9
:10100000B5FD4560DFE7B36853F8351003EBC5075E
:1010100039B1042905D00122204608F0A7FD7B68DC
:1010200043600135BAE700BF05000200FF8A059062
:1010300010B50C46FFF724FE00220430214608F0CC
:1010400095FD18B92146024802F01CFE406810BD0B
:1010500058CF0490024B40F8043B29F03BBE00BF40
:101060008CC6049038B505490546102029F02DFBA3
:1010700004462946FFF7EEFF204638BD8CC6049093
:101080002DE9F041804686B000200D4616461F46E9
:10109000FFF7E8FF0F4B0446C0F80080984502BFF9
:1010A000037943F00403037155EA06030DD03B684E
:1010B00007EB85023146019003A8029329F017FE41
:1010C00003AA01A9681CFFF741FF204606B0BDE84E
:1010D000F08100BFBCC60490F0B5064685B0084656
:1010E0000C461546FFF7CCFD162E074662D005D8F4
:1010F000022E10D0092E61D0002409E0242EFBD14D
:1011000000222946043008F031FD002842D11E2477
:10111000204605B0F0BDA20705F0030326D12268E2
:101120002C498A4222D1002BF1D1296891421FD14A
:1011300001A9CDE9013327F032FB064602A9284672
:1011400027F02DFB0446002E40D00028DFD0216878
:10115000306829F035FB0028D9D06168706829F023
:101160002FFB0028D3D001A93846E4E7002BCED1CD
:101170002A68194B9A42CAD17B686A685340072B88
:10118000C5D800230435029302A9384627F007FB8F
:10119000044608B93E24BBE700222168284608F02F
:1011A000E5FC0028B3D04168606829F009FB0028FD
:1011B000EAD1ACE7204627F06AFB0446074A02A9B9
:1011C0000220CDE90245FFF7C1FEA1E700289ED12C
:1011D000E0E700BFBCC604908CC60490F4C604903F
:1011E0002DE9F0410C4607460D680021606802F0C9
:1011F0007FF9022F064660688CBFA7680E27DFF8CC
:10120000448006F009FDA0B9FFF72CFF45450560B5
:10121000044608BF037900F1040504BF43F004034A
:101220000371304602F0DAF9014620B92046BDE8E4
:10123000F0814010E8E70122284608F097FC47605B
:10124000EFE700BFBCC6049010B50C461AB927F0F2
:1012500068FB0E200EE0042A0DD1FFF711FD0022DD
:101260002146043008F082FC18B92146034802F0F8
:1012700009FD406810BD27F043FBEAE758CF049012
:10128000044B054A9A6603F160029A620348F9F733
:1012900005BE00BF0C230024FCD80490B00C002431
:1012A00070B5044698B10A4DAB6A83B1FEF758FD9C
:1012B000AE6A46B10023012CAB6204D1FEF76AFD91
:1012C00030460CF0F9F8BDE87040FEF763BD70BD24
:1012D0000C230024024BC3E902011861704700BFD0
:1012E0000C23002408B5084AC31D106923F0070326
:1012F000D16803448B4204D944F2F671034802F0EA
:10130000C1FC136108BD00BF0C2300245CCE049017
:1013100038B504460D4627F010FB38B9284606F0CC
:10132000D5F92246C188024801F092FD38BD00BFC0
:10133000E09605907F289DBF024B185CC0F34000EB
:10134000002070477F7F05907F289DBF024B185C6F
:10135000C0F3C000002070477F7F05907F289DBFAD
:10136000024B185CC0F38000002070477F7F05901F
:101370007F289DBF024B185CC0F38010002070478F
:101380007F7F05907F2809D8064B1B5C13F00C0F5C
:1013900006D1A0F15F0358425841704700207047C2
:1013A000012070477F7F05907F289DBF024B185C0E
:1013B000C0F30010002070477F7F05907F289DBFFD
:1013C000024B185CC0F34010002070477F7F0590EF
:1013D00010B50549102029F078F9044604302AF0A8
:1013E000D3FB204610BD00BFA4CB04902DE9F74FDE
:1013F0001C4605460E469046A3079DF83CB0DDE925
:101400000C9A03D12268124B9A4201D022F071F952
:10141000A0685B4652464946000105F045F833682E
:101420000746834203D227F09DF9286037602D6874
:1014300052469DF838304946201DCDE900B52BF0C5
:10144000C3FAC8F80000284603B0BDE8F08F00BF1B
:10145000A4CB049008B5830703D102680A4B9A42D3
:1014600001D022F046F9836853B103F10042C1680C
:101470000133013A31F81220B2FA82F2C2EB0313BF
:10148000580040F0010008BDA4CB049037B5840794
:1014900003D10568074CA54201D022F02AF910F8C3
:1014A000044F0093134604F001022BF002FA03B03C
:1014B00030BD00BFA4CB0490C30707B503D54010CF
:1014C00003B05DF804FB01A904302BF0D9F908B191
:1014D0000198F5E70149024827F052FDCE860590B4
:1014E00078D004902DE9F0438046C80789B00C46B7
:1014F000164632D502AF4B10022201A902A82AF0EB
:1015000075FBF20733D502AD7310022201A902A8C0
:101510002AF06CFBB8F1200F02D0B8F1130F63D1A1
:101520006B68002B00F09F8038462BF02EFA0446A3
:1015300028462BF02AFA01462046EFF715FF014610
:101540000446F0F723F8002840F0128124F0030449
:1015500044F00204A4F1FF443CE0A10703D1226857
:10156000854B9A4201D022F0C4F8271DC9E716F036
:10157000030205D13168804B994210D1351DC9E76E
:10158000022A0CD17D4B3340062B08D038462BF075
:10159000FCF932460146404601F030F919E0784B3B
:1015A00078498B42DFD074498B42DCD076498B423C
:1015B000D9D076498B42D6D082B932689A420DD1C1
:1015C00038462BF0E2F933460146002240460CF043
:1015D0006FFB0446204609B0BDE8F0833246214641
:1015E000404605F0E9F8F4E7A8F109095FFA89F344
:1015F0001A2B00F29880FFF7EBFE0446B9F11A0FA0
:1016000000F2B880DFE809F04F55495B5B0E2127F7
:10161000B62DB63E724F55495B5B0E2127B62DB6EF
:101620003E727C002A46394604302AF011FD05A995
:10163000201D2BF025F90028CCD0059B5A0093EAF9
:101640004303C7D442F00104C4E72A4639460430B4
:101650002AF03AFDEBE72A46394604302AF0EFFE3D
:10166000E5E76B680BB902F043FB05A82AF08CFA9A
:101670002B463A4605A9201D2AF0A2FF05A82AF00C
:1016800088FAD4E76B68002BEDD005A82AF07CFA25
:101690002B463A46211D05A8EEE72A463946043076
:1016A0002AF050FDC3E72A46394604302AF0D7FD18
:1016B000BDE72A46394604302AF056FEB7E73046E1
:1016C000FFF7FAFE021E02DA314801F067FBB8F1BB
:1016D000190F04F10400394602D0B8F10C0F02D101
:1016E0002AF001FCA3E72AF05BFCA0E72B78DB07DC
:1016F0003FF54CAF2A46394604302AF01EFF96E7E4
:101700006B68002BAFD0FFF763FE211D06462B460A
:101710003A4604302AF054FF05A90220CDE90564B9
:1017200007F03AF855E7294638462AF073FBB8F136
:10173000040F1FD8DFE808F00308170D1200002877
:10174000ACBF1E243E2445E70028D4BF1E243E24FF
:1017500040E70028CCBF1E243E243BE70028B4BF4E
:101760001E243E2436E7002814BF1E243E2431E701
:10177000084C2FE700242DE7A4CB0490070080FF3E
:10178000B4DC049040DC0490F0C8049008D90490C4
:10179000AD8705900200400008B5830703D10268B9
:1017A000044B9A4201D021F0A4FF0430BDE8084068
:1017B0002BF0EBB8A4CB04902DE9F041174B0E466B
:1017C0001749884228D08288920504D401243060C9
:1017D0002046BDE8F081847C002CF9D000EB840029
:1017E000006902689A42ECD100F1080547680024BC
:1017F000DFF8308005EB8707AF42E9D92868830717
:1018000002D10368434501D021F073FF314604350E
:10181000FFF7D2FF0444EFE70024D9E70CCD049092
:1018200074CC04907CC70490CA88014929F0DFB8C1
:10183000FF7F059038B504460D460B4929F054F852
:1018400000226968204605F05DFF0849204629F01E
:101850004BF8A9682046002205F054FF20460449B1
:10186000BDE8384029F040B80C800590537F0590C2
:101870000A80059038B504461D460A4B08461146B5
:101880009C4204D0084B9C4201D021F032FF4FF023
:10189000021205F0B9F92146082028F016FF2B683E
:1018A000436038BD28C7049010C704902DE9F04765
:1018B000C36805460C461A680AB121F01AFF5B6836
:1018C000002BFAD1DFF82081DFF82091AB6873B1EB
:1018D000A28896050BD4E15C21B90F2B07D112F435
:1018E000C07F04D0EB6804221A60BDE8F087E37C77
:1018F000002B34D004EB83031869FFF713FB002897
:10190000DBD0E37C0022696804EB830309011869DA
:1019100041F00601043008F029F900B32B7C3BB1FB
:1019200042680020EB682968BDE8F04701F0E6BA9C
:101930002F49304B9942C0D02F4B9942BDD02F4BED
:101940009942BAD02E4B9942B7D04268EB689007C3
:1019500002D110688842C7D021462868E4E72B6886
:10196000F3B9A37C002BC0D004EB83031C6923686C
:101970004B4512D12646DFF88CA056F8047F04EBC5
:101980008707043756F8044FB74204F0030319D809
:10199000002B92D1236853458FD1444596D1A4E7BB
:1019A0002A7C002ADDD1A2889205DAD44445D8D019
:1019B0001869EA68696801F015FBEB681B68002B81
:1019C000CFD092E7002B7FF478AF236853457FF4A4
:1019D00074AF4445D6D021462846FFF767FFEB6831
:1019E0001B68002BCED080E774CC04900CCD049003
:1019F000DCC9049040DC0490A4CB0490F0C80490AF
:101A000008D904907CC704902DE9F043D2F80090E7
:101A10008FB006460C461546B9F1000F40F08C8099
:101A2000019005F053FE83889E0501D421F061FEEC
:101A3000019F26014A4646F0060607F10408314692
:101A4000404608F093F810B143682B6012E040F272
:101A500009339C4211D1754B09930AAB98E80700F2
:101A600083E8070009A826F012FF2860037943F0F5
:101A7000020303710FB0BDE8F0838DF82000CDE9BB
:101A80000605CDE9047404A83968FFF70FFF28683C
:101A9000002838D03B689B889C07EBD5644B654A8F
:101AA0009342C3D0644A9342C0D0644A9342BDD0AB
:101AB000634A9342BAD010F0030412D102689A42EA
:101AC0000FD109A927F021FB00680E2802D15D483B
:101AD00001F07AF901AB2246012101F0C5F9286035
:101AE000C8E709AAB72101F07DFA099B002BC1D0F4
:101AF00001980B9005F0EAFD09AA0C900021022044
:101B000027F06EFAEBE70E2CB4D0B72CB2D0D52C60
:101B1000B0D0B12CAED040F211339C42AAD009AA69
:101B20000E21019801F05EFA099B002BA2D009AAB0
:101B3000002101200B96E3E7016857688B8898071E
:101B40005ED5002302AA09A88DF83430CDE902330E
:101B5000CDE90964CDE90B32FFF7A8FE0298002811
:101B60004ED0334B334A93423FF460AF324A9342F4
:101B70003FF45CAF314A93423FF458AF304A93424E
:101B80003FF454AF820722D102689A421FD101A9C3
:101B900027F0BBFA019BCDE904676FB9022B7FF6F2
:101BA00069AF80680E283FF465AF04AB00220121C5
:101BB00001F05AF9002348E7012B7FF65BAF40683C
:101BC0000E283FF457AF04AB00220221F0E704AA2D
:101BD0005FB9B12101F006FA049B93B104AA39461A
:101BE0000120069627F0FCF9E4E7D52101F0FAF987
:101BF000049B8BB104AA00210220CDE90667F1E71E
:101C000057B921010222301D41F0060107F0AEFF55
:101C100000283FF42FAFCDE721010122301D41F014
:101C2000060107F0A3FF4760C4E700BF8CC604901D
:101C3000DCC9049040DC0490A4CB0490F0C804906C
:101C400008D90490088505902DE9F0478CB01368F9
:101C500014460190002B47D10746B80703D13A68D4
:101C6000454B9A4201D021F044FD7B6813F00306F6
:101C7000F9D1DFF808811A684245F4D1BA680A94AC
:101C80008DF82C60CDE90721A1F11102514251419B
:101C90009A7CC9000991F2B103EB82031969384BB0
:101CA0000A689A4223D10D46DFF8D8A055F8049F60
:101CB0004E4510D055F8041F8B07D4D10B6843450F
:101CC000D1D1514501D10136F2E707A8FFF7EEFD6A
:101CD0002368002BF7D02568002D46D0042D0DD1A8
:101CE000294B2360BB6863600CB0BDE8F087254BCF
:101CF0009942F0D007A8FFF7D9FDECE7234B244A1F
:101D00009342B0D0234A9342ADD0234A9342AAD003
:101D1000224A9342A7D015F0030612D12A689A42AC
:101D20000FD103A9284627F0F0F900680E2802D148
:101D30001B4801F049F801AB3246012101F094F84B
:101D4000206003AAB721284601F04CF9039B002B21
:101D5000CAD00198059005F0B9FC03AA06900021AD
:101D6000022027F03DF92060BEE7064907A8099543
:101D7000FFF79CFDB8E700BF50C704907CC70490F4
:101D80000CCD049074CC049070C70490DCC904900E
:101D900040DC0490A4CB0490F0C8049008D90490CF
:101DA000088505901C4BF0B51B5C89B000250446E6
:101DB00004930C230E4617460DEB03000593CDF854
:101DC00018D08DF81C50CDE902510968CDE90055B5
:101DD000FFF76CFD009B042B09D13A463169204680
:101DE00001F090FF03460D4A934202D100E01BB977
:101DF0000023184609B0F0BD6A4629460120029723
:101E000027F0EEF8242C0346EDD128F0B0FC002892
:101E10000CBF1E233E23E6E72A8005908CDC04904D
:101E2000244B70B50D4688B0195C002301AA064604
:101E300003A88DF81C30CDE903510B21CDE9051223
:101E40002968CDE90133FFF731FD019C042C07D14E
:101E50002969304600F0F4FE0446204608B070BD03
:101E6000CCB12046294627F0A6F8062E04460CD011
:101E7000082EF2D1C207F0D4830703D102680E4BBB
:101E80009A42EAD0002000F0DBFF05F077FD400029
:101E900040F00104E1E7062EDFD1B323296803A84F
:101EA0000493FFF703FD019B002BD6D16D0045F095
:101EB0000104D2E75C800590A4CB049070B5151E98
:101EC00088B00C464FF000030CBF1D211B2101AA56
:101ED000064603A88DF81C30CDE903410921CDE960
:101EE00005122168CDE90133FFF7E0FC019B3BB906
:101EF00035B91B23216803A8CDE90435FFF7D6FCCB
:101F00000198042816D1206906F050FE80B13DB139
:101F10002368D88826F0F4FB0146304628F0E4FC1C
:101F200045F080022169304605F0ECFB08B070BD39
:101F30002A46F7E728B1214627F03DF8002201465E
:101F4000F1E7204605F0C2FB2346C288304602492D
:101F500028F04DFDEAE700BF1580059070B5057AC1
:101F60001DB9C188044800F073FF00EB85042469A3
:101F7000A446BDE8704060477A8C0590134B144A24
:101F8000934273B5044601D121F0B3FB114A934249
:101F9000FAD0114A9342F7D0104A9342F4D0820704
:101FA00002D102689A420AD00D4E00252046012334
:101FB0006A4616F8011B01F0BBF8009810B1012029
:101FC00002B070BD0135032DF0D1F9E7DCC90490F2
:101FD00040DC0490A4CB0490F0C8049008D904908D
:101FE000278005902DE9F04F0D4689B01146834AB0
:101FF00028461C4604F008FE012D03D0032D07D00F
:102000007F4822E0206809B0BDE8F04F05F05EBBD4
:10201000206809F0FBFC7B4B7B4A07469342D4E9DE
:10202000018601D121F065FB784A9342FAD0784AC3
:102030009342F7D0774A9342F4D018F0030403D1C7
:10204000D8F800209A4202D0002000F0F9FE304675
:10205000FEF768FF0028F7D0404602AA01A94FF416
:10206000077906F0CFFCDFF8B0A12346DDE9015087
:10207000AB4208D103B30268557C15B102EB85026F
:1020800015690B231AE050F823209107DCD1116861
:102090005145D9D1117A19B9D188604800F0D8FEDC
:1020A0009188013301F0020449EA04098C0544BF18
:1020B00041F001019180DBE71D460A23002D18BF86
:1020C00001330533980026F053FB554BC0F800A0B0
:1020D00004464361534BA0F804908361524BC78080
:1020E000C361524B86630362514B4362514B83621F
:1020F000514BC362514B0363514B836003F1043373
:10210000C360092303744F4B43630A23C374019BC9
:102110006BB1012B4FF00B03837404BF029BD3F808
:102120000080C0F83C8015B10C2305644374002581
:10213000102204AF0021A9460DEB020035F0ADFAE4
:10214000B3689D4207D303A92046FFF735FB01285A
:102150002ED93D4879E7D6F80C804FEAC50B58F8E0
:10216000353008EBC50A0BB3042B1FD0A388DAF86F
:1021700004009B0706D4FFF701FF18B1A38843F0C2
:102180000203A3803A4640F21131DAF8040058F80D
:102190000B8000F027FF7B6843B1102026F0E2FAA5
:1021A000B860C0F80890C7F80C80BF680135C7E771
:1021B00000224FF4C371301D07F0D8FC054678B1FA
:1021C000436813F003020BD11B68D98840F2DE3359
:1021D000994205D1031D01211C48FFF74BFB6860A4
